:020000022000DC
:1000000000000420391F02000D520600855306002F
:100010000D5206000D5206000D52060000000000B1
:100020000000000000000000000000000D5206006B
:100030000D520600000000000D5206000D52060091
:10004000391E02000D520600B521020025210200D2
:10005000352102000D520600A11A02000D520600C1
:100060000D52060095210200A5210200091F020081
:100070000D5206000D5206000D5206000D520600EC
:1000800005260200191F02000D5206000D5206003F
:100090000D5206000D5206000D5206000D520600CC
:1000A0000D5206000D5206000D5206000D520600BC
:1000B0000D5206000D520600000000000000000076
:1000C0000D5206000D5206000D5206004521020099
:1000D000291F02000D5206000D520600D521020014
:1000E000C52102000D5206000D5206006D210200CE
:0800F000000000000D520600A3
:1010000040F8044B40F8045B40F8046B40F8047B64
:1010100040F8048B40F8049B40F804AB40F804BB54
:1010200040F804CB40F804DB6846704781F000418B
:1010300002E000BF83F0004330B54FEA41044FEABD
:10104000430594EA050F08BF90EA020F1FBF54EA58
:10105000000C55EA020C7FEA645C7FEA655C00F0F4
:10106000E2804FEA5454D4EB5555B8BF6D420CDDC5
:101070002C4480EA020281EA030382EA000083EA48
:10108000010180EA020281EA0303362D88BF30BDE8
:1010900011F0004F4FEA01314FF4801C4CEA11313E
:1010A00002D0404261EB410113F0004F4FEA03339D
:1010B0004CEA133302D0524263EB430394EA050F28
:1010C00000F0A780A4F10104D5F1200E0DDB02FA97
:1010D0000EFC22FA05F2801841F1000103FA0EF22B
:1010E000801843FA05F359410EE0A5F120050EF1F1
:1010F000200E012A03FA0EFC28BF4CF0020C43FA22
:1011000005F3C01851EBE37101F0004507D54FF02E
:10111000000EDCF1000C7EEB00006EEB0101B1F57E
:10112000801F1BD3B1F5001F0CD349085FEA3000C4
:101130004FEA3C0C04F101044FEA445212F5800FCF
:1011400080F09A80BCF1004F08BF5FEA500C50F16C
:10115000000041EB045141EA050130BD5FEA4C0C4F
:10116000404141EB0101013C28BFB1F5801FE9D2AC
:1011700091F0000F04BF01460020B1FA81F308BFCF
:101180002033A3F10B03B3F120020CDA0C3208DD9B
:1011900002F1140CC2F10C0201FA0CF021FA02F176
:1011A0000CE002F11402D8BFC2F1200C01FA02F1E6
:1011B00020FA0CFCDCBF41EA0C019040E41AA2BF0B
:1011C00001EB0451294330BD6FEA04041F3C1CDAD3
:1011D0000C340EDC04F11404C4F1200220FA04F0F3
:1011E00001FA02F340EA030021FA04F345EA03019D
:1011F00030BDC4F10C04C4F1200220FA02F001FA5F
:1012000004F340EA0300294630BD21FA04F02946E0
:1012100030BD94F0000F83F4801306BF81F4801179
:101220000134013D4EE77FEA645C18BF7FEA655CEC
:1012300029D094EA050F08BF90EA020F05D054EABE
:10124000000C04BF1946104630BD91EA030F1EBFC3
:101250000021002030BD5FEA545C05D140004941C7
:1012600028BF41F0004130BD14F580043CBF01F5BA
:10127000801130BD01F0004545F0FE4141F47001A0
:101280004FF0000030BD7FEA645C1ABF194610467B
:101290007FEA655C1CBF0B46024650EA013406BF7C
:1012A00052EA033591EA030F41F4002130BD00BF3B
:1012B00090F0000F04BF0021704730B54FF48064F8
:1012C00004F132044FF000054FF0000150E700BF79
:1012D00090F0000F04BF0021704730B54FF48064D8
:1012E00004F1320410F0004548BF40424FF00001C5
:1012F0003EE700BF42004FEAE2014FEA31014FEA08
:1013000002701FBF12F07F4393F07F4F81F0605156
:10131000704732F07F4208BF704793F07F4F04BFA1
:1013200041F40021704730B54FF4607401F000457E
:1013300021F000411CE700BF50EA010208BF7047DE
:1013400030B54FF000050AE050EA010208BF7047CF
:1013500030B511F0004502D5404261EB41014FF438
:10136000806404F132045FEA915C3FF4D8AE4FF040
:1013700003025FEADC0C18BF03325FEADC0C18BF23
:10138000033202EBDC02C2F1200300FA03FC20FA74
:1013900002F001FA03FE40EA0E0021FA02F11444C1
:1013A000BDE600BF4FEA4102B2F1E04324BFB3F50E
:1013B000001CDCF1FE5C0DD901F0004C4FEAC002CC
:1013C0004CEA5070B2F1004F40EB830008BF20F0B0
:1013D0000100704711F0804F21D113F13872BCBF6A
:1013E00001F00040704741F480114FEA5252C2F1BF
:1013F0001802C2F1200C10FA0CF320FA02F018BF08
:1014000040F001004FEAC1234FEAD32303FA0CFC5A
:1014100040EA0C0023FA02F34FEA4303CCE77FEAE9
:10142000625307D150EA01331EBF4FF0FE4040F433
:101430004000704701F0004040F0FE4040F40000E2
:10144000704700BF53B94AB9002908BF00281CBF24
:101450004FF0FF314FF0FF3000F036B9ADF1080C1E
:101460006DE904CE02F05AF9DDF804E0DDE902236B
:1014700004B0704770B54FF0FF0C4CF4E06C1CEA00
:1014800011541DBF1CEA135594EA0C0F95EA0C0F7A
:1014900000F0DEF82C4481EA030621EA4C5123EAED
:1014A0004C5350EA013518BF52EA033541F480111C
:1014B00043F4801338D0A0FB02CE4FF00005E1FBCF
:1014C00002E506F00042E0FB03E54FF00006E1FB19
:1014D00003569CF0000F18BF4EF0010EA4F1FF045C
:1014E000B6F5007F64F5407404D25FEA4E0E6D419C
:1014F00046EB060642EAC62141EA55514FEAC520AD
:1015000040EA5E504FEACE2EB4F1FD0C88BFBCF528
:10151000E06F1ED8BEF1004F08BF5FEA500E50F1D9
:10152000000041EB045170BD06F0004646EA01019F
:1015300040EA020081EA0301B4EB5C04C2BFD4EBD1
:101540000C0541EA045170BD41F480114FF0000ECA
:10155000013C00F3AB8014F1360FDEBF002001F038
:10156000004170BDC4F10004203C35DA0C341BDCB2
:1015700004F11404C4F1200500FA05F320FA04F084
:1015800001FA05F240EA020001F0004221F00041B8
:1015900010EBD37021FA04F642EB06015EEA430E2B
:1015A00008BF20EAD37070BDC4F10C04C4F120055B
:1015B00000FA04F320FA05F001FA04F240EA02000E
:1015C00001F0004110EBD37041F100015EEA430EDF
:1015D00008BF20EAD37070BDC4F1200500FA05F2FF
:1015E0004EEA020E20FA04F301FA05F243EA02037E
:1015F00021FA04F001F0004121FA04F220EA02008D
:1016000000EBD3705EEA430E08BF20EAD37070BDD2
:1016100094F0000F0FD101F00046400041EB0101B2
:1016200011F4801F08BF013CF7D041EA060195F094
:10163000000F18BF704703F00046520043EB03034E
:1016400013F4801F08BF013DF7D043EA060370473B
:1016500094EA0C0F0CEA135518BF95EA0C0F0CD046
:1016600050EA410618BF52EA4306D1D181EA03018C
:1016700001F000414FF0000070BD50EA410606BF86
:101680001046194652EA430619D094EA0C0F02D1CB
:1016900050EA013613D195EA0C0F05D152EA033610
:1016A0001CBF104619460AD181EA030101F000412E
:1016B00041F0FE4141F470014FF0000070BD41F077
:1016C000FE4141F4780170BD704700BF4A0011D25D
:1016D00012F5001211D20DD56FF47873B3EB62528C
:1016E0000ED44FEAC12343F0004343EA505323FA98
:1016F00002F070474FF00000704750EA013002D10D
:101700004FF0FF3070474FF000007047182A2DE966
:10171000F74F054621D0202A22D00A200423C5F8FD
:10172000002185F8040185F80531284600F098FA73
:101730000022034695F80541A24214D3DFF8DCC02D
:10174000DFF8DCE000EB840395F804210132B4EB10
:10175000820F1AD303B0BDE8F08F0C200623DEE71A
:101760000E200823DBE711F8044B03F8044B11F8B3
:10177000034C03F8034C11F8024C03F8024C11F827
:10178000014C03F8014C0132D4E795F80521B4FB74
:10179000F2FA02FB1A4913F8041C13F8038C13F82D
:1017A000027C13F8016C0192B9F1000F0BD11CF807
:1017B00008B01CF807801CF806701CF801601EF8C1
:1017C0000A108BEA0101D5F80021202A0CD1B9F1C9
:1017D000040F09D1DFF8449019F8011019F80880B6
:1017E00019F8077019F80660019AA21A043310F864
:1017F000229000EB820281EA090103F8041C51786F
:1018000088EA010803F8038C91784F4003F8027CC2
:10181000D278564003F8016C013495E7172C090083
:101820000C2C09002DE9F04F044685B0084600F065
:1018300017FA8946024680462146002043F0C3FC41
:10184000231D019304F11003012502932246214632
:10185000002311F82300324E305C01F823000133DD
:10186000042BF6D1019B01318B42F1D16179637870
:101870006170617A6171617B6172A17A6373A3782F
:10188000A170A17BA372A379A171E17BA373E3781B
:10189000E170E17AE173E179E172E37199F8043181
:1018A000AB4234D092F800B05678917892F803A009
:1018B0008BEA060081EA0A0380EA0307039356F0E5
:1018C000EBF98BEA00007840107086EA010056F0D0
:1018D000E3F946407E405670039856F0DDF94140EA
:1018E000794091708BEA0A0056F0D6F98AEA000A2C
:1018F000029B87EA0A07D77004329342D2D1284666
:1019000042462146013543F05EFCEDB29EE7424679
:101910002146284605B0BDE8F04F43F054BC00BF57
:10192000172C09002DE9F04F504C904603F00302AC
:101930009B101F2B04EB821489469E464C49A8BF7E
:101940004FF01F0E1C2B1D46A8BF1C2551F822204E
:101950006168033587B025EAE57529410192039155
:10196000E268A1688446294100202A41029004913E
:1019700005925CF8045B3F4A154225F0004111D105
:1019800006AA02EB810151F8102C002D40EA02005A
:10199000B8BF5242B8F1010849F8042BE9D107B0A9
:1019A000BDE8F08F344A154209D154F82120002BAC
:1019B000BABFCEF100018A4042FA0EF2E5E72F4AA3
:1019C000154214D110392E4A019E52F8212082FB73
:1019D0000616AEF10302002A44DA51426FF00042CB
:1019E00042FA01F7B742D0DB06FA01F2CDE74A042A
:1019F000B2F1006FB6BF4A0500210421B2F1005FC9
:101A0000B8BF92001F4EB8BF0231B2F1804FBCBFC9
:101A100052000131B242C7BF1B4F1C4E1C4F1D4E1E
:101A2000924687FB0ABA77685744924687FB0ABA00
:101A3000B7685744924687FB0ABAF768BA448AFBEC
:101A4000027236691644144A52F8212086FB02724B
:101A5000019ED20082FB0676104A52F82120AEEB9E
:101A60000202B8E746FA02F28FE700BF7C60090085
:101A70006C600900FCFFFF7FF0FFFF7FC0FFFF7F6E
:101A8000AC5F09009979825A63218510445F09008F
:101A9000A9BDA029585F09008C5F09006C5F09008F
:101AA0002DE9F04F00248BB0CDE90444664B674824
:101AB0006749012225461E6846B1D0F804631642E4
:101AC00004D01D601E680296029E144304338B42AC
:101AD0004FEA4202EFD15D4BD3F87C218AB100225C
:101AE000C3F87C21D3F87C310393039B4FF0A043D0
:101AF00044F00044D3F810350493564BD3F8103516
:101B00000593E3B2D3B1544F01260025344210D0DF
:101B1000AB0003F1804303F5C043D3F81005D3F8BD
:101B2000101557F8253023B1C1F30141C0F305204A
:101B300098470135082D4FEA4606E7D1002C7FDA99
:101B40000DF1200B00230893CBF80430DFF804914B
:101B50004FF0FF33069307930025404B0193A846AF
:101B6000019A12F9013F01925A1C50D0C3F3C200EE
:101B700000F128020DEB020C03F007011CF8102CF9
:101B8000CA40D707DCB203F03F0640D5324A1746B9
:101B90003244A40992F9282057F822A0BAF1000F84
:101BA0000AD1032C33D11BF800E001228A4042EA1B
:101BB0000E020BF8002001E0032CF4D01F2E8BBF87
:101BC00003F01F0333464A464FF0A04203F5E0738B
:101BD00052F823301CF8182CCA40D207C3F3014333
:101BE00005D5022B13D1032C0BD1214604E0032B86
:101BF0000DD1032C05D10221304630F0EFF901352B
:101C0000EDB2BAF1000F02D021463046D04708F1BC
:101C10000103022B4FF00108A2D18DB14FF0A04378
:101C20000499D3F81025D9F81035914202D10599BD
:101C3000994205D00492089ACDE90532099B8AE7BA
:101C40000BB0BDE8F08F00BF0061004000600040B5
:101C50002061004000030050086A00205F6A0020F5
:101C6000D0F80031103B102B07D8054A22FA03F3B5
:101C700013F0010F08BF002070470020704700BF1D
:101C8000010101002DE9F04F04468DB00846FFF731
:101C9000E7FF0D4601900246214695F8040143F006
:101CA00092FA95F80461231D013E099304F1100393
:101CB000F6B20A93627A637B6273627962726278C7
:101CC0006271A27A6370A378A270A27BA372A379D7
:101CD000A271E279A373E378E270E27AE271E27BC7
:101CE000E272E37325462246002312F8231051487E
:101CF000415C02F823100133042BF6D1099B013219
:101D00009342F1D1019A2146304643F05CFA002E0D
:101D100000F08C8095F80080AB780093404655F039
:101D2000BBFF029055F0B8FF039055F0B5FF6F78F8
:101D30000B90384655F0B0FF024655F0ADFF0490C9
:101D400055F0AAFF8246009895F803B055F0A4FF1D
:101D5000059055F0A1FF069055F09EFF814658462C
:101D600055F09AFF079055F097FF089055F094FFB3
:101D7000DDE9023183EA010C0B9B069983EA0C0C26
:101D800082EA0C0C8AEA0C0C81EA0C0C89EA0C0C35
:101D9000009980EA0C0C87EA0C0C81EA0C0C04997F
:101DA0005A404A4005998AEA02024A40089989EA5B
:101DB00002024A404240009988EA02024A408BEA05
:101DC00002026A70039A05995A408AEA02024A405E
:101DD00006994A40079989EA02024A40424088EA45
:101DE00002027A408BEA0C0C8BEA020B85F800C0E9
:101DF00085F802B0029A5340049A53408AEA030AD3
:101E0000089A89EA0A0981EA09035340584000996F
:101E10000A9B88EA000887EA08077940E9700435D8
:101E2000AB427FF477AF013EF6B243E70DB0BDE8B9
:101E3000F08F00BF0C2B090010B54FF08043D3F892
:101E40000443620707D54FF4847051F0D5FA10B1FE
:101E50001C4B1B689847A30606D54FF48A7051F0B7
:101E6000CBFA08B100208047600607D54FF48C708C
:101E700051F0C2FA10B1012000239847210608D57D
:101E80004FF48E7051F0B8FA18B10F4B00201B6858
:101E90009847E20508D54FF4907051F0ADFA18B1AB
:101EA000094B01201B689847A3050AD54FF492708F
:101EB00051F0A2FA28B1044BBDE810401B68022083
:101EC000184710BD886B00208C6B0020DFED0A7A6C
:101ED0009FED0A7ADFED0A6AA0EE277ADFED097A34
:101EE000E7EE007AB7EE007AA0EE267A67EE807A07
:101EF00087EE870A704700BF6BD30DBCBA132FBDA6
:101F0000AEE534BF75AA2A3E0248032200211CF028
:101F100091B800BF00B000400248042201211CF02B
:101F200089B800BF001001400248042202211CF0C1
:101F300081B800BF0040024008B54FF0E0236B4A73
:101F4000C3F8082DBFF34F8F694B6A4A6A498B4229
:101F5000C0F0BF80694B6A4A00219342C0F0BE8046
:101F60004FF08053D3F83021082A4ED14FF08042F1
:101F70000021C2F80C11C2F81011C2F8381502F590
:101F80004042D3F80414C2F82015D3F80814C2F85C
:101F90002415D3F80C14C2F82815D3F81014C2F87D
:101FA0002C15D3F81414C2F83015D3F81814C2F84D
:101FB0003415D3F81C14C2F84015D3F82014C2F815
:101FC0004415D3F82414C2F84815D3F82814C2F8DD
:101FD0004C15D3F82C14C2F85015D3F83014C2F8AD
:101FE0005415D3F83414C2F86015D3F83814C2F875
:101FF0006415D3F83C14C2F86815D3F84014C2F83D
:102000006C15D3F84434C2F8703547F049FD18B167
:102010003C4B3D4AC3F88C2647F042FD18B13B4B80
:10202000FB22C3F8182547F03BFD58B14FF0804222
:102030004FF08051D2F8E43ED1F8581261F3030317
:10204000C2F8E43E47F02CFD20B1314B4FF4007252
:10205000C3F840264FF08053D3F83031082B09D114
:102060004FF08043D3F80024D20744BF6FF0010241
:10207000C3F80024274AD2F8883043F47003C2F82A
:102080008830BFF34F8FBFF36F8F4FF01023D3F81B
:102090000C32DB0725D5204B0122C3F80425D3F8E9
:1020A0000024002AFBD04FF01022D2F80C3223F08B
:1020B0000103C2F80C32184BD3F80024002AFBD0DD
:1020C0000022C3F80425D3F80024002AFBD000F036
:1020D00069FB52F8040B43F8040B38E743F8041B80
:1020E0003BE70E4B0E4A1A6038F084FF00000200F6
:1020F00000200020B06A090084220020C0220020B5
:10210000EC790020005000404881030000F00040BE
:102110000090024000ED00E000E0014000200020BF
:102120000090D003014902483DF048BBCC6A002032
:102130000030004002494FF040203DF03FBB00BF5F
:10214000006B002008B50748D0F8183143B14FF4B0
:102150008C7151F049F9BDE80840034848F0E7BEEA
:1021600008BD00BF003002406C6A002008B5074877
:10217000D0F8183143B14FF48C7151F035F9BDE806
:102180000840034848F0D3BE08BD00BF00F002403D
:10219000906A00200149024849F0CABAB46A002096
:1021A000009000400149024849F0C2BAC06A0020CC
:1021B00000A000400149024854F028BF346B0020C1
:1021C000002000400149024854F020BF586B002015
:1021D000008002402DE9F04FBC4BBD4AD3F80013FC
:1021E000002385B01C4601201D4621FA03F6F607A0
:1021F0000BD552F8236046B100FA03F6344342F897
:102200002350BFF36F8FBFF34F8F0133192BECD1E6
:10221000E10738D5AD4B0122C3F81425C3F81025CA
:1022200000221546930003F1804303F51C3301326D
:10223000082A5D609D62F5D1A44BA6485D629D644D
:10224000C3F85851D3F80024D3F800140A43C3F854
:102250000024D3F80023C3F808239F4AC3F80423BB
:1022600000214FF4927249F031FF9A4A8DF80850DC
:1022700040231383138101214FF4807301A8ADF82B
:10228000043013F019FE14F4006F924D07D08F4BF9
:10229000D3F8A836A5F81631012385F81C31A2021F
:1022A00004F4800635D5894AD2F8143513F48073C6
:1022B00008D01EB1D2F80034DB0702D4082040F069
:1022C000C1FE0123814AD2F81015CF0540F14A81A1
:1022D00095F81C318BB1002385F81C31B5F8163107
:1022E0009BB24FF4E06203930121882301A8ADF86B
:1022F0000420ADF8083013F0DFFD744B4FF440724A
:10230000D3F820350293012101A8ADF8042013F081
:10231000D3FD7EB36D4BD3F8006440F201723240BE
:10232000F005C3F8002409D50121C3F82C1501A834
:102330004FF48063ADF8043013F0BEFD71050FD586
:10234000624B0122C3F808259A65D3F8002312F4E2
:10235000001208BFC3F854214FF40012C3F804233D
:10236000B20507D54FF4A063012101A8ADF80430F0
:1023700013F0A2FD23022ED5544BD3F88014D3F8CA
:102380008424D3F888E4D3F88CC4D3F89074D3F8B9
:102390009464D3F89804D3F89C3411F07F0FD2B230
:1023A00001D1052A17D04FF4C0688DF808108DF8B8
:1023B0000E00012101A8ADF804808DF809208DF8E8
:1023C0000AE08DF80BC08DF80C708DF80D608DF85B
:1023D0000F3013F071FD414B23403BB1BFF35B8FD6
:1023E0003F4B4FF000021A70BFF35B8F394FDFF89D
:1023F000DCB00026B8464FF0140AB14606F10C03D3
:1024000024FA03F3D80726D50AFB06B305EB4611D9
:10241000D3F80827D8F8003013FA82F3C8F8003050
:10242000B1F806C090B2082E1CFA82F24FEA4613A9
:10243000CA8000F0A480B8F80820824240F09F8053
:10244000CA88B8F8041092B2914240F2988016B946
:10245000244815F025F90136092E08F12008CDD1C0
:10246000214B2340002B00F09480184BD3F86C8450
:10247000C3F86C84BFF36F8FBFF34F8F14F4806485
:102480001CBFD3F88044D3F88064DFF848A01DBF98
:10249000C6F3C016C4F3C01486F0010626464FF0FA
:1024A00000094FF4E06B28FA09F1CA0703D4B9F127
:1024B000000F31D184B3054B142202FB09315FFABE
:1024C00089F0D1F80836DAF810100FE000700240F9
:1024D00000710240E03B00200514C001FCFB1F001E
:1024E000003D00204C7002400004000151FA83F1CD
:1024F000CAF8101005EB4911B1F816E05EFA83FC3A
:10250000A1F816C0B1F816C0BAF814E01FFA8CFC96
:10251000E6455ED940F076FD09F10109B9F1080FF1
:102520000AF1200ABFD100244FF0010904F1100381
:1025300028FA03F3DB0701D474B96EB105EB44123A
:102540006301D17A002955D0D288B98892B29142DC
:1025500050D9E0B240F076FD0134082C07F1200795
:10256000E4D116E0002B7FF4C8AE95F82131002BA2
:102570007FF4C3AE4FF40013C2F80833BDE62B441A
:10258000DA7A8AB94FF0E023D3F8F03DD90700D5C5
:1025900000BE1A4A1A4B136010460023536005B060
:1025A000BDE8F04F0AF01EB9DA88A8F8042083F8D5
:1025B0000B90DB888DF808609BB24FF4E06201213C
:1025C00001A8ADF8042003938DF8099013F074FC72
:1025D00041E7C98AADF804B089B260F07F00039189
:1025E00000218DF808008DF8091001A8012113F0D1
:1025F00063FC91E72B4483F80A90ADE73C70002020
:10260000C972070010B5074CD4F8003143B100235C
:10261000984720464FF48071BDE8104050F0E4BE6A
:1026200010BD00BF00000140022A2DE9F04159D140
:102630003B4B826883FB02423A4D846985FB04640C
:1026400022440A60DFF8F0C042688CFB0242364E3A
:10265000C46986FB047422444A60026883FB024218
:10266000046A85FB046422448A60304E026886FB5B
:1026700002422F4C056A84FB05752A44CA604FF05C
:102680006045426885FB0272C76985FB07E73A44EB
:102690000A61826884FB0272876986FB07E73A4415
:1026A0004A61426983FB02728A6102698CFB027291
:1026B000CA61C26883FB02720A62C36886FB032395
:1026C0004B62036985FB03238B62436984FB03230D
:1026D000CB620023C1E91033C1E90E33C1E90C33E9
:1026E000BDE8F081134B902404FB023202F1480E46
:1026F00002F18C0501F14406683250F8043B55F8AC
:1027000004795EF804CB1C468CFB048441F8044B2E
:1027100087FB0343AA4246F80439EED1E0E700BF45
:10272000D8E3CEB8281C3107CD3C410D9A615FC972
:10273000669EA0F6045D090033C3BEB200280CDB20
:102740004309064900F01F0020330122824041F86E
:102750002320BFF34F8FBFF36F8F704700E100E07E
:102760004309064900F01F0020330122824041F84E
:102770002320BFF34F8FBFF36F8F704700E100E05E
:102780000028ABBF00F16040054B00F5614000F050
:102790000F004FEA4111B4BF195480F8001370477D
:1027A00014ED00E0BFF34F8F0549064BCA6802F4F1
:1027B000E0621343CB60BFF34F8F00BFFDE700BF64
:1027C00000ED00E00400FA05014B1868704700BFF7
:1027D0005420002007EE900AF5EEC07AF1EE10FAD0
:1027E00001D400F009B808B580F0004000F004F80A
:1027F000404261EB410108BD70B5FEF77BFD0C4B1B
:10280000002204460D46FEF735FEFEF75FFF064642
:10281000FEF74EFD074B0022FEF72CFE02460B464C
:1028200020462946FEF706FCFEF750FF314670BDF4
:102830000000F03D0000F04170B510EE105A25F098
:1028400000440123B4F1FF4FB0EE403A0646036066
:1028500004D320EE003AB0EE430A70BD34B9DFED88
:10286000D07AB7EE007A87EE273AF4E7B4F1E45F66
:102870000BD2002DBEBF4FF0FF330360B1EE400A14
:102880001DF0EAFBB1EE403AE5E7002D80F2C6828A
:10289000B4F1964FE3D2B4F17A5F9FEDC25A78D289
:1028A000DFEDBF0A20EE050A002000F015FEF0EE75
:1028B000402AF5EE402AF1EE10FAD0D023EE220A9B
:1028C000B0EEC00A85EE000A1DF0C6FBF5EEC02A88
:1028D000F1EE10FAB0EE402A40F1B9804FF0FF332C
:1028E000B4F17E5F336000F09382B4F1804F00F06A
:1028F0008F82B1EE433A6B0000F1DE81AA4B9C421D
:1029000000F2F580B0EE430A1DF0A6FBA74B9C42F7
:10291000B1EE400A40F29D80B7EE007A37EE437A7E
:1029200067EE077ADFEDA26A9FEDA26A9FEDA23AF9
:10293000A7EEA66ADFEDA16AE6EE276A9FEDA06A20
:10294000A6EEA76ADFED9F6AE6EE276A9FED9E6A14
:10295000A6EEA73ADFED9D6AE7EE866A9FED9C6AD8
:10296000A6EEA76ADFED9B6AE6EE276A9FED9A6AFC
:10297000A6EEA76ADFED996AE6EE276A23EE073A2C
:10298000A6EEA73AF6EE007AA7EE673A33EE003AE3
:10299000FFE0B1EE407AB0EE470A18F09DF9B4EED0
:1029A000407AF1EE10FA19D0F6EE007A27EE277A87
:1029B000B0EE470A18F090F937EE400A30EE000A00
:1029C000F0EE407AFEEECF7A17EE903A062B39D829
:1029D000DFE803F02312121F1F2B2B00DFED807A9C
:1029E00077EEC37A17EE903A03F0010307EE903AC0
:1029F0009B00B8EEE70AE9E7F6EE007A37EEC00A88
:102A0000DFED670A20EE050A00F036FBF1EE402A02
:102A10004FE7F7EE007A37EEC00ADFED610A20EEED
:102A2000050A002000F058FDF0E7F7EE087A30EED6
:102A3000670ADFED5B0A20EE050A00F01DFBB1EE30
:102A4000400AE3E7F0EE007A30EE670AE5E701239B
:102A500046E7644B9C4264D99FED637A33EE477A34
:102A600067EE074A9FED616ADFED616ADFED615A4B
:102A70009FED615A9FED613A64EE877AE7EE866AD0
:102A80009FED5F6AA6EEA76ADFED5E6AE6EE276A53
:102A90009FED5D6AA6EEA76ADFED5C6AE7EEA65AD7
:102AA000DFED5B6AE5EEA76ADFED5A5AE6EEA75A5C
:102AB000DFED596AE5EEA76ADFED585AA7EEA55A91
:102AC000DFED575AE5EE275A9FED565AA5EEA75A65
:102AD000DFED555AE5EE275AE5EE876AA6EEE73AAE
:102AE000DFED527A94EE863A33EE673A4EE7504B7A
:102AF0009C4206D9B0EE007A37EE437A9FED280A61
:102B00000EE74C4B9C4206D99FED4B7A9FED240A71
:102B100033EE477AA4E7F7EE007A33EE673A9FED9B
:102B2000200A9FED467ADFED467ADFED466AE3EE56
:102B3000077A9FED457AA7EE837ADFED447AE7EED8
:102B4000037A9FED437AA7EE837ADFED4D7AE7EEC5
:102B5000037A9FED407AE3EE076A9FED3F7AA6EE97
:102B6000837ADFED3E6AE7EE036A9FED3D7AA6EEDB
:102B7000837AF7EE006AE7EE036A67EE837A87EE00
:102B8000A67AFEEE006AF0EE477AE3EE267A37EE9A
:102B9000803A002DBFF65FAE32EE433A5BE600BFEF
:102BA00000000000DB0F49406666663F1F4A3B3F5E
:102BB000A283D337679767393F239E3DA1549C3A40
:102BC0007E02F23B01F0893D752C3C384584E238A9
:102BD00034B6053AC66E3D3B1599A83C661AA53E2B
:102BE0000000004B07336D3E0C5BEC3E6B7BA53960
:102BF00076F4B7BA67F8663A85300DBA521CE631FA
:102C000007E7C73B474D06BD5EB9F73E27F9A3B9B5
:102C1000FE7771BB3D37933C3C2117BEF7E9AF39D6
:102C20009916143BFEFC28BC155A843DCDCDF83DC9
:102C300017A6DD3F1FA69D3FC316BB3F5E3C5B3C16
:102C400078756A3EAF72D53DB24B7A3FE73ABA3FEC
:102C5000F400223FDBD5523BDFEF443F2D390840E3
:102C6000BE2E1D4067FF0538B435F13ABDD7F536A5
:102C7000E440DA3CE6DC153E7ACCA63E5A245C3EC3
:102C80003F239EBDD6EE4B3A54BF983C6E0F303E6C
:102C9000C5D0383F3B2DB23FE8C4D5BAD23D5B3AF0
:102CA0005C061CBAFD0C503A610B36BBABAAAA3DC0
:102CB0001D7FD63E00000000B4F1824FF7EE002ADF
:102CC00075D2FDEEC35A1FED197A5FED196A1FED3B
:102CD000196AF8EEE57A15EE903A73EE677A033BDF
:102CE000E7EE876A1FED1E7AA6EEA77A5FED1F6AF0
:102CF000E7EE276A1FED207AA6EEA77A5FED216A3C
:102D0000E7EE276A1FED227AA6EEA77A5FED236A27
:102D1000E7EE866A1FED246AA6EEA76A5FED256AD4
:102D2000E6EE276A1FED266AA6EEA76A5FED276A20
:102D3000E6EE276A27EE277AE6EEA72A87EE223A02
:102D4000B6EE007AA7EE873A042B3FF622AFDFE813
:102D500003F02B2825220300B1EE087A37EE877A9C
:102D6000F1EE046A77EEA66A66EE876AB1EE007A43
:102D700037EE877A27EE267AB0EE080A37EE800A19
:102D800020EE070AB0EE007A77EE877A27EE800A07
:102D90001DF062F9FAE5B7EE007AE1E7F7EE006AB6
:102DA000E4E7B7EE007AE7E7B7EE000AEAE7B0EE4D
:102DB000430A1DF051F9B4F1B94F30EE620A24D242
:102DC000C2EE836A5FED4C5A1FED4C6A66EEA67A3E
:102DD000B6EE007AA7EEA56A5FED4F5AE6EE275AE7
:102DE0001FED506AA5EEA76A5FED515AE6EE275A2D
:102DF0001FED526AA5EEA76A33EE477A1FED543AEB
:102E0000A6EE263AA7EE003AC3E623EE003AC0E665
:102E10001FED583AC0E61FED593A1CE5B4F17E5F4C
:102E2000F9D0B4F1804FF6D01FED5E2A63E500BF04
:102E30007FB510EE105A834A25F0004393420446B2
:102E400005D8002380ED000A4360002022E07E4A7E
:102E500093423AD825F00043002DDFED7C7A7C4A7E
:102E600023F00F0318DD934230EE670A09BFDFED50
:102E7000797A9FED797A9FED797A30EE670A70EE74
:102E8000477A30EE670AC0ED007A30EE470A80EDEF
:102E9000010A012004B070BD934230EE270A09BF39
:102EA000DFED6C7A9FED6C7A9FED6C7A30EE270A3D
:102EB00070EE077A30EE670AC0ED007A30EE070A4E
:102EC00080ED010A4FF0FF30E4E7654A93426DD888
:102ED0009FED647AB0EEC00AF6EE007AE0EE077A73
:102EE000FDEEE77AF8EEE76A17EE900ADFED577A23
:102EF000A6EEE70A1F28DFED587A66EEA77A30EED5
:102F0000677A09DC5849461E25F0004251F8261020
:102F100022F0FF028A4207D117EE102AC2F3C752ED
:102F2000C2EBD352082A02DC84ED007A1BE09FED4D
:102F3000497AB0EE406AA6EEC76A70EE467AE6EECF
:102F4000C77A9FED467AD6EE877A36EE677A17EE25
:102F5000102AC2F3C752C2EBE353192B15DC84EDE0
:102F6000007AB0EE460A30EE470A002D30EE670ACE
:102F700084ED010A8EDAB1EE477AB1EE400A84EDB3
:102F8000007A84ED010A404284E79FED387AB0EE82
:102F9000460AA6EEC70A76EE407AE6EEC77A9FEDBD
:102FA000347AD6EE877A30EE677ABDE7B3F1FF4F19
:102FB00006D330EE400A80ED010A80ED000A44E7B6
:102FC000DA15863AA3EBC25307EE903ABDEEE77AE4
:102FD000DFED286AB8EEC77A77EEC77A8DED017A11
:102FE00067EEA67ABDEEE77AB8EEC77A77EEC77AD3
:102FF0008DED027A67EEA67AF5EE407AF1EE10FAE0
:10300000CDED037A19D1B5EE407AF1EE10FA16D073
:103010000223214601A800F089F8002DBFF63AAF3F
:10302000D4ED007AF1EE677AC4ED007AD4ED017A3E
:10303000F1EE677AC4ED017AA5E70323E9E70123FE
:10304000E7E700BFD80F493FE3CB1640800FC93FE9
:10305000D00FC93F004435374344353708A3852E88
:10306000800F494384F9223F5C56090000A3852E56
:1030700032318D240000804310EE103A23F00043DB
:10308000B3F1485FB7EE007A04D2FDEEC07A17EED6
:10309000902ABAB360EE006ADFED1C5A9FED1C6AFD
:1030A0001C4AA6EEA56A9342DFED1B5AE6EE265AAD
:1030B0009FED1A6AA5EEA66ADFED195AE6EE265ACA
:1030C0009FED186AA5EEA66A60EEC00A26EE266A93
:1030D000F6EE007AE6EE860A66EEA77A04D877EE78
:1030E000E07A37EE670A70470F4A93429ABF03F1BE
:1030F0007F4306EE903AF5EE026A37EE667A77EE97
:10310000E67AECE7B0EE470A704700BF4ED747AD0E
:10311000F6740F319999993E7CF293B4010DD03732
:10312000610BB6BAABAA2A3D0000483F2DE9F04F2B
:103130009246033A48BF0AF10402D7B0D2109B4628
:10314000551C2DB202910BF1FF31EB0080460DF1C1
:103150006809501A0BF1090CC24F0393AAEBC5057D
:1031600000EB0C064C460028AABF3B5CDFEDC17AA1
:1031700007EE903A00F10100A8BFF8EE677AB0427E
:10318000E4EC017AEFD142AF08EB8B0309EB8B043F
:103190000193BE46DFEDB77A26464046F0EC016A61
:1031A000019B36ED017A9842E6EE877AF6D101313D
:1031B0008C45EEEC017A04F10404EBD1A949DFED72
:1031C000AA6A9FEDAA6A531809240593A3000493E1
:1031D00056AB03EB840212ED140A07EB840006A938
:1031E0002246002A45DC284636F06CFAB0EE407ADA
:1031F000B4EE000A27EE000A17F06EFDF2EE007A38
:10320000A0EE677A002DFDEEC77A17EE906AF8EE11
:10321000E77A37EE677A3EDD06AA601EC5F1080E32
:1032200052F8203043FA0EF10E4401FA0EF1591A09
:1032300042F82010C5F10702114100293ADD0022B1
:1032400001360DF1180E1346944255DC002D03DDB6
:10325000012D62D0022D6AD002292BD1B7EE000ACF
:1032600030EE477A33B3284636F02CFA37EE407A00
:1032700020E060EE267A013AFDEEE77AF8EEE77A92
:10328000A7EEC60ABDEEC00AA1EC010A30ED010AA4
:1032900037EE800AA5E705D1621E06A951F8221073
:1032A0000912CAE7F6EE007AB4EEE77AF1EE10FA08
:1032B00020DA0021B5EE407AF1EE10FA40F0848079
:1032C000601E00230DF1180E082838DC002B56D1A3
:1032D0000FA9012251F8040DB0B3049B3E1D04EB6D
:1032E0000B01601C1E4409EB8101224490422DDD3C
:1032F00014466BE70221A2E7DEF8000053B920B1C3
:10330000C0F58070CEF80000012001320EF1040EED
:10331000034699E7C0F1FF00F4E704F1FF3E06A879
:1033200050F82E2002F07F0240F82E2094E704F19E
:10333000FF3E06A850F82E2002F03F02F4E75EF8A8
:10334000202001381343BFE70132C3E7059B1B5C14
:1033500007EE903AF8EE677A4446E1EC017ADFED49
:10336000457A8C46F4EC015A019B3CED017A9C4273
:10337000E5EE877AF6D1E6EC017A0130B6E7013C5A
:10338000083D06AA52F82430DBB12846B7EE000A01
:1033900036F098F99FED347A381D4FEA840800EB37
:1033A0008400234606AD002B3CDA2346002B63DB6A
:1033B000DFF8BCE0DFED2F7A07EB830C0025E01A85
:1033C00047E0013C083DDDE7039BB0EE470AA3EB75
:1033D0000A0036F077F99FED257AB4EEC70AF1EED0
:1033E00010FA19DBDFED207A60EE277A06AAFDEEEF
:1033F000E77A0835F8EEE77AA7EEC70AFDEEE77A36
:10340000BDEEC00A10EE103A42F8243017EE903AA2
:10341000013442F82430B8E7BDEEC00A06AA10EE27
:10342000103AF6E755F8232007EE902AF8EEE77AEF
:10343000013B67EE807A20EE070A60ED017AB2E781
:10344000FEEC016ABCEC017A01350A2DE6EE877AC2
:1034500001D08542F4DD56AA02EB800040ED287AC7
:10346000013BA3E7DC5609000000803B00008043DD
:10347000A4570900000000002FA81FED027A00EBFE
:1034800008032246002A17DAE1B1F1EE477A029BDF
:10349000C3ED007ADDED2E7A77EEC77A01239C42E8
:1034A00013DA09B1F1EE677A029B06F00700C3ED6B
:1034B000017A57B0BDE8F08F73ED017A013A37EE2B
:1034C000277ADFE7F0EE477AE1E7B0EC017A0133E3
:1034D00077EE877AE3E700BF10EE103A23F000435F
:1034E000B3F1485F04D2FDEEC07A17EE903A5BB3B9
:1034F00020EE007ADFED157A9FED156AA7EE276AB8
:10350000DFED147AE6EE077A9FED136AA7EE876A7D
:10351000DFED127A60EE076AE6EE077A30B99FEDCA
:10352000106AA7EE276AA6EE260A704767EEE67ACB
:10353000B6EE006AE0EE867AD7EE870ADFED097A0A
:10354000E6EEA70A30EE600A704700BFD3C92E2FFF
:10355000342FD7B21BEF3836010D50B98988083C9B
:10356000ABAA2ABEABAA2A3E10EE103A23F00042C4
:10357000B2F1465FF0EE407A14D2BDEEC07A17EE9B
:10358000101A29BB431C134306D1F0EEC07AB7EEE4
:10359000007A87EE270A7047012800F09B80BFEE73
:1035A000007AF6E74C498A4212D3002B9FED4B7A02
:1035B000B8BFF1EE407A37EE677ADFED497AB8BFEF
:1035C000F1EE600A77EEE07ADFED460A77EE877A71
:1035D00067EEA76ADFED445A9FED446A9FED445AB7
:1035E0003D4926EEA67A67EEA64AA7EE256A8A42EC
:1035F000DFED405AE6EE075A9FED3F6AA5EE876A77
:10360000DFED3E5AE6EE075A9FED3D6AA5EE876A6A
:10361000DFED3C5AE7EE055A9FED3B5AA5EE875A7F
:10362000DFED3A5AE5EE075A9FED395AA5EE875A73
:10363000DFED385AE5EE075AB0EE467AA5EEA67AE7
:10364000B0EE606AA7EE246A9FED337AE6EE260AB2
:10365000E4EE870A37EEA00A1DD307EE100AF8EE53
:10366000C76A60EE005A30EE260A9B1785EE806A24
:1036700003F00203C3F1010307EE103A36EE606A6D
:10368000B8EEC77A77EEC67AB0EE006AE7EEC66AA1
:1036900026EE870A704701281CD010EE103A6FF30F
:1036A0000B0306EE903A76EEE77A70EEE70AFFEE4D
:1036B000007A87EE807AF7EE007A17EE103A6FF311
:1036C0000B0300EE103AE6EE807AE0EE807AA7EE89
:1036D000870A7047704700BF40A12C3FDA0F493F6F
:1036E00068212233000000005FAE9BB745F4A33889
:1036F0008453D937C8261A3A16696B3BA427B33CC2
:103700008988083E7AC09538B937813948DEBE3A93
:103710001F37113CD10D5D3DABAAAA3E2DE9F04704
:1037200082B00646DDF828E00846B4460D46002B78
:103730004ED18A4214466DD9B2FA82F242B1C2F138
:103740002003954026FA03F394401D4306FA02FC39
:10375000260CA7B2B5FBF6F14FEA1C4306FB115548
:1037600043EA054301FB07F0984209D9E31801F148
:10377000FF3580F00381984240F2008102392344F2
:103780001B1A1FFA8CFCB3FBF6F006FB10334CEA55
:10379000034C00FB07F363450AD914EB0C0C00F152
:1037A000FF3580F0ED80634540F2EA80A4440238A2
:1037B00040EA0140ACEB030C0021BEF1000F04D045
:1037C0002CFA02F30022CEE9003202B0BDE8F08705
:1037D0008B4209D9BEF1000F01D0CEE90061002172
:1037E000084602B0BDE8F087B3FA83F11746002916
:1037F0004DD1834202D3B24200F20F81B6EB070CE7
:1038000060EB030301201D46BEF1000FDDD0CEE9C1
:1038100000C5DAE7002A00F098801A46B4FA84F36B
:10382000002B40F0AF800B1B270CA6B20121B3FB8D
:10383000F7F54FEA1C4007FB153340EA034306FB4C
:1038400005F8984507D9E31805F1FF3002D29845ED
:1038500000F2E8800546A3EB08031FFA8CFCB3FBDB
:10386000F7F007FB10334CEA034C06FB00F363450B
:1038700008D914EB0C0C00F1FF3602D2634500F2BC
:10388000CE803046ACEB030C40EA054095E7C1F131
:1038900020058B4022FA05FC4CEA030C00FA01F4E7
:1038A00026FA05F3E84002FA01F943EA04084FEA70
:1038B0001C4206FA01FAB0FBF2F71FFA8CF602FB83
:1038C00017004FEA184444EA004407FB06F0A04200
:1038D0000AD91CEB040407F1FF3380F09C80A0425E
:1038E00040F29980023F6444241A1FFA88F3B4FB23
:1038F000F2F002FB104443EA044300FB06F69E424A
:1039000009D91CEB030300F1FF3480F082809E4252
:103910007FD90238634440EA0740A0FB09749B1B2F
:10392000A3423E46A04664D361D0BEF1000F0AD048
:10393000BAEB060263EB080303FA05F5CA40154328
:10394000CB40CEE9005300213FE7730843EAC1733F
:103950004A08190C41EA02414FEAC67C9BB2B2FB0D
:10396000F4F02646A04627461F2243EA0143B1FB56
:10397000F4F1A3EB080341EA004158E72946FFE6CA
:10398000284615E71A46C3F120019C4026FA01F3A8
:1039900020FA01F190400343270C06FA02FCB1FB28
:1039A000F7F0A6B207FB1015190C41EA054100FB20
:1039B00006F58D423BD9611801D28D4220D8491BB2
:1039C0000138B1FBF7F5019505FB06F8019D9BB2A7
:1039D00007FB151143EA0143434526D2E31805F1DD
:1039E000FF31C6D24345C4D2A91E2344C1E7BA451C
:1039F0009BD2B7EB090664EB0C040138A04694E7B0
:103A0000651B29440238B1FBF7F5019505FB06F863
:103A1000DCE720467FE71F4666E70846F4E6A44455
:103A200002382FE7023D234415E70199A1E7491B1E
:103A3000B1FBF7F5019505FB06F8C7E72DE9F0475F
:103A40001C46436816461A791B6886B089460621CB
:103A5000C3F800151A4B9DF83870342101FB02336E
:103A600087F001070222804683F82D207F0154B998
:103A7000144DD8F804002EF01BFE284606B0BDE811
:103A8000F0473BF079BEB4F5806F4FF00003A246DB
:103A90003A4628BF4FF4806A01A94046CDE902A307
:103AA000CDE904638DF804308DF8059000F09EFB9D
:103AB000044B98420546DCD1A4EB0A045644D6E7F1
:103AC000CC6A00200000AD0B074A00231168814238
:103AD00001D1184670470133082B02F10402F5D1D9
:103AE0004FF0FF30704700BF14600020034B53F8C5
:103AF000203013B19A6801329A607047DC3A002096
:103B000038B5144B53F82040ECB120792EF098FAD8
:103B1000054660792EF094FAA2790F49E37940EADC
:103B2000450000F0030040EA8202A0718A5C134461
:103B300094F908205BB29342E37105DBE36801333B
:103B4000E3600023E37138BD52429342FBDCE3683B
:103B5000013BF5E734600020AC1A09002DE9F04F75
:103B60000546A7B08A46014600204AF04CF909AC48
:103B7000002841D1CDE913000CAA7E21284622F06D
:103B800053FFA94B0F9301224023CDE9102316AB1D
:103B900012930FAB0E93A54B09940A9300260820AD
:103BA000CDE9050648F05DF907902046CDE90366AA
:103BB0008DF8206047F017FEDFF880B237463546B3
:103BC0009DF85490B9F1000F13D0204647F00BFE3A
:103BD000B9F15D0F00F092804AD8B9F13A0F3BD8A5
:103BE000B9F11F0F14D8B9F10A0F31D8B9F1080F84
:103BF000E6D88F483CF0CCF90121284622F006F99E
:103C000043680A93002309950B938DF85430C5E758
:103C1000A9F12002D2B20123934013EA0B0F40F026
:103C20000F81844A1340CBD1B9F1220FE1D1069321
:103C30009DF854100029DCD0222940F0A4802046B1
:103C400047F0D1FDDDE9061025F0E2FA81462CE0CF
:103C5000B9F10D0FB4D0CCE7B9F15B0FC9D1002099
:103C60001BF0FAFE8146002D3AD04FF0010821E00A
:103C7000B9F1740F70D039D8B9F1660F4FD0B9F1DE
:103C80006E0FB6D19DF85430752BB2D1204647F057
:103C9000AAFD6C28ADD1204647F0A5FD6C28A8D11F
:103CA000204647F0A0FD4FF00E09002D00F00E81D8
:103CB0004FF00008604B9F4240F0F580494628468F
:103CC00049F02FFEB8F1000F3FF47AAF049B002BB0
:103CD00040F0F780012101A825F070F8049B1D60D9
:103CE000484624F083F94D46074669E7B9F17B0F52
:103CF00000F0D580B9F17D0F7FF47BAF002D3FF44C
:103D000078AF039B002B00F00081013B049A0393E2
:103D100052F82350284624F069F9074650E79DF8E9
:103D20005430612B7FF465AF204647F05CFD6C2872
:103D30007FF45FAF204647F056FD73287FF459AFFC
:103D4000204647F050FD65287FF453AF204647F0EA
:103D50004AFD4FF01E09A8E79DF85430722B7FF4FE
:103D600048AF204647F03FFD75287FF442AF20461C
:103D700047F039FD65287FF43CAF204647F033FD1E
:103D80004FF03E0991E75C290CD1204647F02BFD0E
:103D90007528014606D86D2808D8622840D06628C4
:103DA00008BF0C2105A853F036FC35E0A0F16E03E6
:103DB000072BF7D801A252F823F000BFDD3D020027
:103DC000A53D0200A53D0200A53D0200253E0200E2
:103DD000A53D0200E13D0200E53D02000A21E1E7C8
:103DE0000921DFE74FF000084FF00409204647F0B3
:103DF000FAFC40F02000A0F130025738D2B2C0B235
:103E0000092A88BF0246B9F1010942EA0818EDD132
:103E1000414605A853F011FC204647F0E4FC07E7B3
:103E20000821BFE70D21BDE7FC08080099B706008F
:103E3000ECE6070001100004680808000020FF03FA
:103E4000002306939846494605A853F0E4FB9DF8E5
:103E50005490B9F12E0F17D009F0DF03452B13D082
:103E6000B9F12B0F12D0B9F12D0F0FD048463BF00E
:103E7000D7FF024650B9DDE90610B8F1000F09D0AE
:103E8000134649F02EFFE1E64FF00108204647F0C7
:103E9000AAFCD8E743460A2227F070F8D6E60020AD
:103EA00025F02EF8DEE62EB9B8F1000F7FF4A1AEB2
:103EB0004E4685E631464A46284649F077F90026BF
:103EC00000E7294601A849F02CFD09E7BAF1000FE7
:103ED00011D0B9F1000F3FF48CAE039B002B7FF49F
:103EE00088AE05A853F00EFC484627B0BDE8F08F19
:103EF000204647F078FC9DF8545028463BF0A4FF3C
:103F00000028F5D1002DE4D073E6A946BAF1000FE0
:103F1000F1D0E2E7C20713B5044603D5C0F347006A
:103F200002B010BD830707D102680E4B9A4203D13D
:103F300024F04AF8C0B2F3E7204649F0BFFC48B18C
:103F4000204623F0C9FFFCEEC07ACDED017A9DF842
:103F50000400E5E7204624F049F85E22C1880248C3
:103F60003CF00AF8F0E407000FF10700F8B5284B21
:103F70001D68284B1B681A68012151641B68264A7A
:103F8000D3F844650023146814B12179814230D0FC
:103F90000133082B02F10402F5D1F8BD6369A06971
:103FA000E289218AEB1A89B211FA82F2301AA189C8
:103FB000B2FBF1F7C3EB034303444FF6FF7001FB81
:103FC00017228342A16828BF034621F81230238AB2
:103FD000A2899BB2934203D2238A0133238214E045
:103FE000E3899BB20133B3FBF2F102FB1133E381AE
:103FF0000BE0E379002BD1D02EF022F8637900F0AA
:104000000100834201D00023E3716561A661C4E72A
:10401000806F00203470002014600020242B2DE9D4
:10402000F047884601D8012B06D1FEF7CDFB1623B9
:1040300003600020BDE8F087344E0D46294615F890
:10404000014B375D17F00807F8D12D2C10D12C78D3
:1040500001278D1C33F0100115D1302C0DD129789A
:1040600001F0DF01582908D16C78023510230AE0ED
:104070002B2C04BF2C788D1CECE7002BF6D1302CB8
:1040800014BF0A23082307F1004E0EF1FF3E002162
:10409000BEFBF3F90E4603FB19EAA4F1300CBCF1A8
:1040A000090F10D86446A3421EDDB1F1FF3F07D0CF
:1040B000B14516D301D1A24513DB06FB034601210E
:1040C00015F8014BE9E7A4F1410CBCF1190F01D837
:1040D000373CE8E7A4F1610CBCF1190F04D8573C58
:1040E000E1E74FF0FF31EBE74B1C05D122230360E2
:1040F000764632B930469DE707B17642002AF9D0BC
:1041000009B105F1FF38C2F80080F3E7AD69090095
:104110002DE9F043344E86460D46284615F8014BEE
:10412000375D17F00807F8D12D2C10D12C78012716
:10413000851C33F0100015D1302C0DD1287800F0FB
:10414000DF00582808D16C78023510230AE02B2CA8
:1041500004BF2C78851CECE7002BF6D1302C14BF63
:104160000A2308234FF0FF380026B8FBF3F803FBBF
:1041700008F96FEA09093046A4F1300CBCF1090FC7
:1041800010D86446A3421EDDB6F1FF3F07D080453C
:1041900016D301D1A14513DB00FB0340012615F81E
:1041A000014BE9E7A4F1410CBCF1190F01D8373CF0
:1041B000E8E7A4F1610CBCF1190F04D8573CE1E722
:1041C0004FF0FF36EBE7731C06D12223CEF8003008
:1041D000304632B9BDE8F08307B14042002AF9D039
:1041E00006B1691E1160F5E7AD6909002DE9F74FC9
:1041F00080460D46019251F0EEFDD8F80430AC4FE8
:1042000001225A72D8F804301E791C68342303FB4B
:104210000677002387F82E30EB6803F06043B3F194
:10422000005F81468B4607D0A248D8F804300022B0
:104230005A7203B0BDE8F08F9F4BC4F8083397F86B
:104240002F3003F0FF0A23B1BB689C48C4F8043345
:10425000EBE787F82F20AE46BEE80F0007F10C0C05
:10426000ACE80F00DEF80030CCF8003087F830A062
:104270006B78C4F888354FF4827120464FF0B4F85B
:104280004FF4927120464FF0AFF8C4F850A5C4F82F
:1042900040A52B78032B00F2B380DFE803F0729A7D
:1042A00052022B6903F06043B3F1005FBCD14FF4BD
:1042B0008073C4F800326B68EA68C4F844254FF490
:1042C000A871C4F8483520464FF08EF84FF4B0710D
:1042D00020464FF089F84FF4A47120464FF084F83F
:1042E00001232362A360D4F85031002BFBD04FF49C
:1042F000A87120464FF078F8AB682A69C4F84425C5
:10430000C4F848356A4B342202FB06336C4A9A6083
:104310004FF4827308226B4F2978654D03291CBF27
:104320000121A15034227243A918AA58002A79D039
:104330008B68C4F80433634B9F4200F0A880624846
:1043400073E76B68EA68C4F84425C4F848352B69FC
:1043500003F06042B2F1005F7FF466AFAA68C4F870
:1043600034354FF48453C4F83825C4F80032504B28
:10437000342202FB063340F202229A6001232362B8
:10438000C6E701996B68EA68C4F84425C4F8483563
:104390003422474B89B102FB06334FF48071C4F8D5
:1043A0000012474A9A604FF4A47120464FF01CF85F
:1043B0004FF4A47301222262ACE702FB06334FF4F0
:1043C000007140F20222C4F800129A604FF4827326
:1043D000F0E76B68EA68C4F83425C4F838354FF460
:1043E0008053C4F80032324B342202FB063340F2D1
:1043F00002229A600123236200224FF482738AE72B
:10440000314F4FF48273082286E7D4F8242152B149
:104410004FF4927120464EF0E7FF0123236263615F
:104420004FF4827323441A68002AEED03422D4F861
:10443000C434C4F8C43402FB0651002281F82F2092
:104440008BB1224A224813F0010F08BF104613F027
:10445000020F02F5803218BF104613F0040F1D4BF7
:1044600018BF1846E1E620463EF050FE00287FF4D3
:1044700062AF1648D9E651F0AEFC814574EB0101FC
:1044800009D2D8F80430144800225A72D1E619F53E
:104490007A794BF10004D8F804305A7A002AEAD12C
:1044A0009B7A042B96BF0D4A084852F82300C0E6B9
:1044B000CC6A00200A00AD0B02029C010B00AD0B80
:1044C000000204000000AD0B0400AD0B0100AD0BB9
:1044D0000000AE0B0200AE0B0700AD0B101A090076
:1044E00008B510EE103A23F00042B2F17E5FF0EE14
:1044F000405A10D308D19FED2F0ADFED2F7A002B01
:10450000B8BFB0EE670A08BD70EE405ADFED297AF9
:1045100087EEA50AF7E7B2F17C5F11D2B2F14A5FEC
:104520009FED266A42D920EE000AFDF7CFFCDFEDB1
:10453000247AE0EE657A75EEE75A36EE650AE2E730
:10454000002BB7EE000AF6EE007A14DA75EE805A08
:1045500025EEA70AB1EEC06AFDF7B8FCDFED197AC7
:10456000E0EE067A9FED150A77EE867A30EE670A5E
:1045700030EE000AC7E730EE650A20EE270AB1EEFA
:10458000C05AB0EE407A15EE103A6FF30B0305EE09
:10459000903AA5EEE57A75EE257A87EE276AFDF763
:1045A00095FCA0EE056A36EE250AE1E7B0EE460A74
:1045B000A9E700BF00000000DA0F4940DA0FC93F49
:1045C0006821A2336821A2B308B510EE103A5A0050
:1045D000F0EE407A0FD4B7EE007A70EE477ABDE87D
:1045E000084037EEA77AA7EEA77AB1EEC70A37EEF2
:1045F000800A1BF085BC23F00043B3F18B4F13D22C
:10460000FFEE006AE0EE006ABDE80840B1EEE67A2F
:10461000F7EE006A37EE007A86EE870AB0EE007A8F
:1046200097EE870A1BF018BD1BF016FDDFED027A2E
:1046300030EE270A08BD00BF1872313F30B589B08F
:10464000084611461A4602AB0193194B0093032307
:1046500047F097FE1749029D0C2049F0BDF99DF8DF
:104660000C30037245609DF810300446EBB12846CB
:104670000CF0F4F8606805AA4FF4826122F0D4F9D6
:10468000237A5B0043F0010305AA00210120079370
:1046900047F0B8FF49F01EF90546606842F06FFF29
:1046A0001DB9217A04483BF07BFC204609B030BD9F
:1046B000841A0900745E080080F6070010B58EB0F9
:1046C00003AB51F8044B0193194B009301380323BA
:1046D0001DF0B8FD40F22A41606806AA22F0A4F954
:1046E000237A5B0043F001030893039B099340F690
:1046F00026130A93049B5B0043F001030B93059B75
:104700006FF0004293421FBF40F2E6425B000C9202
:1047100043F0010314BF0221012106AA4FF0020059
:1047200018BF0D9347F06EFF0E200EB010BD00BFF6
:104730006C1A090010B58EB003AB51F8044B01930D
:10474000194B0093013803231DF07CFD4FF4A66143
:10475000606806AA22F068F9237A5B0043F001033F
:104760000893039B099340F626130A93049B5B006E
:1047700043F001030B93059B6FF0004293421FBF70
:1047800040F2E6425B000C9243F0010314BF0221A9
:10479000012106AA4FF0020018BF0D9347F032FF27
:1047A0000E200EB010BD00BF541A090010B596B00F
:1047B00003AB51F8044B01932D4B009301380623B2
:1047C0001DF040FD09AA606840F2315122F02CF939
:1047D000237A5B0043F001030B93039B0C93049B30
:1047E0000D9343F666630E93059B5B0043F0010354
:1047F0000F93069B6FF00042934235D05B0043F06D
:10480000010343F63662119310920923032116AA7D
:1048100002EB830243F2565042F8340C16AA02EB24
:104820008300079A520042F0010240F8302C089AA7
:104830006FF00040824210D016A800EB830043F2D4
:10484000265440F82C4C16A800EB8303520042F08B
:104850000102013143F8282CC9B209AA032047F00C
:10486000D1FE0E2016B010BD07230221CFE700BFF6
:10487000241A0900F0B58BB0084611461A4603AB5E
:1048800001931B4B0093072347F07BFDDDE9036099
:104890000E2816D010F0030203D10168154B99427F
:1048A0000CD023F0A3FBC388009313484FF4BF73CD
:1048B0004FF484724FF421713BF05EFB012142F012
:1048C000F3FF0E49182049F087F89DF820409DF825
:1048D00024109DF81C50069F049A9DF8143005730F
:1048E000C0E9016744738173026103750BB0F0BDC9
:1048F000341B090078590800B8FB0700585E08000F
:1049000030B58BB004466A464068244D4FF49D6133
:1049100022F08AF800216A46084647F073FE48F004
:10492000D9FF002831D060686A4640F29E2122F00B
:104930007BF842F2A6530293A3685B0043F00103A5
:10494000039344F226030493237B5B0043F00103AB
:10495000059343F666730693637B5B0043F00103A4
:10496000079342F246621123CDE9082304216A46E7
:10497000002047F047FE23690E2B03D0217D5868A5
:1049800042F07EFF60680BB030BD07F067FFAB6A96
:10499000002BBFD0012021F061FBBBE7946B00200E
:1049A0002DE9F0418AB0084611461A4605AB01933D
:1049B000234B0093052347F0E4FC0522059802A948
:1049C00021F0D2F9039EA6F11002102A03D81D4B44
:1049D000D340DB0702D41C483BF0DAFA069C022CD9
:1049E00004DC002C04DC19483BF076FA062CFAD1E2
:1049F0000798DDF80880A0B9074615494FF48A707A
:104A000048F0EAFF089B80F80C41C0F810313246AC
:104A10003B464146054642F06AFE28460AB0BDE8DC
:104A2000F081012202A921F09FF90028E4D0039827
:104A300040F2511210211DF0A9FC029FDDE700BFDA
:104A4000DC1A09000101010020F707004DF50700FD
:104A5000145E080070B588B003AB51F8045B019395
:104A6000184B0093013802231DF0ECFB052203983C
:104A700005A921F079F9069CA4F11002102A03D8A7
:104A8000114BD340DB0702D410483BF081FADDE93B
:104A9000040640B9034628462246314642F027FE26
:104AA0000E2008B070BD012205A921F05DF9002893
:104AB000F0D0069840F2511210211DF067FC059BC2
:104AC000E9E700BFCC1A09000101010020F7070047
:104AD00010B50446084648F0DEFB022804DC002836
:104AE00004DC04483BF0F8F90628FAD184F80C01FC
:104AF0000E2010BD4DF5070038B51C46084611467E
:104B00004FF002121DF066FB206840F2FA3152F0BD
:104B100017FD0A490446082048F05EFF6379054600
:104B20001BB940F2FA301DF07FFB20792DF026FAF8
:104B300020790BF035FD6C60284638BDE45D080037
:104B400008B5406842F084FBBDE808409FED010ACB
:104B500024F040BA3333534070B5064640683C4DAC
:104B600042F076FB3B4A002303212B80C2F8F0156C
:104B70000121C2F8F435C2F8001519461A0102F1F4
:104B8000804202F5E0420133082BC2F81415C2F846
:104B90001015F3D12F4C4FF49053C4F818357368A7
:104BA00001265B79C4F814354FF48071C4F81035D0
:104BB0002046C4F82C56C4F830664EF015FC4FF46D
:104BC000827120464EF010FC4FF4847120464EF066
:104BD0000BFC4FF4867120464EF006FC4FF48A71B0
:104BE00020464EF001FC2660D4F80031002BFBD0AB
:104BF00018484FF480714EF0F7FB01236360154CA9
:104C0000D4F80431002BFBD012484FF482714EF0DF
:104C1000EBFB0123A360D4F81431002BFBD00D482B
:104C20004FF48A714EF0E0FB0023C4F80035C4F85D
:104C30001435C4F810352B881BB223EAE37318131C
:104C400040EA830080B2400040F0010070BD00BF28
:104C50004C700020007000401C4608B50846114604
:104C60004FF002121DF0B6FA40F2FA31206852F00D
:104C700067FC0449042048F0AFFE0348E9213BF0FB
:104C800033F900BFC85D080093FC07001B2808B576
:104C9000014604D103212DF081F9012008BD144AF9
:104CA00000231078884206D108462DF087F908467F
:104CB0002DF0A8F9F1E70133082B02F10102F0D140
:104CC000282901D00E2904D10A4B1B78002BE4D1EE
:104CD000EAE70D29E8D00929E6D00F29E4D00A290E
:104CE000E2D02A29E0D01529DED00020D6E700BF87
:104CF000EA170900C87700202DE9F04F2DED088B49
:104D00008FB009AB01936D4B009305231DF09AFA08
:104D1000002109982AF0F8FD002180460A982AF01F
:104D2000F3FD044600210B982AF0EEFDE379012BF8
:104D300005460AD1C379012B07D1A268012A04D9FB
:104D40008368012B01D99A4202D05D483BF020F9DB
:104D50006621D8F808004EF02AFAE669277905900E
:104D6000394630464EF0B2F9A368A069013B00FB1A
:104D700003603946B0EE40AA4EF0A8F90C98EE69EF
:104D80000E28F0EE40AA28D1297930464EF09EF93F
:104D90000D980E28F0EE408A22D1A868AB692979D7
:104DA000013803FB00604EF091F9EB690493D8F8E9
:104DB0001C300293059BD4F81CB0DB690393B0EE62
:104DC000409A4FF00009D8F808304B450BD80598A9
:104DD0000FB0BDEC088BBDE8F08F23F07DF8D7E76E
:104DE00023F07AF8E1E7029898F804104EF06EF993
:104DF000029AD8F81830B4EEC0AA1A44F1EE10FAAC
:104E0000B0EE408A029252DCF4EEC0AAF1EE10FA43
:104E100050D4A668D4F818A02179013E0027F31BCE
:104E2000012B32D80AFB07B006914EF04FF90699D4
:104E300006FB0AB0F0EE40BA4EF048F9AB69049AAE
:104E40002979079103FB0720F0EE409A06934EF074
:104E50003DF9049A069B079906FB0320B0EE40BA81
:104E60004EF034F938EE6B8A30EE4B0A79EEEB9A5D
:104E700028EE008A88EE290A30EE0B0A039BA3EC89
:104E8000010A039309F101099DE707EB530303FBB3
:104E90000AB0079106934EF019F9069B0799B4EEF4
:104EA000C80AF1EE10FAB4BF1F461E46B7E7B0EECF
:104EB000680AE3E7B0EE490AE0E700BF185B0900C3
:104EC00006EC07002DE9F04F2DED048B87B003AB06
:104ED0000193504B009303231DF0B4F90398002174
:104EE0002AF012FD8368012B044640F28C80C679BB
:104EF000012E02D048483BF04BF800792AF088FD9B
:104F000081460498E5690E2857D000212AF0FCFC60
:104F1000C779012F834603D1A26883689A4201D0E2
:104F20003E48E8E700799FED3E8A2AF071FD82460F
:104F30002846DBF81C80C847A3694046EE18F0EE0F
:104F4000408AD047DBF81830B0EE409A9844A56804
:104F5000BD4211D86B1E00EE103AF6EE007A28EE34
:104F6000278AB8EE400A20EE080A07B0BDEC048B91
:104F7000BDE8F04F24F02EB83046C847A36940463C
:104F8000F0EE409A1E44D04778EEA98A30EE499A56
:104F9000F0EE486AD9EE286ADBF8183007EE907A0E
:104FA000B8EE677A9844C6EE877A0137B0EE409A39
:104FB00038EE278AF0EE698AC9E705989FED188ACE
:104FC00022F08AFF2846B0EE409AC847A568F0EE66
:104FD000408AB54202D828EE098ABBE732462179D9
:104FE000E0694EF03AF807EE906A78EE808AB8EE03
:104FF000677A78EEC88A0136C8EE877AF0EE408A82
:1050000038EE278AE5E7074807B0BDEC048BBDE81A
:10501000F08F00BF005B090072E607007CE6070026
:1050200000000000020080801E280CD03E280AD01C
:1050300010F0010307D1820707D10068044BC31A9F
:10504000584258417047012070471846704700BFCA
:10505000F0E40700044B0548D3F8042500210123A0
:1050600002F500422DF0CCB90010014018130900E0
:10507000F0B51B288DB006460C46154672D03CD8BC
:105080000E2800F09C8004D8042840F2B58000244B
:1050900030E01028FBD115F0010206D115F0030312
:1050A000F5D12968704A9142F1D1284648F0F3F8C9
:1050B0000122054609A9204600F024F9102E0A9F76
:1050C0003DD12179002240201DF0E8F9A3686B430F
:1050D00000FB03F1E06846F0E5FEA368E0606B4387
:1050E000A360636803F0FF0363601DB1013DC31952
:1050F000002F34D120460DB0F0BD1D28CBD0242880
:10510000C5D1012203A9284620F02EFE002860D038
:10511000A10712D12268554B9A420ED1012209A94A
:10512000204600F0EFF801230093DDE90901DDE9F5
:10513000032345F0DBFE00285CD11E24DAE7A168DA
:105140009DF82C00694300F035F9C3680446CFE7A9
:10515000184609993A4646F078FF013DC319002DDB
:10516000F6D1C7E70A68424B9A4290D009A90122BA
:10517000204600F0C7F806A90522284620F0F4FDD5
:105180009DF82C10002240201DF088F9A168079D91
:10519000B5FBF0F5064629449DF82C0000F00AF90D
:1051A0000446DDE90912C06846F04FFFE0680A9B3B
:1051B000069905FB06F2184446F047FF9AE70A688D
:1051C0002B4B9A423FF463AF2946204640F068FDDE
:1051D00090E7EA0702D500203AF07EFEAB0703D144
:1051E0002A68214B9A42F6D0284648F067FB0028EF
:1051F000A3D0F0E73E247DE7012209A9204600F074
:1052000081F8012206A9284620F0AEFD002894D09E
:105210000B9A012A21D05A2A21DC20320146089B10
:10522000012B1ED05A2B01DC203301469342D2D1F0
:1052300023F00203642BCED0022E01D00029CAD065
:10524000079B0093DDE90912069B304648F08AFE71
:10525000002814BF3E241E244CE74222DDE7002133
:10526000DDE74223E0E700BFF0E40700FC080800A8
:105270001C080800F0B5012885B007460E4608D086
:105280008B0727D10B681C4A934202D01B4A9342DA
:1052900020D1012201A9304620F066FDD0B1394667
:1052A000002240201DF0FAF8029BB3FBF0F100FB56
:1052B00001F5AB4202D012483AF06AFE384600F0DF
:1052C00079F8019904462A46C06846F0BEFE204699
:1052D00005B0F0BD304623F053FD58B145102946C6
:1052E000384600F067F82B463A463146044640F00F
:1052F0001DFDECE70546F2E70CFE0700FC08080080
:1053000058F1070070B50D460179044601F07F01A0
:105310001646402000221DF0C1F8E3682B60A26809
:1053200042436A60227902F07F02AA602168094A3A
:1053300091420BD194F90420002A01DBB20707D473
:105340006268C2F3172200FB02332B60002070BD9D
:105350000120FCE71C080800074BC1E900300023CE
:10536000C1E90233054B02689A4202BF4368C3F3A6
:1053700017238B6008467047781008001C08080047
:1053800038B50D461C4611462846094A1CF022FF36
:10539000206824F029FF012D007804D1BDE83840B1
:1053A000002100F007B86168BDE83840FFF762BF30
:1053B000040002007828F8B505460E4602D10F48D1
:1053C0003AF0E6FD0022014640201DF067F80C4B44
:1053D0000C490746012D18BF1946102048F0FCFA69
:1053E0000571436803F0FF030446C0E9013606FB7C
:1053F00007F046F054FDE0602046F8BDB9F1070023
:1054000008100800FC08080070B50A79012A054652
:105410000C460DD1184948F0DAFCD4E9022128469F
:1054200026F096FC28461549BDE8704048F0CFBCF0
:10543000134948F0DBFCA368002BF3D01149284640
:1054400048F0C5FC0026A368B34204D80E4928469C
:1054500048F0BDFCE6E71EB10C49284648F0B7FC11
:105460003246E16820791DF0F1F801220146284614
:1054700024F03AF80136E6E7AA800700838907009E
:10548000B6800700C180070054D40700A8D50700E4
:105490002DE9F04F044687B00D4616460AB900259F
:1054A000D0E011F003078068DFF82CA240F0DF8025
:1054B0000B68814A934240F0DA806A4648F0E0FD8A
:1054C00010B97E483AF008FD2179042E01F07F01E1
:1054D0003A464FF0400000F096801CF0DFFF16F0D7
:1054E0000302054655D131688B7B002B42D001EB7E
:1054F00083031869724B98423CD13179402001F006
:105500007F011CF0CBFFA84202D06E483AF040FD6C
:1055100033685345D6E9028B38D17368C3F3172932
:1055200005FB09F9DDE900062368E768361A5345EB
:10553000A8EB06062FD194F90430002BAFDA002E29
:10554000E3D16368C3F3172305FB037705FB08F278
:105550000BEB090105FB007046F0A2FD0199A26862
:10556000009B521A08EB03006A4305FB017105FB1F
:10557000007039E0544B99420BD1012DC5D1052261
:1055800003A9304620F0F0FBDDE903B84FF0000935
:10559000C8E74E4896E7002ED8DD6368B6EB132FB8
:1055A0002FD9A16831446943384646F07BFC6368D3
:1055B000E06066F31F2382466360BB4508BF8346F5
:1055C0000098A268019940443244121A6A4301FBD0
:1055D00005A105FB00A046F063FD009805FB08F25D
:1055E0000BEB090100FB05A046F05AFD6368C6EB12
:1055F000132262F31F236360A3683344A3600E2564
:1056000020E0BA46DCE71CF049FF2168009B5145C9
:1056100006461BD1B3F1807F03DB2D492D4851F0A5
:10562000DBFD102048F0D8F9054694E80F0085E826
:105630000F00009A02EB112363F31F216960019BA5
:105640009B1AAB60284607B0BDE8F08F019920791E
:10565000C91AFFF7AFFEDDE90032E168D21A05464C
:10566000724306FB0311C06846F0EFFCEAE7002333
:105670002A460146206820F095FB236853450246E0
:1056800020790ED16368042E02EB13220BD003069F
:105690007FF505AFE168334600F07F001DF0CEFADC
:1056A000ADE7042EF6D1E16800F07F0007B0BDE859
:1056B000F04F1CF0CBBF00BF4C07080013E90700F8
:1056C000915402006DEB07000CFE070030F207005A
:1056D000D0EA0700200308001C08080010EE102A7A
:1056E00008B522F00043B3F17E5FB0EE406A12D3FA
:1056F00019BF76EE467A9FED1F7ADFED1F7A9FED98
:105700001F7A12BF87EE276AE0EE077AB0EE676A6B
:10571000B0EE460A08BDB3F17C5F0BD2A3F50003DF
:10572000B3F1645FF4D320EE000AFCF7CFFBA0EEE8
:10573000066AEDE7B0EEC06AB7EE000A30EE460A40
:10574000F6EE007A20EE270AB1EEC06AFCF7BEFB47
:10575000002ADFED0B7AA0EE066AB0EE007AE6EEE4
:10576000077A9FED066A36EE676AB8BFB1EE466A01
:10577000CEE700BF0000000000008003DA0FC93F41
:105780006821A2B31FB58DED010A019B23F00042F1
:10579000B2F18B4F00EE102A4FEAD3700AD31AF001
:1057A0005BFCDFED1E7A30EE270A08B1B1EE400A4D
:1057B00005B000BD5B0014D5B7EE007AF0EE476A85
:1057C000E0EE006AF1EEE67A77EE807AC7EE276ABD
:1057D000F0EE007AE0EE276AB0EE660A1AF03CFCC2
:1057E000E3E7B2F1665F10D320EE007AF7EE006ACD
:1057F00037EE266AF1EEC67A77EEA67AC7EE276A0A
:1058000036EE800A1AF07CFBCFE7DFED057A70EE0A
:10581000277ACDED037A039BC7E700BF1872313FAB
:105820000000807B08B5044B1A68044B9A4202D0F2
:105830000D2033F0B1F908BD009C0320EF29780159
:105840001FB50446E0B10E281AD04FF0102300799E
:10585000D3F80C32DB0703D5A0F10903012B02D9E1
:105860002FF068FD60B940F2C713039301A92046E9
:1058700003AB02AA16F0D0FD039902483AF090FB60
:1058800004B010BD42FC0700F4EE400AF1EE10FA3D
:1058900010B5F0EE407A04D770EE207AB0EE670AC9
:1058A00010BD10EE902AB2F17E5F03D1BDE810402A
:1058B00000F082B810EE103A940F04F0020444EAAB
:1058C000D37433F0004308D1022C59D09FED317AC4
:1058D000032C08BFF0EE477AE0E732F0004209D12E
:1058E000DFED2D7A9FED2D7A14F0010F08BFF0EE59
:1058F000477AD3E7B2F1FF4F10D1B3F1FF4F04F174
:10590000FF3407D1022C3ED8254B03EB8403D3EDA3
:10591000007AC3E7022C39D8224BF6E702F1506136
:105920009942DDD3B3F1FF4FDAD0A10703D503F1DC
:10593000506393420CD387EEA00AB0EEC00A00F089
:105940003BF8012CF0EE407A04D1F1EE407AA5E765
:10595000DFED157A022C0AD0002C9FD09FED137A30
:1059600077EE877A9FED127A77EEC77A96E79FED0A
:105970000F7A77EE877A9FED0E7A77EE677A8DE76A
:10598000DFED0B7A8AE7DFED0B7A87E7DFED067A4A
:1059900084E700BFDB0F49C0DB0FC9BFDB0FC93F86
:1059A0003056090024560900000000002EBDBB330C
:1059B000DB0F4940DB0F493F10EE102A22F0004375
:1059C000B3F1994F82B04FEAD2700ED3B4EE400AD1
:1059D000F1EE10FA07D69FED410ADFED417A00287B
:1059E00018BFB0EE670A02B070473E498B420BD831
:1059F000B3F1665F5AD212F0FF4FF4D160EE007A35
:105A0000CDED017A019BEEE7374A9342F0EEC07A82
:105A100037D8A2F5D002934229D8F0EE006ABFEE43
:105A2000007AA7EEA67A002377EEA67A87EE270AF9
:105A30005A1C60EE006A9FED2D6ADFED2D7ADFEDD6
:105A40002D5A26EEA67AE7EE067A9FED2B6AA7EE90
:105A5000876ADFED2A7AE7EE257A67EE877AE6EE47
:105A6000267A67EE807A24D130EE670ABBE7B7EE7C
:105A7000007A77EEC76A77EE877A012386EEA70A67
:105A8000D6E71F4A93420BD8F7EE086AB7EE007AC2
:105A9000A7EEA67A022337EEE66A86EE070AC7E784
:105AA000BFEE007A87EE270A0323C1E74FF0FF33EA
:105AB000BEE7144A144902EB830201EB830393ED22
:105AC000007A77EEC77A37EEC00AD2ED007A37EE69
:105AD000C00A002887D0B1EE400A84E7DA0FC93F38
:105AE000DA0FC9BFFFFFDF3EFFFF973F25AC7C3DCC
:105AF0000DF5113E4712DABDA9AAAA3E98CA4CBEBE
:105B0000FFFF1B404C5609003C5609002DE9F84F99
:105B1000D1F800800128064640468CBF01F1040BF5
:105B20004FF0000B0F46914623F05AF830B940462B
:105B300022F05CFAC18827483AF01EFA06F1FF3AD3
:105B4000B9F1000F2DD0D9F80050C5F3DC051AEBE0
:105B5000050404D02C44A00046F083F9044600223A
:105B6000924520D804EB86000022954221D11A4E9E
:105B7000DFF868903168D9F800000131090146F07A
:105B800091F93368C9F800005A1C32601A0100EB21
:105B9000031340F802A0C3E90158DC603868BDE88F
:105BA000F88F4D46D3E75BF8223044F822300132BB
:105BB000D6E7D9F80830083053F8323040F80C3CBA
:105BC000D9F8083003EBC20301325B6840F8083CA7
:105BD000CBE700BF45FB0700646100205C6100204B
:105BE000F0B50023DFF838E00C4E19460E27DEF83A
:105BF0000020934201D30E20F0BD346804EB031261
:105C00004FEA031C9568854208BF44F80C1003F165
:105C1000010304BFC2E90117D160E8E75C6100201D
:105C20006461002038B590F82330FF2B044629D05A
:105C3000154B01225A600022C3F8002590F8263047
:105C40009B0707D590F821002CF098F994F82200D2
:105C50002CF094F9FF2594F8210032F0B3FF94F86A
:105C6000220084F8215032F0ADFF94F8230084F82C
:105C7000225032F0A7FF054B84F8235000221A600F
:105C800037F086F80E2038BD00500240FC69002035
:105C90002DE9F04788B0084611461A4602AB019339
:105CA000434B0093062346F06CFB9DF81C70029852
:105CB0004FF418710FB33CF02DFB40F2275105460D
:105CC00003983CF027FB40F2B2210446049851F0BF
:105CD00037FC40F296318246059851F039FC35493F
:105CE0008046282047F07FFE0646B8F1000F0DD011
:105CF000314840F296313AF0F7F851F021FC40F289
:105D000027510546039851F01BFCDCE72B4BD3F8D9
:105D10000080B8F1000F02D029483AF013F918605A
:105D200028799DF818900AF03BFC20790AF038FC9D
:105D30009AF804000AF034FC96F8263067F3410321
:105D400086F826301F4B2A7986F82120C3F864256F
:105D5000227986F82220C3F868259AF8042086F86C
:105D60002320C3F8702507B3287941462CF016F993
:105D7000207941462CF012F90122124B0121C3F87F
:105D800004254F400022C3F80825C3F80C15C3F8BA
:105D90001075C3F81C15C3F82025C3F8249537F0F7
:105DA00011F8304608B0BDE8F0873A46E5E700BF95
:105DB0001C1C0900985D080093FC0700FC6900208A
:105DC0009DF807000050024010B5044690F82300EB
:105DD00041F038FA20460AF033FE10B905483AF08F
:105DE000B1F894F8263043F0200384F826300E20D2
:105DF00010BD00BF28F607002DE9F04F0D4685B015
:105E000055F8044B064694F82300174641F01AFA59
:105E100002AB0193664B0093701E294602233A465B
:105E20001CF010FA2046029D9DF80C600AF008FE56
:105E300058B1604A0123536094F8263043F00803B8
:105E400084F826302023C2F80833284625F0F6FAD5
:105E500094F82630656066F3861384F826302A7B32
:105E60006968544FD20884F82520AB7BE87B6D7BB2
:105E700084F82450003B18BF0123DB0143EA0023D0
:105E8000E08C013A03F4C07320F4C07018BF012203
:105E90000343E384C7F81C2594F824305A1E534268
:105EA0005341C7F8283594F8263013F002033DD04B
:105EB0000B4694F82500638394F8243048435843F4
:105EC00000014FF47A73B0FBF3F0033020F00300CD
:105ED00080B2208345F0E3FFA060208B45F0DFFF18
:105EE000E060606840F069FE0023C4E9043384F890
:105EF000203094F8263023F03C0343F0040320467E
:105F000084F8263016F0A8FF228B2A4B9208C3F89B
:105F100050252022C3F804230122C3F800251A606B
:105F200016F07CFF0E2005B0BDE8F08F2248DFF8A8
:105F30009090B7EE007A9E4698461E46D7F81C25EC
:105F4000012A01D182793AB307EE901A1B4AD0F8A0
:105F500000B0B0F904C099FBFCFCF8EE676A02F1EE
:105F6000580A55689CFBF5F507EE905AF8EEE77A6B
:105F700076EEE77AF0EEE77A87EEA66AB4EEC76AC5
:105F8000F1EE10FA05D5D2F800E0B0EE467A2B46D5
:105F9000D84608329245E4D10136092E00F10800B6
:105FA000CCD1044AC2F81885C2F814E581E700BFD5
:105FB0000C1C090000500240C41B09006C1B0900A6
:105FC0000048E80110B5044690F8230041F03AF982
:105FD000064A0123536094F8263043F0080384F8FE
:105FE00026302023C2F808330E2010BD0050024096
:105FF00038B5084B1B6800220446C3F80025FF256E
:10600000007932F0DFFD6079257132F0DBFD6571DA
:106010000E2038BD142100202DE9F0432DED028B18
:106020008BB0084611461A4603AB01933E4B0093D2
:10603000072346F0A6F94FF42371039851F080FA34
:1060400040F2B3210746049851F07AFA9DF81850AF
:106050006A07064604D040F26121344839F0A0FFB7
:106060009DF820305B0702D040F2EA31F5E709984D
:10607000DDF814809DF81C9010B321F02DFFB0EED8
:10608000408A40F2A64201210020B0EE480A46F0C4
:106090008DF92749082047F0A6FC044638790AF014
:1060A0007FFA30790AF07CFA84F806903A79227106
:1060B00033796371B8F57A5F05D01E4839F068FF0F
:1060C0009FED1D8ADDE7102D01D01C48F6E71C4B23
:1060D000DFED1C7A1B681C49C3F840256279C3F8C0
:1060E000442528EE278A4FF00462C3F804250022D5
:1060F000C3F82025FCEEC87A2822C3F81825C3F877
:106100001C250122C3F8002517EE900AC3F860157C
:10611000C3F864251A601FF0E3FE20460BB0BDEC07
:10612000028BBDE8F08300BF4C1C0900C4FB0700D4
:106130007C5D080028E90700AE47E13D40E9070023
:106140001421002000007A44E86100202DE9FF417D
:106150001446074600790D4641F06EF801A9204625
:1061600021F00CFF48B9204621F040FF5E22C38891
:10617000344840F2823139F0FFFE019C40F2823215
:106180000021204646F034F9AB0706D12A682E4B91
:106190009A4202D12D4839F09FFE062201A92846D5
:1061A0001FF0E2FD9DF80C10029D002240201CF023
:1061B00075F9B5FBF0F5A54202D2254839F0E8FEA5
:1061C000039B482B01D02348F8E7DFF89480019D1A
:1061D000D8F800300122C3F80825C3F86055C3F889
:1061E00064451D4B4FF4485043F001039847D8F8DD
:1061F00000300022C3F80821184AC3F860250122A4
:106200002E46C3F86425D8F80030D3F808316BB1B6
:1062100005EB4405B5420CD1BB7983B124F00104F0
:10622000640044F0010004B0BDE8F08106F016FB04
:10623000E9E73388A3F5004326F8023BEAE724F0B8
:106240000304EDE7AEFB0700F010090020F907009A
:10625000A1F807003BEF0700901C0900E86100204F
:10626000142100202DE9F04F2DED028B89B0426BF7
:10627000079390F83030B3FA83F35B0980F830303D
:106280000A33044650F82370037BDB08B2FBF3F8B3
:10629000436C0193836C5B080493C36C0393BA460D
:1062A000B8F1000F0FD194F83030079A0A3301206B
:1062B00054F823301360626B149B1A6009B0BDEC74
:1062C000028BBDE8F08FE36B4BBB94F8413033B9E0
:1062D00094F84030ABB1606D98B140F06EFC606DE9
:1062E00060B104F13C0204F1380140F022FC0228C4
:1062F0000AD100236365E36384F84130617B0D02BA
:1063000016E000236365EAE7227BE36BD208B3FB68
:10631000F2F3E363431E5842584184F84100617B25
:10632000636D0D02002BE9D0E36B9D4228BF1D4633
:10633000454528BF45466068B5FBF1F189B234F0A8
:10634000B1F804F1200037F08BF8F7EE007AB4EEE4
:10635000E70AF1EE10FA30DD04F1200037F080F8A2
:10636000FDEEC07A17EE909AF7EE000A04F12400D1
:106370009FED5F0A4FF001FE04F11400F0EE408A39
:1063800037F06EF8D4ED067A94ED077A77EEC07A9E
:10639000F0EEE77AF4EEC77AF1EE10FA02DB20466F
:1063A0000AF0C6F8616D11BBA37B227B43B1D20812
:1063B0006A43384645F08AFE0BE04FF00109D3E707
:1063C000102A0FD107EB45023B464FF400419342A0
:1063D00005D1A8EB050807EB4507AA4460E723F8B9
:1063E000021BF4E7D2086A4380215046E2E74FEAF5
:1063F000C933A3F5DA43603B6FF0704292FBF3F3CD
:106400000593A36B029309F1FF334FF0000B069342
:106410005D45227B08D1A36BD20805FB0233A36341
:10642000E36B5B1BE363D4E7102A029B3DD133F996
:106430001B60226D019B511CB9F1010F216523F8EE
:10644000126049D0069A049BB3FBF2FC226D002136
:106450000CF1FF3C013A0846894530DC059937F0DC
:1064600017FA0090DDED007AF8EEE77A022167EE88
:10647000A87AFDEEE77A17EE900A304437F008FA72
:10648000227B102A2AD127F81B00A27B1AB980F49C
:10649000004027F81B00039B226DB2EB530F24BF73
:1064A000002323650BF1010BB2E7A27B13F90B600C
:1064B000002ABED186F07F06F64376B2B9E7002AFD
:1064C000BCBF039B02EB5302019B33F912E0013185
:1064D0007044A2EB0C02BFE70096C3E7A27B12B1A7
:1064E0000AF80B00D7E780F07F00C043F8E700BF51
:1064F000000000002DE9F04F2DED028B8DB0084615
:1065000011461A4603AB01935E4B0093092345F0F5
:1065100038FF40F29B334FF47A620121039845F033
:106520005BFF40F28223064602220B98012145F0D0
:1065300053FFDDF820B0BBF1000F824604DC40F2CF
:106540006B4101201BF010FF099D082D04D0102D78
:1065500002D04D4839F01CFD4C49582047F03CFA18
:106560000446DDE906809DF8283025730025DDE925
:106570000497A37384F80DA0C4F804B0E573A06079
:10658000606345F08CFC626BA06218B96073606454
:10659000E0620BE0294645F099FD606B45F07FFC19
:1065A000626BE06228B960736064A062104639F0E3
:1065B00069FC294645F08AFD35486565012384F864
:1065C0003030002F18BF384640F21A5204F1200133
:1065D000C4E90E55A4F8405036F01AFF2D489FED3F
:1065E0002E8A04F1140740F2C2223946B9F1000F95
:1065F00018BF484636F00CFF28484FF46C7204F17F
:106600002401B8F1000F18BF404636F001FFD4ED69
:10661000017A637B2661B8EE677A5B00C7EE087A81
:1066200007EE106AB8EE477A67EE877A07EE103AFF
:10663000B8EEC77A67EE877AFCEEE77A17EE900A33
:10664000C4ED137A45F02BFCE26C606410B9607302
:10665000A0629DE7294645F039FDD4ED017AF8EEB8
:10666000677A384688EE277A84ED077A36F0F8FEA6
:10667000204609F05DFF204625650DB0BDEC028B7C
:10668000BDE8F08FC81C0900AAF10700FC5C0800F7
:10669000020000C00200C8C200007A44020080BFAD
:1066A000F0B50D4685B055F8044B0646607B17469D
:1066B00040F03AFA02AB0193154B00933A4602239D
:1066C0002946701E1BF0BEFD029D9DF80C602946F8
:1066D0000022204606F042F82846656584F84060AE
:1066E00040F06BFA04F13C02606D04F1380140F0B7
:1066F00020FA227BE36BD208B3FBF2F3E363431E81
:106700005842584184F84100204605B0F0BD00BF12
:10671000B81C09002DE9F04F2DED068B8FB0D0F895
:1067200054A00D930B1E0A9314BF134600230B9322
:1067300090F84030426CDFEDACAAB3FA83F35B090A
:1067400080F840300E33044650F823300193037B29
:10675000DB08B2FBF3F30293019B0493029B002B33
:1067600000F09680E36C4BBB94F8513033B994F849
:106770005030ABB1E06E98B140F01FFAE06E60B1FE
:1067800004F14C0204F1480140F0D3F902280AD187
:106790000023E366E36484F85130617B0B0216E06A
:1067A0000023E366EAE7227BE36CD208B3FBF2F353
:1067B000E364431E5842584184F85100617BE26E05
:1067C0000B02002AE9D0E26C934228BF1346029ADA
:1067D00060689A4228BF1A46B2FBF1F189B293462B
:1067E00033F060FEF7EE000A04F134009FED7F0AFB
:1067F0004FF0C3FBF7EE000A04F1200070EE008AB0
:106800009FED7A0A4FF0B9FB04F11400B0EE409A04
:1068100036F026FED4ED067A94ED077A77EEC07A4C
:10682000F0EEE77AF4EEC77AF1EE10FA02DB2046DA
:1068300032F0F2F804F12403184606933FF07EFF8D
:10684000A36D627BE16E5B080393E36D013AD34075
:106850005B080793002940F0DD80F4EEEA8AF1EE50
:1068600010FA2BD8A37B227B33B1029B0198D2086C
:106870005A4345F02BFC0BE0102A19D14FF400438A
:10688000019A22F8023B0192029A013A0292F7D150
:1068900094F840300D9A0E33012054F823301360E1
:1068A000626C1E9B1A600FB0BDEC068BBDE8F08FCA
:1068B000029B0498D2085A438021DAE70E46F7EE8D
:1068C000009A0A9B002B4FD00B9B012B52D1079BA8
:1068D000002B4FD0656E984694F85270B8F10002C4
:1068E00018BF0122002F67D008EB1523A76E3AF9D5
:1068F00013302F4408EE103A3B0A4FEA152B05934C
:10690000059B5B453AD8F4EEE89AF1EE10FAB8EE42
:10691000C88AD4BFF0EE697AF0EE687A67EE887ABA
:10692000227BFDEEE77A102A17EE903A60D1019AA9
:1069300022F81630A27B22B9019A83F4004322F890
:10694000163094F85230002B5DD0039B1B02B7FB2E
:10695000F3F503FB1575B8F1000F59D06566029B7E
:106960000136B342ADD893E7627BB6FBF2F302FB8C
:106970001363AAE7256E4FF00008ADE7039BBBFB4E
:10698000F3F903FB19B9C144617B3AF91930069850
:10699000089207EE903AF8EEE77A0BF1010B67EEFA
:1069A000897AFDEEE77A17EE903A1BB23FF072FE5D
:1069B000089A2AF81900A3E705EB0809617B3AF960
:1069C0001930069808EE103AF8EEC87A013567EEED
:1069D000897AFDEEE77A17EE903A1BB23FF05AFE45
:1069E0002AF819008FE700BF0AD7233C00000000F7
:1069F000049A9355A27B002AA3D1049A83F07F03C3
:106A0000DB4393559DE7039B9D4228BF0025A2E7EA
:106A10002566A4E7F4EEEA8AA36C0893F1EE10FA77
:106A200040F288800026B3456ED0227B089B102A56
:106A300040F0828033F916300A99002900F08680F0
:106A40000B99012940F088800799002900F0848083
:106A5000656E0591059994F85270003907EE903AE9
:106A600018BF0121B8EEE78A0991002F77D0059B66
:106A7000A76E03EB15232F443AF91330102A09EEC1
:106A8000903A4FEA17234FEA15280C9300F0A7809D
:106A90000C9B434540F2A680039BB8FBF3F903FB34
:106AA0001989059B617B06989944F0EE487A3AF97A
:106AB000193007EE103AB8EEC77A6FF07F02E7EEB2
:106AC000097A08F10108FDEEE77A17EE903A934251
:106AD000B8BF13467F2B099AA8BF7F233FF0DAFD8A
:106AE00040B22AF81900D3E7227B102A089A0BBF7C
:106AF0000199049932F91320D2560CBF21F81320C2
:106B0000CA5401339B45EFD1029B227BA3EB0B03BD
:106B10000293019B03EB4B030193049B5B4404939F
:106B2000A36CD2080BFB0233A364E36CA3EB0B034F
:106B3000E36413E60023E5E7A17B9B5700297FF47C
:106B40007BAF83F07F03DB435BB275E7607BB6FB13
:106B5000F0F100FB116174E7256E002179E7059BD8
:106B600005EB0308F0EE487A3AF9183009EE903A4E
:106B7000B8EEE97A102AE7EE097AFDEEE77A17EE29
:106B8000900A6CD000F30703099A617B06983FF0E6
:106B900081FD013540B26DE0039BB8FBF3F903FBC7
:106BA0001989059B9944B0EE487A3AF9193007EEF5
:106BB000903AF8EEE77A41F6EF31A7EE897A08F1DC
:106BC0000108FDEEC77A17EE900A36F061FE099AC9
:106BD000617B034606983FF05DFD2AF819000C9B87
:106BE0004345D9D8B0EE007A37EE687AF7EE007AEE
:106BF000F4EEC77AF1EE10FAF4EEE87AD8BFB0EE10
:106C0000677AF8EEE99AF1EE10FAC8BFF0EE687A0A
:106C100067EEA97A41F6EF31E7EE087AFDEEE77A02
:106C200017EE900A36F034FE237B102B25D1019B02
:106C300023F81600A37B23B9019B80F4004023F8BE
:106C4000160094F852300BB3039B1B02B7FBF3F50D
:106C500003FB1575059BF3B165660136E3E641F666
:106C6000EF3136F015FE099A617B034606983FF036
:106C700011FD01352AF81800B4E7A37B13B1049B7A
:106C80009855DEE780F07F00C043F8E7039B9D4204
:106C900028BF0025DEE72566DFE700BF2DE9F04FBE
:106CA0002DED028B8FB0084611461A4603AB0193B7
:106CB000614B00930B2345F064FB40F29B334FF490
:106CC0007A620121039845F087FB40F2822308EEA7
:106CD000900A02220C98012145F07EFB099E002EAD
:106CE000054604DC40F26B4101201BF03DFBDDF862
:106CF00028B0BBF1080F05D0BBF1100F02D04F48F0
:106D000039F046F94E49702046F066FE04469DF87B
:106D1000341008989DF82C2084F85210DDE906A85C
:106D200065730025DDE9049784F80CB0A2736660F2
:106D3000E573A060606445F0B2F8A06328B920460E
:106D400040F002FD606C39F09DF8626C294645F018
:106D5000BDF9606C45F0A3F8E0630028EFD0626CE9
:106D60009FED388A294645F0B1F9012384F8403077
:106D7000627BE566514604F12400C4E91255A4F88B
:106D8000505001F06BFC304840F2B722002F18BF82
:106D9000384604F1200136F03BFB2C4804F114077F
:106DA00040F2C2223946B9F1000F18BF484636F00A
:106DB0002FFB27484FF46C7204F13401B8F1000F37
:106DC00018BF404636F024FBD4ED017A637BC4ED56
:106DD000048AB8EE677AC7EE087AB8EE687A67EE8A
:106DE000877AFCEEE77A17EE900A58434000E06598
:106DF00045F055F8606520B9204640F0A5FCE06DEF
:106E0000A1E7E26D294645F061F9D4ED017AF8EE8B
:106E1000677A384688EE277A84ED077A36F020FBC9
:106E2000204631F0F9FD2046C4E918550FB0BDECFD
:106E3000028BBDE8F08F00BF981E0900AAF1070081
:106E40001C5D080000007A443233B3BF0200FAC36D
:106E5000020000BFF0B50D4685B055F8044B06465C
:106E6000607B17463FF060FE02AB0193154B009329
:106E70003A4602232946701E1BF0E4F9029D9DF854
:106E80000C6029460022204605F068FC2846E5668D
:106E900084F850603FF091FE04F14C02E06E04F182
:106EA00048013FF046FE227BE36CD208B3FBF2F3CD
:106EB000E364431E5842584184F85100204605B00F
:106EC000F0BD00BF881E09002DE9F04F2DED068BA7
:106ED0008FB0C76B0B930B1E039390F8383090F86C
:106EE0000D80D0F850A0B3FA83F34FEA531380F823
:106EF000383003F10C03044650F82390037B08BF9D
:106F00000022DB08B7FBF3F7002948D0012A46D15D
:106F1000A8F102014B424B4108934FEA0823079323
:106F2000DFED819ACDF804904FEA4A030A93002FCF
:106F300000F0E580636C002B47D194F8493033B9F9
:106F400094F848306BB3A06E58B33FF036FEA06E95
:106F500050BBB7FBF8F1606889B233F0A3FA04F1D3
:106F6000100036F07DFA04F1140036F079FA04F1DD
:106F7000180036F075FA04F11C0036F071FA04F1CD
:106F8000200036F06DFAA37B227B002B00F0AF804F
:106F9000D2087A430021484645F098F8AFE0002334
:106FA000BAE70023A366D2E704F1440204F14001EA
:106FB0003FF0BFFD227B636CD208B3FBF2F3421EAD
:106FC00050425041636484F84900A36E6068002B0E
:106FD000BFD0079A636C9FED558A934228BF134632
:106FE000BB4294BF04930497236C0593049BB3FBAB
:106FF000F8F189B233F056FAD4ED097A94ED0A0A21
:10700000F8EE670A04F110004EF0B7FFF3EE040A41
:10701000B0EE409A04F11400B0EE690A4EF0ADFFF4
:10702000F7EE000AB0EE40AA04F11800B0EE690ACB
:107030004EF0A3FFDFED3E0AF0EE40AA04F11C0083
:107040009FED3C0A4EF099FF04F1200060EE088AA3
:10705000F7EE000AB0EE690A4EF08FFFD4ED097A20
:10706000F8EE677AB0EE496A77EEC97A20EE088AC0
:10707000A7EEAA6A20460026B0EE490A13F05CFD8E
:10708000B0EE460A0690204613F056FDD4ED017A84
:10709000069BB8EE677AC31ACAEE077A0993B6EE72
:1070A000007AB4EEE77AF1EE10FAD8BFF0EE477A44
:1070B0009FED217A67EE877AFDEEE88AFCEEE77AAB
:1070C000BDEEC88AC4ED197A049B9E4236D1019B5D
:1070D000227B33440193236CD20806FB02332364E2
:1070E000636C9B1BBF1B09EB460963641FE7102AF7
:1070F00015D14FF40043013F29F8023BFBD194F82E
:1071000038300B9A0C33012054F823301360E26BB3
:107110001E9B1A600FB0BDEC068BBDE8F08FD20845
:1071200001987A43802137E70000000000FEFF4607
:107130003333733F333373BF0000804F039B002B07
:1071400078D1B6FBF8F008FB1060431E5842584156
:10715000237B102B059B6FD133F91650636E04EB24
:107160008002D16D1944434BD165A3EBD13C4FEA6A
:10717000D13E099B3EEA210E28BFE646A3FB0E1C2A
:10718000090C069B41EA0C4119440028E36C0A985B
:1071900008BF00200344506D029050441FFA81FC48
:1071A000A0EB11418A4598BFA1EB0A0100294CD000
:1071B000481E33F911B033F910100C93A1EB0B01F9
:1071C00018EE903A0CFB01F10BEB214B0BFB03F09B
:1071D0000F210D9236F002FC0021284436F0FEFB10
:1071E000029A0C9B23F81200531C0D9A534508BFBA
:1071F0000023536518EE103AB3F5A47F0DDD0BFBA9
:1072000003F00F2136F0EAFB94F82C3003B3281A70
:1072100041F6EF3136F03CFB0546237B102B19D1AC
:1072200029F81650A37B1BB985F4004529F81650A0
:10723000013649E708988BE79D57A37B002B8DD13A
:1072400085F07F05ED436DB288E70AF1FF30B0E7C6
:107250002844DDE76FF07F039D42B8BF1D46A27B47
:107260007F2DA8BF7F2512B1019B9D55E0E75D40B2
:10727000FAE700BFFFFF01002DE9F04F2DED028B73
:1072800091B0084611461A4604AB0193674B009330
:107290000C2345F076F840F29B33642201210498D8
:1072A00045F09AF840F2822308EE100A02220F9865
:1072B000012145F091F80C9D0290002D04DC40F274
:1072C0006B4101201BF050F80D9B082B04D0102BB4
:1072D00002D0574838F05CFE564903936C2046F0C4
:1072E0007BFB0446039B0B98099E9DF828B09DF8F4
:1072F0003810E063DDE90787DDE905A923736560E0
:10730000029BA17300256373E573A06044F0C4FD84
:10731000E26B206328B96073E0646063104638F064
:10732000B1FD294644F0D2FEE06B44F0B5FDE26BBE
:10733000606318B96073E0642063EFE7294644F0A6
:10734000C5FE3D48A5660123BAF1000F18BF50469F
:10735000DFF8ECA084F8383040F2AD3204F11001CF
:10736000C4E91055A4F8485036F052F840F22342D0
:1073700004F11401B9F1000F14BF4846504636F02D
:1073800047F84FF4327204F11801B8F1000F14BF3E
:107390004046504636F03CF840F20A3204F11C01F7
:1073A000002F14BF3846504636F032F8002E14BF76
:1073B000304650464FF46C7204F1200136F028F844
:1073C000D4ED017ADFED1D6A84ED098AB8EE677AA3
:1073D000B8EE488AC6EE877A667B84F82CB0C4ED96
:1073E0000A7AC7EE267A67EE887AFCEEE77A17EE1D
:1073F000903A02335E4376002365304644F04CFDFC
:10740000E06420B9C4E90C006073304687E7324677
:10741000294644F05BFE2046C4E91555C4E91755DA
:10742000656611B0BDEC028BBDE8F08F281E090027
:10743000AAF10700DC5C0800020000C000007A44EA
:10744000020080BF10B50446407B3FF06DFBE16D4C
:10745000094A9FED0A0ACB0BA2EBD13233EA210392
:1074600028BF134607EE903AF8EEE77ABDE81040E1
:1074700087EE800A21F0AEBDFFFF010000FF7F47CD
:10748000F0B50D4685B055F8044B0646607B1746AF
:107490003FF04AFB02AB0193154B00933A4602239F
:1074A0002946701E1AF0CEFE029D9DF80C602946FA
:1074B0000022204605F052F92846A56684F8486067
:1074C0003FF07BFB04F14402A06E04F140013FF069
:1074D00030FB227B636CD208B3FBF2F36364431E80
:1074E0005842584184F84900204605B0F0BD00BF1D
:1074F000181E09002DE9F04F2DED048B8DB00029E9
:10750000099314BF13460023069390F82430876A2A
:10751000B3FA83F35B0980F8243000EB830304465D
:10752000D3F81CB0037BDB08B7FBF3F7836B029344
:10753000D0E93A239A42C0F0DF81B2FBF3F305931E
:10754000DA466BE10023C4F808317CE1227B236B2F
:10755000D208B3FBF2F3421E50425041236384F839
:107560003500D4F80831002B00F07F81617B226B5D
:1075700060680B02934228BF1346BB4294BF03933B
:107580000397E36A0493039BB3FBF1F189B232F0F2
:1075900089FF04F1100035F063FF04F118008DED50
:1075A0000B0AF7EE000A9FED130A4EF0E6FC0422E8
:1075B00004F114010BA830EE008A44F032FD20B132
:1075C0009DED0B0A204615F029F804F1A00307935E
:1075D00004F144030025B0EE009AF7EE008A089308
:1075E0000BE1102A01D17A0047E1D2087A438021C9
:1075F000504643E100000000069B012B00F05F8134
:10760000637BB5FBF3F803FB185808F1FF33D3F1A4
:10761000000848EB0308237B102B049B40F05281A9
:1076200033F91530D4E90F1201FB0822029921F831
:10763000123000222646A44601929CF8441061B301
:10764000DCF84810E06B029A090AB1FBF0F900FB84
:10765000191900FB0899013132F91990B1FBF0F2C8
:1076600000FB121100FB0811029ADCF8500032F9FD
:107670001110DCF84820A1EB09015FFA82FE0EFB35
:1076800001FED4F8FC10019A31F9101009EB2E2EEE
:1076900001FB0EFE02EBEE320192079A0CF1140C84
:1076A0006245CAD179EE487AD4F8F810019AF4EE1E
:1076B000E78AD017F1EE10FAA1FB022C01FB00CCF7
:1076C000D4BFB0EE686AB0EE676AD20B07EE903AAC
:1076D00042EA4C42B8EEE77A07EE902AF4EEC88A06
:1076E000F1EE10FAF8EEE77AD4BFF0EE686AF0EE49
:1076F000486A66EEA77A41F6EF31E6EE077AFDEECC
:10770000E77A17EE900A36F0C3F8237B102B40F08F
:10771000E3802BF81500A37B1BB980F400402BF805
:107720001500637B012B02D0B8F1000F64D096F8EE
:10773000443063B1D6E912321344B364336D726DD1
:1077400001339342336524BF002386F84430079BFE
:107750001436B342EBD1D4F8E430002B40F0CA80A9
:107760001946142208984A43825C002A40F0BD80E2
:1077700094ED3C7AD4F8E800B5EEC07AF1EE10FA58
:1077800019DD07EE900AF8EE677A67EE877AFCEE6D
:10779000E77A17EE903A73B1D4F8F42082EA4232D5
:1077A00082EA524282EA42120133C4F8F420B2FB68
:1077B000F3F603FB1623D4E90F623244121AD21AED
:1077C000B2FBF6F306FB1323142202FB01421B0259
:1077D000012182F844109364D4F80431D364002367
:1077E000C2E91430059BC4F8E430236CE26B01332A
:1077F000934228BF002323640135039B9D427FF4FD
:10780000FBAE227BE36AD20805FB0233E362236B03
:107810005B1B7F1B0BEB450BAA442363002F3ED061
:10782000236B002B7FF49DAE94F835305BB994F850
:107830003430002B3FF486AED4F8080100283FF422
:1078400081AE3FF0BAF9D4F8080170B104F130020A
:1078500004F12C013FF06DF902287FF477AE00238C
:10786000C4F80831236384F83530A17B227B0029DA
:107870003FF4B7AED2087A430021584644F026FCC4
:10788000617B6068B7FBF1F189B232F00BFE04F165
:10789000100035F0E5FD04F1180035F0E1FD94F835
:1078A0002430099A04EB83030120DB691360A26A88
:1078B0001A9B1A600DB0BDEC048BBDE8F08FDDF8AB
:1078C0001880A8E6A27B5B57002A7FF4ABAE83F05A
:1078D0007F03DB435BB2A5E6A37B13B10AF8050087
:1078E0001FE780F07F00C043F8E7013108297FF4EB
:1078F00038AF77E7013B76E7012320E62DE9F04F2B
:107900002DED068B8DB0084611461A4602AB019349
:107910008C4B00930A2344F034FD0B9840F28223F1
:107920000222012144F058FD089D002D064604DC8A
:1079300040F26B4101201AF017FDDDF81080B8F11C
:10794000010F03DC40F23F310220F4E7059840F2DA
:10795000C7230822012144F03FFDDDF824B0BBF12C
:10796000080F074605D0BBF1100F02D0764838F05B
:107970000FFB76494FF4867046F02EF804460698C1
:10798000DDE902A920F0A8FA07989DF82830656083
:10799000002584F80CB0A3736673E573A060A06241
:1079A000B0EE408A44F07BFAE06128B920463FF00F
:1079B000D6FEA06A38F066FAA26A294644F086FB31
:1079C000A06A44F06CFA20620028EFD0A26A29462F
:1079D00044F07CFB012384F8243040F27C4204F123
:1079E00010015046C4E90B55C4F80851A58635F07E
:1079F0000FFD4FF46C7204F11801484635F008FD94
:107A0000082F28BF0827012FB5EEC08A38BF0127ED
:107A1000F1EE10FAC4F8E880C4F8EC7029D4B7EE9F
:107A2000000AB4EEC08AF1EE10FAD8BFB0EE480AF0
:107A3000474B657BC4F8F4304FF48033B3FBF7F366
:107A4000B3F5004F28BF4FF4004308FB05F5C4F819
:107A5000F830AD004FEA480384ED3C0AE363284662
:107A600044F01DFAA06338B920463FF078FE28465E
:107A7000A0E79FED380ADBE72A46002144F026FB09
:107A8000D4F8E850C4F8005100236D002364284660
:107A900044F005FAC4F8FC000028E5D0D4F8003121
:107AA000DFED2D8A9FED2DAA012B83BF03F1FF335C
:107AB00007EE903AB8EE678AB7EE008A0025B7EE77
:107AC000009AF6EE009AD4F800319D421FD30023AD
:107AD00084F8443084F8583084F86C3084F880306E
:107AE00084F8943084F8A83084F8BC3084F8D0301E
:107AF000C4F8E43004F1100035F0B2FC204614F074
:107B00008DFD20460DB0BDEC068BBDE8F08F07EE75
:107B1000905AB8EE670A20EE280A80EE080A0DF0A7
:107B20008BFBD4F8FC3039EE400A20EE290A20EE17
:107B30000A0ABDEEC00A10EE102A23F815200135FE
:107B4000C1E700BFC81D0900AAF107009C5C08003E
:107B5000CDAB341200000000DB0FC94000FEFF4631
:107B6000F0B50D4685B055F8044B0646607B1746C8
:107B70003EF0DAFF02AB0193164B00933A46022324
:107B80002946701E1AF05EFB029D9DF80C60294686
:107B90000022204604F0E2FD2846C4F8085184F88B
:107BA00034603FF00AF804F13002D4F8080104F11F
:107BB0002C013EF0BEFF227B236BD208B3FBF2F315
:107BC0002363431E5842584184F83500204605B0CF
:107BD000F0BD00BFB81D090010B50446084620F0EE
:107BE0007BF9B5EEC00AF1EE10FA0CD4F7EE007A8C
:107BF000B4EEE70AF1EE10FAD8BFF0EE407AC4ED29
:107C00003C7A0E2010BDDFED017AF8E7000000009D
:107C10002DE9F04F2DED068B8BB0D0F85CA00993C9
:107C20000B1E049314BF13460023069390F83C30B8
:107C3000026CB3FA83F35B0980F83C3000EB8303FA
:107C400004465B6B0093037BDB08B2FBF3F3019309
:107C5000036D427B0593436DB3FBF2F34FEA530B85
:107C600021B1069B012B08BFD0F860A0236BDB037A
:107C7000A3F5DA43603B6FF07042B2FBF3F3089375
:107C8000009B0393F0EE009A019BCBB9049B002B61
:107C900000F05881069B012B40F05481C4F860A08D
:107CA00094F83C30099A04EB830301205B6B13606A
:107CB000226C1A9B1A600BB0BDEC068BBDE8F08FEE
:107CC000A36C4BBB94F84D3033B994F84C30ABB146
:107CD000606E98B13EF071FF606E60B104F14802D1
:107CE00004F144013EF025FF02280AD10023636617
:107CF000A36484F84D30617B0D0216E000236366B7
:107D0000EAE7227BA36CD208B3FBF2F3A364431E21
:107D10005842584184F84D00617B636E0D02002B80
:107D2000E9D0A36C9D4228BF1D46019B60689D421F
:107D300028BF1D46B5FBF1F189B232F0B3FBF7EE77
:107D4000000A04F120009FED810A4EF016F9F7EECB
:107D5000000A30EE008A04F11C009FED7C0A4EF010
:107D60000CF9636E0293B0EE40AA0BB1636C029300
:107D70000027F7EE008ABD4217D1019B5B1B0193E0
:107D8000009B03EB45030093039B2B440393636E1B
:107D9000002B3FF479AF227B636CD20805FB0233E2
:107DA0006364A36C5B1BA3646EE7049B002B40F031
:107DB000AE80637BB7FBF3F903FB1979B9F1010FCF
:107DC000666E14BF4FF000094FF001090BFB09F973
:107DD00036B1237B102B029B40F09C8033F9176057
:107DE000226B002A00F0A080E06AA16A031F0793BB
:107DF00001EB820C4FF000080798B1EC017A50F8C3
:107E0000043F0790ABEB03035344B3FBFBFE0BFBB8
:107E10001E3305984B448C4530F9133007EE903AE9
:107E2000F8EEE77A67EE877AFDEEE77A17EE903A9A
:107E30009844E1D1012A06D040460899079235F0CE
:107E400027FD079A8046059BD14433F91900237B0F
:107E500007EE900AF8EEE77A002A08BF804667EE40
:107E60008A7A102BFDEEE77A17EE900A30445DD146
:107E700041F6EF3135F00CFD79EEC87A059BF4EE52
:107E8000E78AF1EE10FAD4BFB0EE686AB0EE676A26
:107E900007EE906AB8EEE77A07EE908AF4EEC88AA9
:107EA000F1EE10FAF8EEE77AD4BFF0EE686AF0EE81
:107EB000486A66EEA77A23F81900E6EE077A41F6DB
:107EC000EF31FDEEE77A17EE900A35F0E1FC237B07
:107ED000102B2ED1009B23F81700A37B23B9009B06
:107EE00080F4004023F81700627B012A07D0049B2E
:107EF0002BB9B7FBF2F302FB1373012B05D10AF187
:107F0000010AD34598BF4FF0000A013733E7069BBB
:107F1000012B55E7DE57A37B002B7FF461AF86F082
:107F20007F06F64376B25BE790468CE700F30700E6
:107F3000A2E7A37B13B1039BD855D5E780F07F0060
:107F4000C043F8E7C4F85CA0AAE600BF0000000048
:107F50002DE9F04F2DED028B8DB0084611461A46E3
:107F600002AB0193594B00930A2344F00AFA40F202
:107F70009B334FF47A620121029844F02DFA40F2CB
:107F8000822308EE900A02220B98012144F024FA81
:107F9000089E002E054604DC40F26B4101201AF0D9
:107FA000E3F9DDF824B0BBF1080F05D0BBF1100FE9
:107FB00002D0474837F0ECFF4649682045F00CFDF9
:107FC0000446DDE9059707989DF82820657300258C
:107FD000DDE9038A84F80CB0A2736660E573A060E3
:107FE000206443F059FF606328B920463FF0BFFB8F
:107FF000206C37F047FF226C294644F067F8206C6C
:1080000043F04AFFA0630028EFD0226C9FED328A34
:10801000294644F05BF831486566012384F83C301A
:1080200040F2B72204F11C01BAF1000F18BF50460C
:10803000C4E91155A4F84C5035F0EAF928484FF43A
:108040006C7204F12001B9F1000F18BF484635F0F9
:10805000DFF9D4ED017A637BC4ED048AB8EE677A68
:10806000C7EE087AB8EE687A67EE877AFCEEE77AB0
:1080700017EE900A58434000A06543F00DFF2065BD
:1080800020B920463FF073FBA06DB2E7A26D2946F0
:1080900044F01CF8D4ED017AF8EE677A414688EE98
:1080A000277A204684ED067A08F0DEFC2046C4E9F3
:1080B0001755C4E90955C4E90B55394608F012FDB6
:1080C00020460DB0BDEC028BBDE8F08F681D0900A5
:1080D000AAF107007C5C080000007A443233B3BF89
:1080E000020000BFF0B50D4685B055F8044B0646BA
:1080F000607B17463EF018FD02AB0193154B0093D1
:108100003A4602232946701E1AF09CF8029D9DF8FB
:108110000C6029460022204604F020FB28466566B4
:1081200084F84C603EF049FD04F14802606E04F1B1
:1081300044013EF0FEFC227BA36CD208B3FBF2F3B9
:10814000A364431E5842584184F84D00204605B0B0
:10815000F0BD00BF581D09002DE9F04F2DED048B37
:108160008BB00029079314BF13460023069390F8A1
:108170003030476B456A427BB3FA83F35B0980F882
:1081800030300A33044650F82390037BDB08B7FBFA
:10819000F3F7436C0393036A5B08B3FBF2FB002D18
:1081A00000F07B81C36C02936D08B5FBF2F5CA4603
:1081B000F0EE009A08E10023E36519E1227BE36B0E
:1081C000D208B3FBF2F3421E50425041E36384F8FD
:1081D0004100E36D002B00F01B81617BE26B606866
:1081E0000B02934228BF1346BB4294BF04930497EB
:1081F000A36B0593049BB3FBF1F189B232F052F902
:1082000004F1100035F02CF904F118008DED090A85
:10821000F7EE000A9FEDA20A4DF0AFFE042204F132
:10822000140109A830EE008A43F0FBFE20B19DED59
:10823000090A204630F052FC0026F7EE008AB2E030
:10824000102A01D17A00EBE0D2087A43802150460F
:10825000E7E0069B012B00F00581637BB6FBF3F89A
:1082600003FB186808F1FF33D3F1000848EB03085B
:10827000237B102B059B40F0F88033F91630227FCA
:10828000019308FB0BF0A2B9A26C0244002D00F090
:10829000F680216D029B08FB051133F91110039B39
:1082A00023F81210226D08FB052CDDE9012323F8C9
:1082B0001C20616D039B00EB11200A0A33F91000AA
:1082C000F5B1A16C91428CBFDC464FF0000C944498
:1082D000BCEB010E14D0AE4512D8226D7244B2FB35
:1082E000F5F305FB132208FB0522029BA1EB0C0111
:1082F00033F9122029444A4300FB0E2292FBF5F089
:1083000079EEC87A06EE900AF4EEE78AF1EE10FAFA
:10831000F4EEC88AD4BFB0EE686AB0EE676AF8EED1
:10832000E66AF1EE10FADDED017AD4BFB0EE687ABC
:10833000B0EE487AF8EEE77A27EE267A41F6EF318A
:10834000A6EE277AFDEEC77A17EE900A35F0A0FA6E
:10835000237B102B40F0988029F81600A37B1BB9D3
:1083600080F4004029F81600637B012B02D0B8F19D
:10837000000F17D0227F62B9A36C01335B4528BF81
:108380001346A3642DB1236D0133AB4238BF1A46A7
:108390002265D4E915321344B3EB0B2F28BFA3EBAE
:1083A0000B2363650136049B9E427FF452AF227B10
:1083B000A36BD20806FB0233A363E36B9B1BBF1BBB
:1083C00009EB4609B244E363002F3BD0E36B002B7B
:1083D0007FF4FFAE94F8413053B994F84030002B4D
:1083E0003FF4E9AEE06D00283FF4E5AE3EF0E5FB7A
:1083F000E06D68B104F13C0204F138013EF099FBF4
:1084000002287FF4DBAE0023E365E36384F84130A8
:10841000A17B227B00293FF413AFD2087A430021CD
:10842000484643F053FE617B6068B7FBF1F189B2C7
:1084300032F038F804F1100035F012F804F11800A9
:1084400035F00EF894F83030079A0A33012054F8CA
:1084500023301360626B189B1A600BB0BDEC048B69
:10846000BDE8F08FDDF8188002E7A27B9B57002A59
:108470007FF405AF83F07F03DB435BB2FFE6039B32
:10848000019923F8121014E7A37B13B10AF8060030
:108490006AE780F07F00C043F8E7029587E600BFF7
:1084A000000000002DE9F04F8DB0084611461A4635
:1084B00003AB0193494B0093092343F062FF0B98F0
:1084C00040F282230222012143F086FFDDF820B032
:1084D000BBF1000F824604DC40F26B41012019F031
:1084E00043FF099D082D04D0102D02D03C4837F0E1
:1084F0004FFD3C49602045F06FFA0446DDE9057602
:1085000007989DF8283025730025DDE90398A373AB
:1085100084F80DA0C4F804B0E573A060606343F074
:10852000BEFCA06228B920463FF02AF9606B37F004
:10853000A9FC626B294643F0C9FD606B43F0AFFCB8
:10854000E0620028EFD0626B294643F0BFFD0123B3
:1085500084F8303040F27C4204F110014846C4E90E
:108560000E55E565A4F8405034F052FF4FF46C729C
:1085700004F11801404634F04BFF25772762384656
:1085800043F08DFC606420B920463FF0F9F8206A82
:10859000CDE7226A294643F099FD6662E6B130468E
:1085A00043F07DFCE06420B920463FF0E9F8606AC2
:1085B000BDE7626A294643F089FD0023C4E914330C
:1085C000A36404F1100034F04BFF204630F086FA2B
:1085D00020460DB0BDE8F08FE664EEE7101D0900FF
:1085E000AAF10700BC5C0800F0B50D4685B055F84F
:1085F000044B0646607B17463EF096FA02AB0193A9
:10860000154B00933A4602232946701E19F01AFEB4
:10861000029D9DF80C6029460022204604F09EF839
:108620002846E56584F840603EF0C7FA04F13C0254
:10863000E06D04F138013EF07CFA227BE36BD20856
:10864000B3FBF2F3E363431E5842584184F8410000
:10865000204605B0F0BD00BF582009000E29F7B52F
:10866000944604463FD011F003032ED108681F4DF5
:10867000A84227D10E461E4F56F8045FAB420DD1DB
:1086800001F1080605FB0CF22160E068110143F0DE
:1086900009FCC4E90165E06003B0F0BD56F8040FC1
:1086A00082070AD01FF0A2FCC3881248009340F250
:1086B0001132F123752137F05FFC0268BA42F1D123
:1086C0000133DBE70A4B98420AD008461FF08EFCC4
:1086D000C388009308489D23F12240F21131EAE754
:1086E00026460125CEE700252E46CBE72CDB0700EA
:1086F0003853080047FC0700B8FB07002DE9F04F8E
:108700002DED0E8B85B00446039390F82C30076B4B
:10871000B3FA83F35B0980F82C3000EB8303D3F8C2
:108720002480037BC146DB08B7FBF3F7002F45D05D
:10873000A36B04F11002019204F1140B04F118066A
:1087400004F1200A002B57D194F83D3043B994F836
:108750003C30002B42D0206C00283FD03EF02DFA58
:10876000206C60B104F1380204F134013EF0E1F90B
:10877000022836D100232364A36384F83D30A17B13
:10878000227B002900F00B81D2087A430021404669
:1087900043F09CFC617B6068B7FBF1F189B231F07A
:1087A00081FE04F1100034F05BFE584634F058FEB0
:1087B000304634F055FE504634F052FE94F82C30DA
:1087C000039A04EB830301205B6A1360226B1C9BFA
:1087D0001A6005B0BDEC0E8BBDE8F08F002323645A
:1087E000BEE7227BA36BD208B3FBF2F3A363431E65
:1087F0005842584184F83D00236C002BBFD0617B68
:10880000A36B60689FEDB48A0D029D4228BF1D4690
:10881000BD42636B019328BF3D46B5FBF1F189B2C0
:1088200031F040FEF7EE000A04F110009FEDAB0AB4
:108830004DF0A3FBDFEDAA0A5846F0EE408A9FED0B
:10884000A90A4DF09AFB20EE080A10F0C9F930464B
:10885000F3EE080AF0EE40BA9FEDA30A4DF08DFB4F
:1088600020EE080A10F0BCF9F7EE000AB0EE40AABC
:1088700050469FED9A0A4DF080FB267FB0EE409A5D
:10888000002E40F09580DFED997A77EEE88ADFEDF3
:10889000987AB4EEE79AF1EE10FA40F2C080DFED7C
:1088A00095AA9FED95BA4FF0000AAA4500F0A9805D
:1088B000237B0293102B019B40F0B38033F91A30D5
:1088C00007EE903AB8EEE78A237F68EE2B7A012B09
:1088D000FDEEE77AB7EE00CA17EE90BA05D1617FD8
:1088E0000BEA060B002900F0E48007EE90BAB8EE20
:1088F000E70A022B20EE2A0A00F09E80032B00F0EC
:10890000C68053B9F0EE680AB0EEC00A2DF044FDFF
:10891000BBF1000F01DAB1EE400A94F81DB020EE71
:108920000A0ABBF1000F0BD0B5EEC00AF1EE10FA47
:1089300040F3BA80B1EE400A10F052F93CEE400A22
:1089400020EE0B0AFDEEC07ABBF1000F0CD117EE42
:10895000903A6A4A9342B8BF1346B3F5004FA8BF96
:108960004FF4004307EE903AF8EEE77A3CEE49CA3E
:1089700067EE897A029BE8EE0C7A102BFDEEE77A1F
:1089800017EE903A40F09E8028F81A30A17B19B972
:1089900083F4004328F81A300AF1010A85E7102A07
:1089A00001D17A00F3E6D2087A4380214846EFE607
:1089B000032E09D1DFED4D7A38EEA87A77EEE87A0A
:1089C000C7EE278A002662E7012EFBD1B2EE0C0A21
:1089D00028EE800A30F066FABCEEC00A10EE103ABB
:1089E0009E40764253E7227B102A019A0BBF32F950
:1089F0001320D25628F8132009F803200133AB4284
:108A0000F1D1227B636BD20805FB02336363A36B56
:108A10005B1B7F1B08EB4508A944A36386E6002384
:108A2000EDE7A17B13F90A3000297FF449AF83F009
:108A30007F03DB435BB243E7DFED317A60EE27CAA9
:108A4000F0EEEC7AB1EEE70AFEEE087A20EE270AA5
:108A500010F0C6F8B0EE40DAB0EE6C0A10F0C0F8D4
:108A6000F0EE40DA3DEE0C0AB1EE6CEA2CEEC00AF4
:108A700010F0B6F8F0EE40CAB0EE4E0A10F0B0F8C2
:108A80007DEEECCA70EE2D7A8CEEA70A45E778EE03
:108A90008C7AB0EE4C7A67EE807AB0EEC00AA0EE27
:108AA000287A87EE870A38E710F09AF830EE4C0AF9
:108AB00046E707EE90BAF8EEE77A67EE8A7AFDEEBF
:108AC000E77A44E7A17B11B109F80A3064E783F043
:108AD0007F03DB43F8E700BFE3C8EB3D0000000085
:108AE00000007042000070C20000A0C24703803F37
:108AF0000AD7233C0000003800FEFF460180FFFF3C
:108B0000C0B12F3F2DE9F04F91B0084611461A46EB
:108B100005AB0193404B00930B2343F032FC0F98BD
:108B200040F282230222012143F056FC0C9E002ECB
:108B3000834604DC40F26B41012019F015FC0D9FC7
:108B4000082F04D0102F02D0344837F021FA089DA6
:108B500035B1284632494FF46D7219F055FC2D7924
:108B60003049442044F038FF0446079B0B989DF899
:108B700038209DF824800293DDE905A90A9B6660F0
:108B80000026A273277384F80DB0E673A0602063FB
:108B9000039343F084F9226B606220B96073A06292
:108BA000104637F06FF9314643F090FA206B43F0EE
:108BB00076F9226BA06210B960736062F0E731460B
:108BC00043F084FA012384F82C3004F1100150465C
:108BD000C4E90D662664A68740F2E12234F018FC51
:108BE00004F11401484640F20C4234F011FC0298A2
:108BF00004F1180140F20A4234F00AFC03984FF4E1
:108C00006C7204F1200134F003FC2046257784F8CF
:108C10001D8011B0BDE8F08F00200900AAF1070007
:108C2000005C08003C5C080010B50446407B3DF049
:108C30007BFF217F0248BDE8104040F0DFB800BF55
:108C4000005C0800F0B50D4685B055F8044B0646AB
:108C5000607B17463DF068FF02AB0193154B009314
:108C60003A4602232946701E19F0ECFA029D9DF83F
:108C70000C6029460022204603F070FD284625643A
:108C800084F83C603DF099FF04F13802206C04F157
:108C900034013DF04EFF227BA36BD208B3FBF2F30D
:108CA000A363431E5842584184F83D00204605B056
:108CB000F0BD00BFF01F090038B50C460546054958
:108CC0004FF46D72204619F09FFBA3882B770E207E
:108CD00038BD00BF005C08002DE9F04F2DED028B80
:108CE00089B00446079390F82C30066BB3FA83F3EF
:108CF0005B0980F82C3000EB8303F7EE008AD3F891
:108D000024B0037BCDF804B0DB08B6FBF3F6002EED
:108D100000F0AA80A36B04F12007002B42D194F845
:108D2000413033B994F840305BB3606C48B33DF0E8
:108D300044FF606C60B104F1380204F134013DF08D
:108D4000F8FE022820D100236364A36384F8413035
:108D5000617B6068B6FBF1F189B231F0A3FB384664
:108D600034F07EFB04F110003DF0E8FCA37B227B95
:108D7000002B71D0D20872430021584643F0A6F967
:108D800072E000236364D4E700F1FF3E227BA36B13
:108D9000DEF1000040EB0E00D20884F84100B3FB86
:108DA000F2F3A363636C617B6068002BD0D0A36B8C
:108DB0000D029D4228BF1D46B54228BF3546636B54
:108DC000B5FBF1F189B2029331F06CFB9FED910A92
:108DD000F7EE000A38464DF0D0F8DFED8F7AB4EEAA
:108DE000E70AF1EE10FAB0EE408A71D9E369002B80
:108DF0005CD00027AF425BD2637BEA1B013B22FAC7
:108E000003F3B3F5807F28BF4FF4807303937B0097
:108E10000693029B03EB470305930021627B039BB0
:108E200003FB02F0884255D84FF00009A2695FFAAF
:108E300089F8424572D8069B03EB0B09019B4FF062
:108E4000000803EB070A627B039B03FB02F1414529
:108E500000F284800F44CDE7102A15D14FF400436F
:108E6000013E2BF8023BFBD194F82C30079A04EB1F
:108E7000830301205B6A1360226B149B1A6009B0A4
:108E8000BDEC028BBDE8F08FD208019872438021BF
:108E900074E7227B102A029A15BF019932F9132038
:108EA000D2562BF8132018BFCA540133AB42F0D16D
:108EB000019B227B2B440193636BD20805FB023399
:108EC0006363A36B5B1B761B0BEB450BA3631EE776
:108ED0000023EBE7B1FBF2F002FB101202F1FF3CC2
:108EE000DCF1000242EB0C0200EB0220227BE36B80
:108EF000102A06D1059A32F9112043F820200131B9
:108F00008CE7029A94F80EE03A445256BEF1000FF4
:108F1000F3D182F07F02D24352B2EEE7626952F897
:108F200028300493184608F001FF4FF0000A617BD7
:108F30005FFA8AFC614502D809F1010976E7E06928
:108F4000E26B039B18FB01C100EB011102EB8C22C9
:108F500004984CF0BAFF0AF1010AE8E7B8FBF2F115
:108F600002FB1182531E5A425A4101EB0221E26B6D
:108F700002EB8103D3ED007A227BF8EEE77A102A28
:108F800078EEC86A67EE887A1FD1059B33F91830EE
:108F900007EE103AB8EEC77A41F6EF31E7EE267ADF
:108FA000FDEEE77A17EE900A34F072FCA9F80000A3
:108FB000A27B1AB980F40040A9F8000008F101086A
:108FC00009F102090AF1010A3DE7029BA17BDA19C6
:108FD00012F9082061B107EE102AB8EEC77AE7EE61
:108FE000267AFDEEE77A17EE902A8AF80020E5E768
:108FF00082F07F02D24352B207EE102AB8EEC77A4F
:109000006FF07F02E7EE267AFCEEE77A17EE903AF1
:109010005A40EAE7000000000AD7233C2DE9F0435C
:109020008BB0084611461A4603AB0193304B0093B0
:10903000072343F0A6F9099840F282230222012176
:1090400043F0CAF9069E002E814604DC40F26B41D3
:10905000012019F089F9079D082D04D0102D02D0A8
:10906000244836F095FF2449482044F0B5FC0446D6
:109070009DF82030059825730025A373DDE903874B
:1090800084F80D906660E573A060206342F007FFEE
:10909000226B6062294643F019F8206B42F0FFFE14
:1090A000226BA062294643F011F8607B012384F80B
:1090B0002C30800242F0F3FE627BE063294692028C
:1090C00043F004F8627B6564414604F11000C4E992
:1090D0000D55A4F84050FFF7C1FA38464FF46C72B2
:1090E00004F1200134F094F920460BB0BDE8F08380
:1090F000B81F0900AAF107005C5C0800F0B50D4636
:1091000085B055F8044B0646607B17463DF00CFDD4
:1091100002AB0193154B00933A4602232946701E79
:1091200019F090F8029D9DF80C6029460022204617
:1091300003F014FB2846656484F840603DF03DFD73
:1091400004F13802606C04F134013DF0F2FC227B42
:10915000A36BD208B3FBF2F3A363431E58425841FA
:1091600084F84100204605B0F0BD00BFA81F0900EB
:109170002DE9F04F2DED068B8FB004460B930B1E9F
:10918000089314BF13460023099390F82C30056B05
:10919000B3FA83F35B0980F82C3000EB8303D3F838
:1091A0002480037BC346DB08B5FBF3F5002D00F0FC
:1091B000FB80A36B04F1100904F11407002B43D1C9
:1091C00094F83D3033B994F83C307BB3A06C68B36D
:1091D0003DF0F3FCA06C60B104F1380204F13401FD
:1091E0003DF0A7FC022824D10023A364A36384F8E4
:1091F0003D30617B6068B5FBF1F189B231F052F925
:10920000484634F02DF9384634F02AF904F11800B4
:1092100034F026F9A37B227B002B00F0BD80D2081E
:109220006A430021404642F051FFBDE00023A364A1
:10923000D0E7411E227BA36B48424841D20884F804
:109240003D00B3FBF2F3A363A36C617B6068002B6A
:10925000CFD0A36B0E029E4228BF1E46AE42636B68
:10926000029328BF2E46B6FBF1F189B231F01AF90C
:10927000D4ED080A9FED820A48464CF07EFEDFEDF1
:10928000810A3846B0EE40AA9FED7F0A4CF075FE89
:10929000F7EE000AB0EE408A04F118009FED780A5C
:1092A0004CF06BFEDFED796A20EE260ABDEEC00AB7
:1092B00010EE103A1BB2B3F5A47F049340F3A580DF
:1092C00094ED087ACAEE077A0027B7EE007A37EEF7
:1092D000676A37EE877A28EE268AC6EE077ABDEEF1
:1092E000C88A67EEA67A18EE103AFDEEE77A1BB24E
:1092F000079317EE903A1BB205935B420A93B7426D
:1093000075D0089B002B40F08280627BB7FBF2F3A4
:1093100002FB13735A1E53425341227F12FB03F286
:109320000392227B102A029A73D132F917200192FC
:10933000626C32F91300079B0F21584334F04EFB47
:10934000019B0021184434F049FB039B81464FEAFE
:10935000430A0022237F934264D8039B626C003B44
:1093600018BF01230F2122F81390049B09FB03F07F
:1093700034F034FB019B0221184434F089FA237B3A
:10938000102B73D128F81700A37B1BB980F4004081
:1093900028F817000137B2E7102A15D14FF400431F
:1093A000013D28F8023BFBD194F82C300B9A04EBDA
:1093B000830301205B6A1360226B1E9B1A600FB04F
:1093C000BDEC068BBDE8F08FD2086A438021584679
:1093D00029E7227B102A029A0BBF32F91320D256BA
:1093E00028F813200BF803200133B342F1D1227B7C
:1093F000636BD20806FB02336363A36B9B1BAD1B3D
:1094000008EB4608B344A363D0E60023EDE7099BCD
:1094100080E7A17BD257002989D182F07F02D24315
:1094200052B284E70A9B0D9209FB03F00F2134F03E
:10943000D5FA236C069333F90A300021184434F02E
:10944000CDFA059A03460F2150430C9334F0C6FA27
:109450000021484434F0C2FA069B0D9A23F80A0012
:10946000DDF8309001320AF1020A73E7A37B13B1F1
:109470000BF807008EE780F07F00C043F8E700BFDD
:10948000000000006666663FCDCCCC3D00FEFF4686
:109490002DE9F04F8DB0084611461A4603AB0193F3
:1094A0003E4B0093092342F06CFF0B9840F282235D
:1094B0000222012142F090FFDDF820B0BBF1000F45
:1094C000824604DC40F26B41012018F04DFF099DFB
:1094D000082D04D0102D02D0314836F059FD314905
:1094E0004C2044F079FA04469DF828309DF8187015
:1094F000079825730025A373DDE90396DDF8148032
:1095000084F80DA0C4F804B0E573A060206342F0B5
:10951000C6FC226B6062294642F0D8FD206B42F007
:10952000BEFC226BA062294642F0D0FD607BA564A0
:10953000012384F82C309840C4E90D55A58742F0EA
:10954000AEFC627B60642946520042F0BFFDD4ED60
:10955000017A154BFBEEEF7A0E2E08BF1E46C4EDC6
:10956000087A04F1100148464FF4487233F050FF76
:1095700004F11401304640F20A3233F049FF4FF44F
:109580006C7204F11801404633F042FF2046394620
:109590003EF0FDF820460DB0BDE8F08F601F0900D9
:1095A000AAF107001C5C08003233B3BFF0B50D46CA
:1095B00085B055F8044B0646607B17463DF0B4FA7B
:1095C00002AB0193154B00933A4602232946701EC5
:1095D00018F038FE029D9DF80C60294600222046B6
:1095E00003F0BCF82846A56484F83C603DF0E5FA39
:1095F00004F13802A06C04F134013DF09AFA227BA8
:10960000A36BD208B3FBF2F3A363431E5842584145
:1096100084F83D00204605B0F0BD00BF501F090092
:109620002DE9F04F2DED028B8FB09FED818A0A93CB
:1096300090F84430826CB3FA83F35B0980F84430CD
:1096400000EB83030446D3F83CA0037BF7EE008ACB
:10965000DB08B2FBF3FBBBF1000F0FD194F84430F1
:109660000A9A04EB83030120DB6B1360A26C1A9B44
:109670001A600FB0BDEC028BBDE8F08F236D6BBBA1
:1096800094F855303BB994F85430C3B1D4F838014C
:10969000A8B13DF092FAD4F8380168B104F1500253
:1096A00004F14C013DF045FA02280CD10023C4F826
:1096B0003831236584F85530617B0D0218E00023B2
:1096C000C4F83831E7E7227B236DD208B3FBF2F30D
:1096D0002365431E5842584184F85500617BD4F8F5
:1096E00038310D02002BE7D0236D9D4228BF1D4667
:1096F0005D4528BF5D466068B5FBF1F189B230F089
:10970000D1FE9FED4B0AF7EE000A04F114004CF075
:1097100034FCB4EEE80AF1EE10FA00F38380B4EE04
:10972000C08AF1EE10FAC8BFB0EE480ADFED417A08
:1097300020EE270AF7EE000ABDEEC00A04F1380059
:1097400010EE103A1BB20193C3F500431BB2B0EE0A
:10975000480A08934CF011FC30EE000AF0EE007A53
:1097600077EEC07A9FED347AF4EEE78AF1EE10FAE4
:10977000D8BFF0EE687AF4EEC08A67EE877AF1EE31
:1097800010FAD8BFB0EE680AFDEEE77A20EE070ABD
:1097900017EE903ABDEEC00A1BB2069310EE103AD7
:1097A000F7EE000A1BB2B0EE480A04F1100007936E
:1097B0004CF0E3FBB4EEE80AF1EE10FA35DCB4EE5F
:1097C000C08AF1EE10FAC8BFB0EE480ADFED1B7A8E
:1097D00020EE270A0027BDEEC00A10EE103A03F56E
:1097E000B34319331BB2059304F1180318460293CF
:1097F0003CF0A4FF04F12803184603933CF09EFFBD
:10980000E36C0493BD421BD1227BE36CD20805FBC1
:109810000233E364236D5B1BABEB050B0AEB450ADC
:10982000236518E7B7EE000A80E7B7EE000ACDE738
:1098300000000000CDCC4C4600FEFF46295C0F46E0
:10984000D4F8383113B1049B33F91730617B00939E
:10985000B5FBF1F201FB1252009B0298D2B23CF030
:1098600019FF42F222235843112134F0B7F804F1D2
:1098700094030B9004F1740904F1540609934FF01A
:10988000000859F8042FB6F96430B6F8840032F9AC
:1098900013C0CDE90C32019B10FB03F0089B0F2194
:1098A0000CFB0300E04434F099F8059BA6F8840013
:1098B0000F21584334F092F80B9B0021184434F0E8
:1098C0008DF8DDE90C3222F81300B6F8643036F971
:1098D000021F01331BB29942D8BF0023A6F86230A1
:1098E000099B4B45CDD147F6E12000FB08F0112143
:1098F00034F074F804F58278034604F5937604F5A1
:109900008A7958F8042FB6F9021032F9110003EBE6
:10991000600C22F811C0C01A012134F05FF836F84B
:10992000022F36F9301C013212B29142D8BF002208
:10993000C14503463280E4D1617BB5FBF1F201FB06
:109940001252D2B203983CF0A5FE069B0646009840
:109950000F21584334F042F8079B80465E431E2097
:109960000F21704334F03AF841F6EF31404433F0C0
:109970008FFF2AF81700013744E700BF2DE9F04FA9
:109980008FB0084611461A4604AB0193834B0093EF
:109990000A2342F0F6FC0D9840F2822302220121B4
:1099A00042F01AFD0A9D002D064604DC40F26B4190
:1099B000012018F0D9FC9DF8303013B9784836F002
:1099C000E7FADDF82CA0BAF1100F01D07548F6E7E0
:1099D00075494FF49E7043F0FFFF0446DDE90870BF
:1099E000DDE906B39DF83020A273DDE904986560D7
:1099F000002584F80CA06673E573A060A06403934F
:109A000042F04AFAE06328B920463DF0D8FEA06C47
:109A100036F038FAA26C294642F058FBA06C42F0AE
:109A20003BFA20640028EFD0A26CDFF898A1294609
:109A300042F04CFB012384F84430627BC4F8385177
:109A4000594604F11800C4E91355A4F85450FEF720
:109A500005FE627B039904F12800FEF7FFFDB9F1D2
:109A6000000F14BF4846504640F2594204F110011D
:109A700033F0CEFCB9F1000F14BF4846504640F217
:109A8000594204F1100133F0C3FCB8F1000F14BFC8
:109A90004046504640F2B12204F1140133F0B8FCC4
:109AA000002F08BF5746B8F1000F14BF404650467C
:109AB00040F2B12204F1140133F0AAFC38464FF40D
:109AC0006C7204F1380133F0A3FC38464FF46C7229
:109AD00004F1380133F09CFC3449354A354840F2F2
:109AE0005C43A4F85630344B2367C4E91612C4E92A
:109AF0001A12C4E9183040F25163A4F87430F6B277
:109B000004F1540704F17408A946B5EBC60F12D34B
:109B10002A4A2B4BC4E93E23C4E94023002504F123
:109B2000F60704F58278A946B5EB860F1ED32046CA
:109B30000FB0BDE8F08FB7F90200400042F0ACF979
:109B400048F8040F38B904EB450520463DF037FED0
:109B5000B5F956005CE737F9022F002142F0B6FA5A
:109B60000135A7F86290A7F88290CEE7B7F9020016
:109B7000400042F091F948F8040F30B97C35204696
:109B80003DF01DFE34F9150042E737F9022F0021A0
:109B900042F09CFA0135A7F83090C5E7001F090094
:109BA000CBE70700B3F10700E05B0800A404FD0465
:109BB0004C058E0551065C04D30515062C02B9012F
:109BC0005501E100020080BFF0B50D4685B055F8A3
:109BD000044B0646607B17463CF0A6FF02AB0193A0
:109BE000164B00933A4602232946701E18F02AFBB2
:109BF000029D9DF80C6029460022204602F0AEFD31
:109C00002846C4F8385184F854603CF0D6FF04F17B
:109C10005002D4F8380104F14C013CF08AFF227B59
:109C2000236DD208B3FBF2F32365431E584258411B
:109C300084F85500204605B0F0BD00BFF01E0900B5
:109C400070B58AB0084611461A4606AB0193264BFA
:109C50000093042342F095FB0698052203A91CF00B
:109C600083F8059C622C0ED0682C0FD0482C1FD096
:109C7000422C01D1002507E0012C1BD01B4840F2EB
:109C8000722136F08DF90125012401E0012502241D
:109C90009DF8243083B9079B049A63435B00B2FBB1
:109CA000F3F103FB11223AB1114840F27221E8E7C7
:109CB0000025ECE70025EBE70E49182043F08CFE69
:109CC000E4009DF824309DF81C10089A039E04734C
:109CD000049CC373002306618573846041734260F2
:109CE00003750AB070BD00BF981C0900E1FB0700B6
:109CF000FBF607005C5D08002DE9F0411C460D46AF
:109D000092B011462846824A18F064FA2668814BC0
:109D10003340062B05D0B10710D132687E4B9A42F2
:109D200008D144F2562231467C4842F061FC820759
:109D3000064603D132687A4B9A4202D0794836F00F
:109D400013F9012D14D9062208A960681CF00CF83B
:109D500040F272230998089F4FF48062082118F09E
:109D600031FB4307054605D06F48082136F018F946
:109D700000252F466D49402043F02EFE0446066321
:109D80000022002306F108003FF000FF206B1022A4
:109D90006B460DEB0201083040F0E5F910B10520EB
:109DA00036F0AEF8009B102B0BD16149042204A8B9
:109DB00042F037F928B95F49082206A842F031F984
:109DC00018B14FF4437018F02FFA206B04226B4641
:109DD0000DEB0201083040F0C6F90028DFD1009BEE
:109DE000042B02D1019A282A02D9534836F0D0F820
:109DF000206B6B4608A9083040F0B5F90028CED199
:109E0000019A282A03D0BDF82030012B0CD1BDF8CF
:109E10002210022908D8BDF82E30102B04D8122A9F
:109E200004D1BDF830208AB14448DFE7282A0DD19B
:109E3000BDF820004FF6FE729042F5D1BDF83820F3
:109E4000012AF1D1BDF832209A42EDD1082B099AAE
:109E5000237394BF00230123A3734FF40073A36003
:109E6000002362606173E373206B6B46042202A9D6
:109E7000083040F078F9002891D1009E042E8ED150
:109E80002F49324602A842F0CCF88046206B6B4640
:109E9000324603A9083040F066F900287FF47FAF0E
:109EA000009B042B7FF47BAF206B039AB8F1000F6B
:109EB0000AD0D0E91013521843F1000308303FF0E4
:109EC00065FE0028D0D06AE72262036CA38465B9DE
:109ED0004FF48070E06241F0E2FF03462061E06AE7
:109EE00063B9A561657335F0CDFF6D0827612F4417
:109EF000E562A761204612B0BDE8F08141F0CFFFD6
:109F0000A0610028F6D1E06A25616573EBE700BF28
:109F1000040002000F0080FF64E30700D005080082
:109F2000F010090060EE07009AF907003C5D080098
:109F30009DD40700A2D4070040F70700E5F707000B
:109F4000CAA007002DE9F04F2DED048B95B0044613
:109F50000C920993426A002943D00C9B012B00D13B
:109F6000826A229BA1691960216A237F914240F095
:109F70002484D4E90421002B18BF1146099B0791C2
:109F80001960237F83F001032377A3699B080B9358
:109F900004F130030E9300230D93069394F82C30B4
:109FA0000D9A93421FDC069B3BB9079A0B99069BBF
:109FB00002EB8101914240F0E083A37B002B00F093
:109FC000DF83236A013323620C9B002B40F0FC8368
:109FD000636A01336362012015B0BDEC048BBDE8F8
:109FE000F08F0C91BDE70E9B53F8045F0E93AB68A6
:109FF0000A93002B40F0B5830D9B01330D93CDE701
:10A00000AB60069B002B00F0B18301230693F3E7BE
:10A010006B699B086B61431E5842584168730A98EC
:10A02000617B407BD5F810B06B6988424FEA012212
:10A0300040F09D809A4228BF1A46089B934294BFE5
:10A0400005930592059B6068B3FBF1F189B230F08E
:10A0500029FAF7EE000A05F118009FEDB50A4BF05A
:10A060008CFFDFEDB40AB0EE408A05F11C009FEDD5
:10A07000B20A4BF09EFFDFEDB17A627B28EE278AB1
:10A08000022ABCEEC88A18EE103A9BB2029374D131
:10A0900010F4004F47F6FF73029909BF1B1AC0184E
:10A0A0009BB24FF400401CBF80B24FF400434B43BF
:10A0B0004843C113DB13039102932B6A11936B6A1C
:10A0C000129306980A9B217B5B7B0026139600283F
:10A0D00040F08681102940F0FA80A17B002900F031
:10A0E00084809A427FD0DDF810A0DDF81880059BAF
:10A0F000434565D95BF81890039B01931FFA89F0DB
:10A10000029B009340EA094012AB11AA13A93BF04D
:10A1100053FE119E360436FB00F6129F3F0437FBB8
:10A1200010F726F3CF3627F3CF37C6EA07464AF8AB
:10A13000086B4FEA1940039E01960004029E0096A8
:10A1400040EA19403BF038FE119B1B0433FB00F33F
:10A15000129A120432FB10F223F3CF3322F3CF32E0
:10A16000C3EA02434AF8043C08F10208BFE75B0077
:10A17000934228BF1346089A60E7029B03939CE72B
:10A18000039B5BF826000193029B009311AA12AB7C
:10A1900013A93BF011FE119B1B0433FB00F3129A31
:10A1A000120432FB10F223F3CF3322F3CF32C3EA8F
:10A1B0000243049A42F826300136059BB342DFD1B0
:10A1C000059A089B607B9B1A0893049B03EB820310
:10A1D00004930A9B5B7B9842D5E9041200F09482B9
:10A1E000059B5B0891E2069EE7E79A426BD0DDE9AA
:10A1F00004A35B080BEB8303D9460F934FF0802B2E
:10A200000F9B4B45DCD059F8043B93FA4BF8039B6A
:10A2100001931FFA88F0029B009340EA084012ABBA
:10A2200011AA13A93BF0C8FD119E360436FB00F6B7
:10A23000129F3F0437FB10F726F3CF3627F3CF37B3
:10A24000C6EA07464AF8086B4FEA1840039E019693
:10A250000004029E009640EA18403BF0ADFD119BC1
:10A260001B0433FB00F3129A120432FB10F223F3A7
:10A27000CF3322F3CF32C3EA02434AF8043CBFE7AC
:10A280005BF8260090FA47F0039B0193029B009332
:10A2900011AA12AB13A93BF08FFD119B1B0433FBDA
:10A2A00000F3129A120432FB10F223F3CF3322F39D
:10A2B000CF32C3EA0243049A42F826300136059BA6
:10A2C000B342DDD17CE7069E4FF08027F7E79A4244
:10A2D000059B4FEA430933D1069E4FF080274E4538
:10A2E000BFF46EAF3BF816004CF09FFFA37B0BB999
:10A2F00090FA47F0039B0193029B009311AA12ABC3
:10A3000013A93BF059FD119B1B0433FB00F3129A78
:10A31000120432FB10F223F3CF3322F3CF32C3EA1D
:10A32000024049F0EFF9049B23F816000136D6E706
:10A330000000000000FE7F3F00FE7FBF00000047DE
:10A34000069F4FF080287B1C4B45BFF439AF3BF88C
:10A3500007004CF06AFFA37B06460BB990FA48F65B
:10A36000039B0193B0B2029B009340EA064012ABFC
:10A3700011AA13A93BF020FD119B1B0433FB00FC29
:10A38000129B1B0433FB10F32CF3CF3C23F3CF338E
:10A39000CCEA034049F0B6F9049B23F81700039B6D
:10A3A0000193300C029B0093000412AB40EA16406C
:10A3B0003BF002FD119B1B0433FB00F3129A1204C5
:10A3C00032FB10F223F3CF3322F3CF32C3EA024041
:10A3D00049F098F9049B023323F817000237B2E7DB
:10A3E000102940F0F880A17B002975D09A424CD00A
:10A3F000DDE90483D9464FEA530B09EB8B0BD945B2
:10A400003FF4DEAE59F804AB039B01931FFA8AF0C8
:10A41000029B009340EA0A4012AB11AA13A93BF039
:10A42000CBFC119E360436FB00F6129F3F0437FB2F
:10A4300010F726F3CF3627F3CF37C6EA074658F88A
:10A44000080B96FA10F648F8086C4FEA1A40039E7B
:10A4500001960004029E009640EA1A403BF0ACFCD4
:10A46000119B1B0433FB00F3129A120432FB10F20F
:10A4700023F3CF3322F3CF32C3EA024358F8042C3C
:10A4800093FA12F348F8043CB9E7049B1F1F059B9D
:10A490000BEB8308C3453FF493AE039B5BF8040BBF
:10A4A0000193029B009311AA12AB13A93BF084FC09
:10A4B000119B1B0433FB00F3129A120432FB10F2BF
:10A4C00023F3CF3322F3CF32C3EA024357F8042FEA
:10A4D00093FA12F33B60DDE79A4251D0DDE9049331
:10A4E0005B080BEB8303DA460F934FF0802B0F9B37
:10A4F0009A453FF465AE5AF8043B93FA4BF8039B38
:10A5000001931FFA88F0029B009340EA084012ABC7
:10A5100011AA13A93BF050FC119E360436FB00F63D
:10A52000129F3F0437FB10F726F3CF3627F3CF37C0
:10A53000C6EA074659F8080B96FA10F649F8086C6F
:10A540004FEA1840039E01960004029E009640EADE
:10A5500018403BF031FC119B1B0433FB00F3129AB3
:10A56000120432FB10F223F3CF3322F3CF32C3EACB
:10A57000024359F8042C93FA12F349F8043CB6E765
:10A58000049B1F1F059B4FF080290BEB8308C345DD
:10A590003FF416AE5BF8040B90FA49F0039B01936D
:10A5A000029B009311AA12AB13A93BF005FC119B6F
:10A5B0001B0433FB00F3129A120432FB10F223F354
:10A5C000CF3322F3CF32C3EA024357F8042F93FA72
:10A5D00012F33B60DBE705999A424FEA410A40F0EB
:10A5E0008E80049B4FF080289F1E5645BFF4E8AD37
:10A5F0003BF816004CF019FEA37B0BB990FA48F01B
:10A60000039B0193029B009311AA12AB13A93BF089
:10A61000D3FB119B1B0433FB00F3129A120432FB91
:10A6200010F223F3CF3322F3CF32C3EA024237F8DA
:10A63000020F4CF0FAFD92FA10F049F063F801367F
:10A640003880D2E73BF806004CF0EFFDA37B0746CD
:10A650000BB990FA49F7039B0193B8B2029B0093A0
:10A6600040EA074012AB11AA13A93BF0A5FB119BCE
:10A670001B0433FB00FE129B4FEA034C3CFB10FC17
:10A680002EF3CF332CF3CF3CC3EA0C430F93049B40
:10A6900033F816004CF0C9FD0F9B93FA10F049F007
:10A6A00031F8049B23F81600039B0193380C029B9E
:10A6B0000093000412AB40EA17403BF07DFB119B76
:10A6C0001B0433FB00F3129A120432FB10F223F343
:10A6D000CF3322F3CF32C3EA0242049B33F818008F
:10A6E0004CF0A3FD92FA10F049F00CF8049B0236EE
:10A6F00023F8180008F10208C245A3D860E54FF01E
:10A7000001084FF08029F7E7059B01EB8301D21A7E
:10A71000C5E90412029B2B62039B6B62089B002B12
:10A720003FF473AC6B69002B7FF479AC6B7B33B96E
:10A730002B7B002B3FF464ACA8683CF03EFAA86881
:10A7400000283FF46CAC05F1140205F110013CF057
:10A75000F0F902287FF45CAC0023AB606B616B7393
:10A760004FE40B9B0893079B0493D7E7089B06993C
:10A7700004989A0041F0AAFC47E442F8043B19E42B
:10A78000237B0B9A102B079B03EB82020AD04FF01E
:10A7900080309A423FF415AC196881FA40F143F8D1
:10A7A000041BF6E74FF0802093423FF40AAC19688F
:10A7B00091FA40F143F8041BF6E71BB92369099AA3
:10A7C000136001E46369FAE70C9B012B7FF403AC8F
:10A7D000A36A227B0133A362099B1B6803EBD203AC
:10A7E000099A1360FFF7F7BB2DE9F04788B00846D8
:10A7F00011461A4602AB0193364B0093062341F0F3
:10A80000C0FD40F21953FF220121029841F0E4FDFE
:10A8100040F28223064602220498012141F0DCFD29
:10A82000079D002D804604DC40F26B41012017F0AB
:10A830009BFDDDF814A0BAF1080F05D0BAF1100F96
:10A8400002D0254835F0A4FB06F10D002349800015
:10A8500043F0C2F8039F9DF818900446F808800062
:10A86000A06141F01CFB03462061A0691BB9637322
:10A87000636135F007FB41F012FB606118B960734A
:10A880002061A069F5E765600025A76084F80CA049
:10A8900084F80E9084F80D80E57384F82C6004F140
:10A8A0003007B5420ADB94F82C0004F134011EF0A5
:10A8B0004BFD2063204608B0BDE8F0870023084820
:10A8C0001A46194600F06AF8013547F8040F44604B
:10A8D000E7E700BF6C220900AAF10700C05B08008F
:10A8E00050220900F0B50C4687B054F8045B0646C8
:10A8F000687B17463CF018F903AB0193124B0093A9
:10A900003A4603232146701E17F09CFC95F82C2034
:10A910009DF810309A4203D84FF4A36017F084FCDE
:10A9200005EB8303039E5C6B9DF814706068012245
:10A93000314601F013FF2046A66027733CF04DFF1F
:10A94000284607B0F0BD00BF38220900F0B50D461B
:10A9500085B055F8044B0646607B17463CF0E4F89A
:10A9600003AB01930C4B00933A4601232946701E1A
:10A9700017F068FC94F82C209DF80C309A4203D80C
:10A980004FF4A36017F050FC04EB83040022636BC8
:10A990000E209A6005B0F0BD3022090010B50846BF
:10A9A0001146002217F016FC0B49282043F014F83A
:10A9B00000230446836000F1180140F28332074807
:10A9C00032F026FD064840F2ED3204F11C0132F06F
:10A9D0001FFD204610BD00BF50220900020000C02C
:10A9E000020080807FB502AB51F8044B01930B4B02
:10A9F00000930138022317F025FC029D60689DF842
:10AA00000C600122294601F0A9FE2046A5602673AC
:10AA10003CF0E3FE0E2004B070BD00BF2022090010
:10AA20001FB503AB0193064B51F8044B009301385B
:10AA3000012317F007FC00230E20A36004B010BD13
:10AA4000182209002DE9F04FAFB0446A04901CB9F8
:10AA5000389B1C60022021E0002904998968149128
:10AA60003899149C0C60049991F9541008BF002285
:10AA70008A42049915D1049891F9551000EB81018F
:10AA8000496B01EB42021A60FF2380F85430389B77
:10AA90001A68836D03EB5203836501202FB0BDE874
:10AAA000F08F91F84410049CB1FA81F1490984F8BF
:10AAB000441084F85510C2F1010204EB810184F8BE
:10AAC00054204A6B1A60069241F097FB04980021CB
:10AAD00041F06EFB049B044670B99A6801460698E3
:10AAE00041F0F4FA389B1C60049B93F8450080F019
:10AAF00001004000C0B2D1E7049ADB6A126BD21A9F
:10AB00000992049A12690392002A01F01685049AA8
:10AB10000398576A1F44394639F01AFF421C06460B
:10AB200001F00F85039BD3F80090B9F1000F00F0FE
:10AB30003D81D3F80480B8F1000F00F0378199F817
:10AB400000B099F81C303C18BBF1000F3ED1032B2C
:10AB50004FF0090114BF4FF0200A4FF0110A2AA844
:10AB6000CDE92A4BCDE92CBA4DF02EF8C8F80000FB
:10AB700099F81C30032B14BF032105212AA84DF09E
:10AB800023F8454645F8040F039BD3F8BC379B4593
:10AB90000DDB4FF0000B039BD3F8C4379B4580F2CD
:10ABA000C880902303FB0B850023059392E005F1F9
:10ABB000100301212AA805934DF006F8059B45F8DE
:10ABC000040F9D42F5D10BF1010BDDE7032B4FF094
:10ABD000080114BF4FF0110A4FF0090A00232AA8F8
:10ABE000CDE92B332A94CDF8B4A04CF0EDFFC8F892
:10ABF000000099F81C30032B14BF022101212AA860
:10AC00004CF0E2FFC8F80400C3E70C212AA84CF07E
:10AC1000DBFF0921A8622AA84CF0D6FF0821E862D0
:10AC20002AA84CF0D1FF286399F80030002B14BFFC
:10AC3000092104212AA84CF0C7FF012168632AA832
:10AC40004CF0C2FFA863002856D002212AA84CF07D
:10AC5000BBFF0121E8632AA84CF0B6FF0521286458
:10AC60002AA84CF0B1FF052168642AA84CF0ACFF7B
:10AC70000023EB64A86403212AA84CF0A5FF03215C
:10AC800028652AA84CF0A0FF032168652AA84CF08B
:10AC90009BFFEB6BA86533BBC5E90A336B63E86DBB
:10ACA000C0F11400286699F80030002B3FD1012133
:10ACB0002AA84CF089FF686601212AA84CF084FF7D
:10ACC0000121A8662AA84CF07FFF059BE8660133A6
:10ACD00005934835039B059AD3F8BC379A4294DB19
:10ACE0000BF1010B57E7022B04D12B6C13B908238E
:10ACF000EB65D4E70723FBE7C5E90F0005212AA888
:10AD00004CF062FF052168642AA84CF05DFF052124
:10AD1000A8642AA84CF058FF0421E8642AA84CF043
:10AD200053FF0321E8652AA84CF04EFFBAE7002044
:10AD3000C1E7039A0999D8F80080C2F8D88706EBD2
:10AD40000A028A1A03990992D1F8B817039A04EBF8
:10AD50000A05D2F8B02700295AD0002A40F0A48072
:10AD6000039BD3F8CC27099B934280F2AE800699CF
:10AD700003983AF00BFB4FF0FF34149A0698002129
:10AD800041F0A4F9049B93F845300BB903341BD868
:10AD9000049B06989A68002141F098F9389A00239C
:10ADA0001360049A012382F8453053E6069903980C
:10ADB0003AF0ECFA6FF00604049B099A1B6B9B1A9D
:10ADC000049AD362002CD8D1049B149A9B6D03EB98
:10ADD0005203049A9365104641F00FFA049800213B
:10ADE00041F0E6F9049B049A1B6BD26A9A1A049B01
:10ADF0009B6A9B1AB3F5007F044607DD049AAE4BAD
:10AE000002F11400C2E9053201F0ECFC204645E6EF
:10AE1000002A49D10399DDF824B00122C1F8B027F6
:10AE2000A9465946484605933AF0C4FA431C059B87
:10AE300018D019F800C039788C4509EB00021DD1F3
:10AE400092F801C079788C4518D197F802C09178B2
:10AE50008CEA0101032911D81CF0020F18BF02F17E
:10AE6000FF32501B039A0028C2F8B4070CDA069987
:10AE700010463AF08BFA6FF002049DE7033002F1BE
:10AE80000309ABEB000BCCE7039A0644D2F8C027CA
:10AE900056445643039AD2F8C8275343039AF60000
:10AEA00096FBF3F3C2F8B837039BD3F8B4271B68BB
:10AEB00043B15B69003B18BF01231344039AC2F8F6
:10AEC000CC374DE74FF0FF33F7E7039B0399D3F8F7
:10AED000DC37434501F11C003DDBA3EB0801424692
:10AEE00041180A9041F0DCF8039BD3F8D807D3F857
:10AEF000CC270A9B2946184441F0A7F8039B0399E5
:10AF0000D3F8CC27D3F8D8371344C1F8DC37DB00AB
:10AF10001093039B099903F2DC738A1A1A93002396
:10AF200009920C930593039B059AD3F8C4379A4270
:10AF300081F21E837C23534311939023534319932F
:10AF4000119B013B1F93119B08931A9B189300239D
:10AF50000D939B46FEE32946184441F076F8039B87
:10AF60000399D3F8CC27D3F8DC3703981344C1F8FE
:10AF7000DC37099B06999B1A09936FF001043AF09C
:10AF800005FA19E7039B1E68002E00F0D4805B6869
:10AF90000793002B00F0CF80039B9D68002D00F0ED
:10AFA000CA800A9B22930023CDE923330C9A109B7D
:10AFB0009A18D31D48BF02F10E03DB1025930C9B9A
:10AFC0001BB1194622A84CF0FFFD059B3178902259
:10AFD0005A43482303FB0B22079B1A44536BD2F8B6
:10AFE0003CC0002940F04E81344810F8136000EB5B
:10AFF0004300BCF1020F477862D1D2F84090B9F11A
:10B00000000F10D0089B884605EB0309314622A8A3
:10B010004CF0DAFD08F10108B8F1080F09F8010B4E
:10B02000F4D14FF00309119B05EB03080D9B9844E5
:10B0300009EB49039844314622A84CF0C5FD31463E
:10B0400088F8170022A84CF0BFFD314688F8180098
:10B0500022A84CF0B9FD09F10109B9F1060F88F8F1
:10B06000190008F10308E6D1089BEE18394622A81A
:10B070004CF0AAFD394686F8290022A84CF0A4FD20
:10B08000394686F82A0022A84CF09EFD09F10109F4
:10B09000B9F10C0F86F82B0006F10306E6D1059AEC
:10B0A0007C2353433E2202FB0B332B44002283F8C4
:10B0B0003B209A8724E000BF712104001C55090041
:10B0C000059B002B3ED10D9BDDF8148005EB030999
:10B0D000314622A84CF078FD08F10108B8F10B0FB9
:10B0E00009F8010BF4D10D9B1D44394622A84CF000
:10B0F0006BFD05F8080008F10108B8F1150FF4D14F
:10B10000059B189A90265E434820079B00FB0B6620
:10B1100033449B6A5360229B0A9A9B1A249AC2EB7F
:10B12000C302D71007D4189B53F804CF1893109B71
:10B13000634580F2ED81069903983AF027F96FF0A4
:10B14000070439E64FEA0B13079A083302EB0309A9
:10B1500052F80380B8F1000F1FD00D9B8846EB1802
:10B160001F9913F8012B5A5408F10108B8F1060F82
:10B17000F6D1D9F80430FBB9089B4FF0060805EB6F
:10B18000030A314622A84CF01FFD0AF8080008F116
:10B190000108B8F10B0FF4D121E0089B05EB030A7D
:10B1A000314622A84CF010FD08F10108B8F1060F55
:10B1B0000AF8010BF4D1DCE7059C3E2303FB0BF3FB
:10B1C0007C20EA1800FB04332B4491799971D179E2
:10B1D000D971117A1972517A5972927A9A72D9F890
:10B1E00008306BB9089B0B2605EB0308394622A8EB
:10B1F0004CF0EAFC08F806000136102EF6D112E0F9
:10B20000059C3E2303FB0BF37C20EA1800FB043370
:10B210002B44D17AD972117B1973517B5973917B6D
:10B220009973D27BDA73D9F80C306BB9089B10266E
:10B2300005EB0308394622A84CF0C6FC08F80600C6
:10B240000136152EF6D112E0059C3E2303FB0BF3CD
:10B250007C20EA1800FB04332B44117C1974517CC8
:10B260005974917C9974D17CD974127D1A75059AA0
:10B270007C2353433E2202FB0B332B4400225A759E
:10B280009A753DE7366A16F0010603D0BBF1010F4F
:10B2900000F0B280B3F5C87F7BDA1911052291FB6B
:10B2A000F2F2269202EB8202891AC3F381022892FB
:10B2B00003F0030300222791299311461346BCF1A2
:10B2C000020F40F0CE80059C902060434827079CE9
:10B2D00007FB0B002044006C002808BF4FF0010C56
:10B2E00001EB41018948614410F821702A9700EB75
:10B2F000810148782B908878C9782C902D910EB3D5
:10B30000BBF1010F1ED10DF1980C05F1FC070DF1F9
:10B31000A80E664603CE764538607960B44607F1DC
:10B320000807F6D10DF1A80C05F58677664603CE21
:10B3300079602EA98E423860B44607F10807F5D12E
:10B34000C5F8F820059990224A43482101FB0B22B9
:10B3500007990A445366D36B022B40F0C580176CE3
:10B36000002F00F0A880089B0026EF18269922A83D
:10B370004CF02AFC0136062E07F8010BF6D14FF0EF
:10B3800001080327119B05EB030A0D9B0AEB03043D
:10B390008BE0B3F5FA7F12DAA3F5C8739910052292
:10B3A000B1FBF2F2269202EB8202891A03F0030348
:10B3B0000022279128932992134601217FE7A3F5C4
:10B3C000FA730321B3FBF1F101EB410205982691D9
:10B3D0009B1A0022CDE9282290224243482000FBFC
:10B3E0000B22079827930244126C0AB1CDE9271368
:10B3F00000220123022162E7B3F5B47F03F00102CA
:10B400004FEA630110DA242091FBF0F3269300FB4E
:10B410001313062093FBF0F100FB11332893002354
:10B420002791299303214AE7F3290CDCB4390B1146
:10B430002693C1F38103279301F003010023289190
:10B44000299304213BE7F4390323B1FBF3F326935B
:10B4500003EB4303C91A00232791CDE928330521C3
:10B460002DE74FF0000C3BE726AB22A853F828A0AD
:10B4700051464CF0A9FB5146F07522A84CF0A4FBB4
:10B480005146307622A84CF09FFB033609F10109A2
:10B49000B0752AAB53F828209145E5DB08F1010887
:10B4A000B8F1040F3FF4FBAD4F4407EB47062644C9
:10B4B0004FF00009EDE7B84664E753F8261022A8DC
:10B4C0004CF082FB09F8010B013726AB5AF8262015
:10B4D0009742F2DB0136042E0DD0B84404EB080984
:10B4E00000270DF1A80AF1E7089B4FF00008EC18BF
:10B4F000464626ABF2E7059A7C2353433E2202FBE5
:10B500000B331D440023AB756B75F9E53C55090001
:10B51000039B1D68002D00F0C2815B680B93002B1C
:10B5200000F0BD81039B9B68002B00F0B881039B5A
:10B53000D968002900F0B38102F0070313930C9B34
:10B54000139AC3EBC70313441C93BCEB0303079389
:10B5500000F1A5810A9B6A6B3B441D930B9B1E4423
:10B56000B36B002B00F02381F36B022B40F01F81A3
:10B57000336C002B40F00381059C9023634300FB58
:10B580000B330B9803440320DB6D013393FBF0F383
:10B5900002EB4303B3F92E0000EB40004FF41072AE
:10B5A000059C9023634348250B9C05FB0B332344E8
:10B5B000DB6A5B00B3F5107FA8BF4FF410739342B2
:10B5C000D4BF2C932C920A932D938342D4BF2B93F8
:10B5D0002B9001EB8B03209303F580530A9AC3F859
:10B5E00000224FF4106303FB0B131593139B0F936F
:10B5F0001D9B0C93002316930E93199B4033E31865
:10B6000021930E9B169F01332AAA0E9352F82330E2
:10B610001693A3EB070EBEF1000F23DD159B0E9AC8
:10B620000C9903EB8707219B53F82250B14B03EB96
:10B63000C5031E790F9B5A4202F0070213462AB136
:10B6400011F8010BC2F1200200FA02F2002E40F0C4
:10B65000C08033463A1D47F8263042F8263002367D
:10B66000B645F8DC00230F9A0C991A4401EBE2016D
:10B6700002F007020F92079A0C91D31A07930E9BC0
:10B68000032BBED1109B1C9A9B1A0E93079B002B79
:10B6900000F09F82159B0A9A0C9803EB8205059A8D
:10B6A00090235343482202FB0B330B9AD318924A40
:10B6B000DB6E52F823200B92904A52F823100F9B16
:10B6C0005B4203F007031A462BB110F8016BC3F17C
:10B6D000200306FA03F3079CA61A0A9C4FF0000900
:10B6E000C4F50F7AC1F120014F460AF1010A0A910F
:10B6F000BA4500F3F081209B03F58052D2F8003266
:10B700003B44C2F800320022B3F5107FC0F26382DE
:10B71000079A0F9B13440C9A02EBE30203F0070312
:10B720000C93089B0A923E3308930D9B3E330D9376
:10B73000199B4833199313461D9A9B1A00F1AF8049
:10B74000139AC2EBC3030C9A13440E9AD31A1093A4
:10B750000BF1010B039BD3F8BC379B45FFF612ACF2
:10B760000599039837F008FD013040F05785069998
:10B77000039839F00BFE6FF00904FFF71DBB2B781F
:10B780005BB9059C9023634300FB0B330B98034488
:10B79000DB6D013332F9130000E7B2F93600B2F97C
:10B7A0003430C31AB2F90C0000EB4300F6E6059BF7
:10B7B00090255D43482303FB0B550B9B1D44EB6D0C
:10B7C0002D6E013332F913002B44013332F913206B
:10B7D000E6E64B4850F825C04A4800EB4C0017906D
:10B7E0000798012EA0EB030040F08E80454C34F802
:10B7F0001C6006F00F064FF000094FF0004AC6F13A
:10B8000020060F2853DD8C46C3F118081CF8025B94
:10B81000497805FA08F5C3F1100801FA08F10D435B
:10B820002A431033103861460A2BEADD22FA06F566
:10B83000179C013534F815504FEA153C15F0F00F00
:10B8400002FA0CF218BF02F0004CA3EB1533C5F35B
:10B8500003181EBF520003F1FF334CEA080815F429
:10B86000706FC5F3032C1FBF03F1FF3302F00045D7
:10B8700045EA0C0C52004B4511DB47F8088BAEF142
:10B88000020EBEF1000F47F804CCCDDCA3EB090398
:10B89000079A0344D31A079A93427FF6E4AE0699B7
:10B8A000039839F073FD6FF00804FFF785BA1D188F
:10B8B000002DF4DD002812DD082891F800C0C8BF73
:10B8C0004878C3F118080CFA08FCC8BFC3F110038C
:10B8D00042EA0C02C9BF98400131024302316B1E9B
:10B8E0004AFA03F31A404FF00B0905F10B0300204D
:10B8F0009AE700BF18320900145509000C550900D9
:10B900003C54090018330900A6F1020CBCF1010FE8
:10B91000C5D8DFF8F0C25CF83580DDF85CC00024E3
:10B92000129408F101041B94C8F120041E940F28FE
:10B9300027DD8946C3F1180A19F8025B497805FA30
:10B940000AF5C3F1100A01FA0AF10D432A43103334
:10B95000103849460A2BEADDBCF8009009F00F09BF
:10B96000C9F1200522FA05F501353CF815505FEACA
:10B97000153A2AD1A3EB090302FA09F20CEB450CA4
:10B98000E8E7C518002D8ADD002812DD082891F8A7
:10B990000090C8BF4878C3F1180A09FA0AF9C8BF6D
:10B9A000C3F1100342EA0902C9BF984001310243C2
:10B9B00002314FF000406B1E40FA03F30B201A4097
:10B9C000129005F10B030020C4E7C5F30319B9F188
:10B9D0000F0FA3EB0A0302FA0AF2C5F3032523D1E2
:10B9E000032E24D11B9C03EB000C002D0CBFA246A0
:10B9F00004F1010AE2453FF752AF9C46E24552DCB2
:10BA00000344B3EB0C0006D5581E9C464FF0004390
:10BA100003411A4000201E9B22FA03F909F10F0985
:10BA2000ACEB080302FA08F2B9F1000F05D002F0FE
:10BA3000004C49EA0C095200013B0F2D1DD1032E89
:10BA40001CD11B9C1D18AC423FF729AF9C461B9C88
:10BA5000644533DC0344B3EB0C0006D5581E9C460A
:10BA60004FF0004303411A4000201E9B22FA03F5C9
:10BA70000F35ACEB080302FA08F22DB102F0004CCE
:10BA800045EA0C055200013B129CA342FFF607AFAA
:10BA9000AEF1020EBEF1000FC7E9009518DDDDF82A
:10BAA0005CC0083756E711F8019BCCF1180409FA7D
:10BAB00004F942EA09020CF1080C9FE711F8015B56
:10BAC000CCF1180A05FA0AF52A430CF1080CBEE776
:10BAD000129A9B1ADCE60F2E56DD8446C2F1180E30
:10BAE0001CF8021B407801FA0EF1C2F1100E00FAA8
:10BAF0000EF001430B431032103E60465745BFF62F
:10BB0000F7AD092A7FF7F4AD0A990B9C23FA01F1EE
:10BB100021443B4C615C4FEA111C03FA0CF311F019
:10BB20000808A2EB11121FBF03F0004802F1FF3218
:10BB30005B0048F0010811F0040E1FBF03F0004E37
:10BB400002F1FF325B004EF0010E11F0020C1FBF3C
:10BB500003F0004C02F1FF325B004CF0010C11F0DD
:10BB600001011FBF03F0004102F1FF3241F001016A
:10BB70005B004A45FFF6BFAD45F8108B043745E939
:10BB800003EC45F8041CB9E7B11800297FF7B3AD01
:10BB9000002E12DD082E90F800C0C8BF4678C2F112
:10BBA000180E0CFA0EFCC8BFC2F1100243EA0C03D7
:10BBB000C9BF96400130334302304A1E4FF0004463
:10BBC00044FA02F213404FF00A0901F10A0200267A
:10BBD00094E7079F8FE5159941F82320013393E5FA
:10BBE000059903982A4638F087FA01300CD1069956
:10BBF000039839F0CBFB6FF00A04FFF7DDB800BF04
:10BC0000BC540900183209000135039BD3F8BC3736
:10BC10009D42E5DB039AD268002A00F08684039AED
:10BC200052690B92002A00F08084039A926907926D
:10BC3000002A00F07A84039AD2F8C867059A56431E
:10BC4000069A5E43022B02EB460640F0E9820B9B0C
:10BC50001193331D089300230E93079B03F50053A4
:10BC60000D930E9B0D9A0799119803F001030F9302
:10BC70000B9B03F580554FF00077D5F8183B0093E8
:10BC8000D2F800220F9B37F017FFD5F81C3B0D9A16
:10BC9000079911980093D2F800220F9B803100F58C
:10BCA000106037F009FF0F9B0D9A5B42D2F800221B
:10BCB00003F488631344079A02EB830B4FF0000CE4
:10BCC00052F82320DBF85C306046C2FB007C6FF04A
:10BCD0007301C3FB017C4FF00076DBF88020DBF8BA
:10BCE000DC300546C2FB0065C3FB01654FF45579A6
:10BCF000DBF80430DBF85820C3FB097C834BC2FB24
:10BD0000037CDBF88410DBF8D820C1FB0965C2FB9B
:10BD1000036541F6D478DBF80830DBF85420C3FB28
:10BD2000087C7B4BC2FB037CDBF88810DBF8D4205B
:10BD3000C1FB0865C2FB036546F2B86EDBF80C3048
:10BD4000DBF85020C3FB0E7C724BC2FB037CDBF89C
:10BD50008C10DBF8D020C1FB0E65C2FB03656E4A78
:10BD6000DBF81030DBF84C10C3FB027C6B4BC1FBE3
:10BD7000037CDBF89000DBF8CC10C0FB0265C1FB54
:10BD80000365DBF81420DBF84830C2FB0E7C45F27B
:10BD90008401C3FB017CDBF89420DBF8C830C2FBD4
:10BDA0000E65C3FB0165DBF81820DBF84430C2FBED
:10BDB000087C40F22C71C3FB017CDBF89820DBF897
:10BDC000C430C2FB0865C3FB0165DBF81C20DBF84F
:10BDD0004030C2FB097C7421C3FB017CDBF89C2052
:10BDE000DBF8C030C2FB0965C3FB01650C24384693
:10BDF0004FF014080CFA04F34CFA08FC20FA08F08F
:10BE000040EA030039F0F6F9089B23F8040C3046A9
:10BE100005FA04F345FA08F520FA08F040EA0300B1
:10BE200039F0E8F9089B0BF5805723F8020C3B68C2
:10BE30004FF4D0704FF000724FF0000CC3FB002C99
:10BE40004FF00073D7F880100026C1FB003641F692
:10BE50007C007968C1FB002CD7F88410C1FB003648
:10BE600049F2FC70B968C1FB002CD7F88810C1FBFF
:10BE700000362B49F868C0FB012CD7F88C00C0FBBA
:10BE8000013628493D69C5FB012CD7F89050C5FB08
:10BE900001366FF0B3057969C1FB052CD7F8941012
:10BEA000C1FB05364FF41275B969C1FB052CD7F8F3
:10BEB0009810C1FB05366FF0130EF969C1FB0E2C0B
:10BEC000D7F89C101D46C1FB0E5610460CFA04F321
:10BED0004CFA08FC20FA08F040EA030039F08AF92D
:10BEE000089B9887284606FA04F346FA08F620FAD3
:10BEF00008F040EA030039F07DF9089B0A49D88729
:10BF000004331293089B043B13930FE0D4F8FFFF14
:10BF10007CAFFFFF3CB6FDFF78940400C4490200EB
:10BF20004CE803002464FFFFF82D0900D1F840E03D
:10BF3000DBF80051DBF85C014FF000730022C5FB19
:10BF40000E324FF000764C6C4FF00009C5FB0469CF
:10BF5000C4F1000CC0FB0C32C0FB0E69DBF8DC0145
:10BF6000DBF8804115904FF000774FF0000AC4FBDA
:10BF70000E7A4FF00075486C4FF00008C4FB005873
:10BF80001598C0FB0C7AC0FB0E58D1F848E0DBF8DE
:10BF900004C1DBF85801CCFB0E32CC6CCCFB04693D
:10BFA000C4F1000CC0FB0C32C0FB0E69DBF8D801F9
:10BFB000DBF884411590C4FB0E7AC86CC4FB0058B2
:10BFC0001598C0FB0C7AC0FB0E58D1F850E0DBF896
:10BFD00008C1DBF85401CCFB0E324C6DCCFB04697C
:10BFE000C4F1000CC0FB0C32C0FB0E69DBF8D401BD
:10BFF000DBF888411590C4FB0E7A486DC4FB0058ED
:10C000001598C0FB0C7AC0FB0E58D1F858E0DBF84D
:10C010000CC1DBF85001CCFB0E32CC6DCCFB0469BB
:10C02000C4F1000CC0FB0C32C0FB0E69DBF8D00180
:10C03000DBF88C411590C4FB0E7AC86DC4FB005828
:10C040001598C0FB0C7AC0FB0E58D1F860E0DBF805
:10C0500010C1DBF84C01CCFB0E324C6ECCFB0469FA
:10C06000C4F1000CC0FB0C32C0FB0E69DBF8CC0144
:10C07000DBF890411590C4FB0E7A486EC4FB005863
:10C080001598C0FB0C7AC0FB0E58D1F868E0DBF8BD
:10C0900014C1DBF84801CCFB0E32CC6ECCFB04693A
:10C0A000C4F1000CC0FB0C32C0FB0E69DBF8C80108
:10C0B000DBF894411590C4FB0E7AC86EC4FB00589F
:10C0C0001598C0FB0C7AC0FB0E58D1F870E0DBF875
:10C0D00018C1DBF84401CCFB0E324C6FCCFB046979
:10C0E000C4F1000CC0FB0C32C0FB0E69DBF8C401CC
:10C0F000DBF898411590C4FB0E7A486FC4FB0058DA
:10C100001598C0FB0C7AC0FB0E58D1F878E0DBF82C
:10C110001CC1DBF84001CCFB0E32CC6FCCFB0469B8
:10C12000C4F1000CC0FB0C32C0FB0E69DBF8C0018F
:10C13000DBF89C411590C4FB0E7AC86F1691C4FBC6
:10C1400000581599C1FB0C7AC1FB0E580C241846F7
:10C15000142102FA04F342FA01F220FA01F040EA53
:10C16000030039F047F8129B23F8040C38461427D3
:10C170000AFA04F34AFA07FA20FA07F040EA030041
:10C1800039F038F8129B23F8020C304609FA04F310
:10C1900049FA07F920FA07F040EA030039F02AF8D3
:10C1A000139BA3F87C00284608FA04F348FA07F822
:10C1B00020FA07F040EA030039F01CF8139B1699A7
:10C1C000A3F87E00129B04331293139B043B13933A
:10C1D000DE4B40318B420BF5807B7FF4A7AE0D9B8D
:10C1E0000F9AD3F800329B1A0D9A03F00703C2F896
:10C1F00000320E9B01330E93119B80331193089BE9
:10C20000803308930E9B122B7FF42BAD059B0133DB
:10C2100005931A9B08331A93FEF785BE0025F4E4B4
:10C22000079B4036002703F5005807F001030E93E3
:10C230000B9B0B98079903F5805300EBC710D3F8BD
:10C24000183B0093D8F8002207F0010337F034FCC4
:10C2500007F00103D8F800225B4203F4886313441B
:10C26000079A02EB8309002052F82310D9F85C20CA
:10C270004FF000730446C1FB04306FF07301C2FB42
:10C2800001304FF4557ED9F80420D9F85810C2FB7C
:10C290000E30AF4AC1FB023041F6D47CD9F80820F9
:10C2A000D9F85410C2FB0C30AA4AC1FB023046F246
:10C2B000B865D9F80C20D9F85010C2FB0530A64A51
:10C2C000C1FB0230A54AD9F81010C1FB0230A44AC4
:10C2D000D9F84C10C1FB0230D9F81410D9F8482015
:10C2E000C1FB053045F28401C2FB0130D9F81810BA
:10C2F000D9F84420C1FB0C3040F22C71C2FB013054
:10C30000D9F81C10D9F84020C1FB0E307421C2FBB3
:10C3100001300C2402464FF0140A184602FA04F3C6
:10C3200042FA0AF220FA0AF040EA030038F062FF0B
:10C3300009F5805126F8400C0A684FF00070002380
:10C340004FF4D075C2FB050341F67C054A68C2FB79
:10C35000050349F2FC758A68C2FB0503814DCA6872
:10C36000C2FB0503804A0D69C5FB02036FF0B305EC
:10C370004A69C2FB05034FF412758A69C2FB0503C3
:10C38000CA696FF01301C2FB010303FA04F243FA16
:10C390000AF320FA0AF040EA020038F02BFFDFF837
:10C3A000CCA126F8200CA6F140030D930896DAE9FB
:10C3B00010ECD9F80021D9F85C114FF0007000237F
:10C3C000C2FB0E034FF000754FF0000BC2FB0C5B7D
:10C3D000CCF10002C1FB0203C1FB0E5BDAE912ECF7
:10C3E000D9F80411D9F85821C1FB0E03C1FB0C5B2D
:10C3F000CCF10001C2FB0103C2FB0E5BDAE914ECD5
:10C40000D9F80811D9F85421C1FB0E03C1FB0C5B0C
:10C41000CCF10001C2FB0103C2FB0E5BDAE916ECB2
:10C42000D9F80C11D9F85021C1FB0E03C1FB0C5BEC
:10C43000CCF10001C2FB0103C2FB0E5BDAE918EC90
:10C44000D9F81011D9F84C21C1FB0E03C1FB0C5BCC
:10C45000CCF10001C2FB0103C2FB0E5BDAE91AEC6E
:10C46000D9F81411D9F84821C1FB0E03C1FB0C5BAC
:10C47000CCF10001C2FB0103C2FB0E5BDAE91CEC4C
:10C48000D9F81811D9F84421C1FB0E03C1FB0C5B8C
:10C49000CCF10001C2FB0103C2FB0E5BDAE91EEC2A
:10C4A000D9F81C11D9F84021C1FB0E03C1FB0C5B6C
:10C4B000CCF10001C2FB0103C2FB0E5B0C24142172
:10C4C00003FA04F243FA01F320FA01F040EA020011
:10C4D00038F090FE0D9B23F8020F14210D9328468F
:10C4E0000BFA04F34BFA01FB20FA01F040EA0300D7
:10C4F00038F080FE089B23F8020D0893134B0AF1D5
:10C50000400A9A4509F580797FF451AFD8F8003296
:10C510000E9A01379B1A03F00703122FC8F8003256
:10C5200006F140067FF481AE70E60699039838F074
:10C530002DFF6FF00B04FEF73FBC6FF00404FEF715
:10C540003BBC6FF00504FEF737BC00BFB8310900F3
:10C55000D4F8FFFF7CAFFFFF3CB6FDFF78940400EA
:10C56000C44902004CE803002464FFFFF82D0900D1
:10C570000024FEF721BC00BF2DE9FF411C460D46FB
:10C5800028461146424A15F025FE2768414B3B409C
:10C59000062B05D0BA070AD13A683F4B9A4206D11A
:10C5A00039463E4844F2562240F022F8074601211F
:10C5B000384619F02BFC067C16F0010602D03848EC
:10C5C00033F0D2FC012D2BD96068062201A919F0A5
:10C5D000CBFBDDE9015633495C2041F004FAEB075F
:10C5E00004461FD50135013EB6F5305F1CD905F56F
:10C5F00090536563A6F5105605F51055A363656263
:10C60000A6620023C4E90B334BF06CFA20610028CA
:10C6100035D120463BF0F6F8234924484AF0DCFDAA
:10C620003546D8E7002DDFD14FF40068C4F82880E4
:10C6300040463FF034FC606228B920463BF0E2F807
:10C64000404633F01FFCB6F5105F04D3656305F573
:10C650009055A563D5E74FF490503FF020FC606300
:10C6600028B920463BF0CEF84FF49050E9E74FF45C
:10C6700090503FF014FCA0630028C2D1F1E720469F
:10C68000394604F0F9FA204604B0BDE8F08100BF55
:10C69000040002000F0080FF64E30700D0050800DB
:10C6A00060EE0700A05B0800BDF80700E8E20700A5
:10C6B00010B50446407B3AF037FAA3689FED107A34
:10C6C0005A0800EE102A94F8442004EB820423F068
:10C6D0000103626B13449A4209D1F1EEC77ABDE8B7
:10C6E0001040B8EEC00A87EE800A1CF073BC32F925
:10C6F000021B07EE901AF8EEE77AA7EEA77AEAE7B0
:10C700000000000038B504460D46407B3AF00CFAB4
:10C7100044F25622294604483FF06AFF014620466B
:10C7200004F0AAFA0E2038BDD005080038B50D4631
:10C730000446407B3AF0F8F90121284619F066FBDF
:10C74000037CDB0702D5044833F00EFC2046294663
:10C7500004F092FA0E2038BD60EE0700F8B50C46E2
:10C760000546084617461EF069FE667B30463AF0DD
:10C77000DBF962686B689A4204D040F26B410D4865
:10C7800033F00EFC6B7B0FB1022B04D0B34202D00E
:10C7900040F28221F3E7227B2B7B9A4202D040F2C7
:10C7A0006521ECE7A27BAB7B9A4202D040F28D413F
:10C7B000E5E7F8BD82F40700064A00231370064A35
:10C7C0001370064B01221A71054B1B780BB10BF04D
:10C7D00037BD7047CA770020C8770020B46F0020AB
:10C7E000C977002010B5044604F070FEE3681BB959
:10C7F0000A4A1168A14203D1BDE8104004F07CBE92
:10C80000A360074B1968E160196809B119688C6069
:10C81000116801B914601C60EEE700BF6061002080
:10C820006861002008B504F051FE044A1368013B1A
:10C830001360BDE8084004F05FBE00BF54610020F3
:10C8400008B504F043FE044A136801331360BDE8E1
:10C85000084004F051BE00BF546100202DE9F041B2
:10C86000154E01F08DFF29F0A9FC33680BB3134D71
:10C8700004F02CFE2C681CB1BDE8F04104F03CBE75
:10C880000F4A01232B603368346014601BB92B6896
:10C89000013B2B60F0E7D3E900689F68C3E90244DD
:10C8A00004F02AFE0EB14046B04704F00FFE3B46AE
:10C8B000ECE7BDE8F08100BF60610020546100201A
:10C8C0006861002008B51BF091FBC18803489729D7
:10C8D00014BF9722422233F04FFB00BFE7F007005E
:10C8E00010B5064A002352F83340844202EBC301DC
:10C8F00001D90133F7E7486810BD00BFC819090026
:10C90000F0B595B0054601A80E4617461C4646F000
:10C910003FFD10B1002015B0F0BD3A463146284623
:10C9200015F01EFF25F0FCFA830703D10268034BC4
:10C930009A42EFD020600120EDE700BF3CE3070002
:10C94000014A04232AF0B0B88C2A0900F0B587B058
:10C95000084611461A4602AB0193254B0093042367
:10C960003FF00FFD2349182041F03DF8DDE9042395
:10C970000361214B9A428CBF0123B3FBF2F3C360E6
:10C980001E4BD3F8A431DDE9027604465BB30FF009
:10C99000A1F980F00105EDB204F115030093002226
:10C9A0002B4640F27341384609F050FF04F116035C
:10C9B00060600022009340F274412B46304609F03B
:10C9C00045FF01221146A060606809F0C3FF012203
:10C9D000A068114609F0BEFF204648F09CFC20B933
:10C9E000052033F08DFA0125D6E7204607B0F0BDCB
:10C9F000F8210900845B080020A10700946B002047
:10CA0000F0B50C4687B054F8045B06462846174636
:10CA10003AF023FC28463AF02DFC02AB0193094B77
:10CA200000933A462146701E042315F00BFC059B2B
:10CA300000932846DDE90323029947F046FC0E20C7
:10CA400007B0F0BDD8210900F0B50C4687B054F806
:10CA5000045B0646284617463AF0FFFB28463AF0A4
:10CA600009FC02AB01930A4B00933A462146701E23
:10CA7000042315F0E7FB01230193059B009328464F
:10CA8000DDE9032302994AF0BEFF0E2007B0F0BD96
:10CA9000B8210900F0B50C468BB054F8045B06468B
:10CAA000284617463AF0D9FB28463AF0E3FB03AB99
:10CAB00001930E4B00933A462146701E072315F052
:10CAC000C1FB00230193079B0093DDE90312069B42
:10CAD00028464AF098FF099B00932846089B059A30
:10CAE000039947F0F2FB0E200BB0F0BD8021090046
:10CAF000F0B50D4687B055F8044B0646204617465C
:10CB00003AF0ABFB20463AF0BBFB02AB0193204B63
:10CB100000933A462946701E042315F093FB40F219
:10CB200002430122002103983FF056FC40F2F63305
:10CB3000012200210646C5B204983FF04DFC4FF497
:10CB4000197309220821074605983FF045FC029910
:10CB5000104AB2FBF1F301FB132202B1013323614E
:10CB6000237DC3F38002AA420AD066F382032375B1
:10CB70006B1E594260684FF00002594109F0EAFE0D
:10CB8000237D0E2067F3C303237507B0F0BD00BFFC
:10CB90004821090020A107002DE9F04186B0084690
:10CBA00011461A4603AB01932D4B009303233FF02C
:10CBB000E8FB2C49182040F00FFF2B4B059ED3F8C3
:10CBC000A431DDE903870446002B47D00FF082F83B
:10CBD00080F00105EDB204F11503009300222B460D
:10CBE00040F28B21404609F031FE217D6060002239
:10CBF000C1F3800109F0AEFE04F116030093012297
:10CC00002B464FF46F71384609F020FE227DA0605C
:10CC1000B0F10E0318BF012363F34102930722759D
:10CC200003D50022114609F095FE04F11703009385
:10CC300001222B4640F2AF31304609F007FE0523B2
:10CC40002361237DE06023F00D030E2818BF43F01D
:10CC500001032046237506B0BDE8F0810125BAE73F
:10CC600068210900685B0800946B00202DE9F04FF3
:10CC70000D468DB055F8044B0646204617463AF04F
:10CC8000ECFA20463AF0FCFA08AB01934A4B0093C9
:10CC900029460423701E3A4615F0D4FA062205A947
:10CCA000089819F061F89DF81C100022402015F03A
:10CCB000F5FB099B04930546069B0A99B3FBF0F329
:10CCC00003AA04A8039346F07BFB049E039B6E43D8
:10CCD0005D4304960395002D4BD0237DDF0704D4DC
:10CCE000364840F2AF3133F05BF99807DDF814A015
:10CCF000DDF82C90276940D4554406EB0A083544EA
:10CD00005FFA89F64FF0080B4FF0000A237D990770
:10CD100003D5A068F1093CF0CFFB217D0A0735D48B
:10CD2000384625F045FA217D606881F00401C1F3A1
:10CD300080013CF0C1FB0DF10B01E0683CF0A3FB6E
:10CD40009DF80B30217D43EA4A0A0B072BD4384665
:10CD500025F02EFA217D6068C1F380013CF0ACFB28
:10CD60007600BBF1010BF6B2D0D108F801AB454516
:10CD7000C6D10E200DB0BDE8F08FA06800213CF0B8
:10CD80009BFB0028B8D1052033F0BAF8C1F380012D
:10CD900081F00101606801F001013CF08DFB384633
:10CDA00025F006FAC7E76068C1F380013CF084FB18
:10CDB000384625F0FDF9D3E76423090093F6070010
:10CDC0002DE9F04F0D468BB055F8044B0646204632
:10CDD00017463AF042FA20463AF052FA07AB01936E
:10CDE000444B0093294603233A46701E15F02AFA55
:10CDF000052204A9079818F0B7FF9DF81810002223
:10CE0000402015F04BFB089B03930546059B0999B1
:10CE1000B3FBF0F302AA03A8029346F0D1FA039BF6
:10CE2000029A6B43554303930295002D5AD0227DFD
:10CE3000920704D430484FF46F7133F0B1F8049A7C
:10CE4000D4F8109002EB0308002798F800604FBB5D
:10CE5000A068F1093CF030FB002847D0BA46217D9C
:10CE60000B0708F1010B24D4484625F0A1F9217DD8
:10CE7000606881F00401C1F380013CF01DFB48466D
:10CE800025F096F9217D6068C1F380013CF014FB28
:10CE90000AF1010ABAF1080F21D07600F6B203E0D8
:10CEA000D846D2E74FF0000AA068F1093CF004FB35
:10CEB000D5E7C1F3800181F0010101F00101606853
:10CEC0003CF0FAFA484625F073F9217D6068C1F319
:10CED00080013CF0F1FA484625F06AF9D8E70137BD
:10CEE000BD42DDD10E200BB0BDE8F08F052033F040
:10CEF00007F800BF8423090093F607002DE9F04FDF
:10CF00000D4697B055F8044B0646204617463AF0B2
:10CF1000A4F920463AF0B4F910AB0193614B0093A9
:10CF200029460623701E3A4615F08CF905220DA9F4
:10CF3000109818F019FF9DF83C100022402015F0C1
:10CF4000ADFA129B1399099305460E9BB3FBF0F3C0
:10CF500008AA09A8089346F033FA06220AA91198EC
:10CF600018F002FF9DF830100022402015F096FACC
:10CF7000149B1599079306460B9BB3FBF0F306AA87
:10CF800007A8069346F01CFA089A099B06996B437A
:10CF90005543079A099372434E43B5420895079249
:10CFA000069602D0404832F0F3FF002D76D00D995E
:10CFB000C8180390207D860706D4CE1826B14FF4FA
:10CFC0006F713A4832F0ECFF0A9EC00706EB020A86
:10CFD00005D4BAF1000F02D040F2AF31F1E7CE5CD8
:10CFE000A068D4F810B0F1093CF066FA00283BD1F3
:10CFF000052032F085FF7600F6B2A068F1093CF01A
:10D000005BFA217D0A0733D4584625F0D1F8217DFB
:10D01000606881F00401C1F380013CF04DFA0DF12C
:10D020001701E0683CF02FFA9DF81730217D43EAA4
:10D0300049090B0729D4584625F0BAF8217D6068C4
:10D04000C1F380013CF038FA08F10108B8F1080F8B
:10D05000D1D10AF807900137BD421FD0039B4FF092
:10D060000008DE5DC146C8E70027B846B946C8E7F4
:10D07000C1F3800181F00101606801F001013CF021
:10D080001BFA584625F094F8C9E76068C1F380019F
:10D090003CF012FA584625F08BF8D5E70E2017B071
:10D0A000BDE8F08F3423090072F1070093F6070002
:10D0B0002DE9F04F0D4687B00021924622F024FC66
:10D0C00004460021284622F01FFC2379662B02D05B
:10D0D0000379662B02D1C84832F05AFF002303902F
:10D0E00008208DF817303EF0BCFE074608203EF0C1
:10D0F000B8FE064608203EF0B4FE0399CDE9006074
:10D1000005463B460DF11702204645F09BFE03996C
:10D1100050B938460EF022FC30460EF01FFC28466F
:10D120000EF01CFCB548D7E70AF1FF3A9DF817004E
:10D13000D4F81C90D1F81C802279BAF1030F05D8DD
:10D14000DFE81AF0E901BD0398053B08AA46B3469B
:10D150002379D4F81C90D1F81C80422B40F0C18078
:10D160000A79422A3DD1394646F019F8C269044687
:10D170000020134698F800C099F8001001EA0C014D
:10D1800003F8011BDAF80410D4F810C0DBF804E04F
:10D1900003918844991A8C45F144EBD8DBF80010D0
:10D1A000DAF800200CFB1E11894403990CFB1122B4
:10D1B0009044E2680130904211D338460EF0CEFB25
:10D1C00030460EF0CBFB28460EF0C8FB204607B0D9
:10D1D000BDE8F08F5A461C46D3469246B8E71A4639
:10D1E000C7E7622A28D13946682245F0D8FFC169CD
:10D1F00004460023002298F900C099F8000000EAD4
:10D200000C0021F8020B2069DBF804E0DAF804C016
:10D2100001328242F144E044EDD3DBF8002000FB10
:10D220001E229144DAF8002000FB1C229044E268A0
:10D2300001339342DED3C0E7482A27D1394645F06F
:10D24000AEFFC169044600230022B8F800C099F877
:10D25000000000EA0C0021F8020B2069DBF804E072
:10D26000DAF804C001328242F144E044EDD3DBF845
:10D27000002000FB1E229144DAF8002000FB1C2253
:10D280009044E26801339342DED396E7682A41F086
:10D290003782394645F083FFC169044600230022E6
:10D2A000B8F800C099F8000000EA0C0021F8020B61
:10D2B0002069DBF804E0DAF804C001328242F1446C
:10D2C000E044EDD3DBF8002000FB1E229144DAF8A5
:10D2D000002000FB1C229044E26801339342DED31D
:10D2E0006BE7622B40F08C800A79622A2CD1394698
:10D2F00045F055FFC26904460020134698F800C067
:10D3000099F8001001EA0C0103F8011BDAF8041087
:10D31000D4F810C0DBF804E003918844991A614501
:10D32000F144EBD3DBF80010DAF800200CFB1E11FF
:10D33000894403990CFB11229044E2680130904229
:10D34000BFF43BAF1A46D8E7482A27D1394645F003
:10D3500026FFC169044600230022B8F800C099F9ED
:10D36000000000EA0C0021F8020B2069DBF804E061
:10D37000DAF804C001328242F144E044EDD3DBF834
:10D38000002000FB1E229144DAF8002000FB1C2242
:10D390009044E26801339342DED30EE7682A0B46DD
:10D3A00021467FF417AF394645F0F9FEC1690446BE
:10D3B00000230022B8F800C099F9000000EA0C0030
:10D3C00021F8020B2069DBF804E0DAF804C001322E
:10D3D0008242F144E044EDD3DBF8002000FB1E2242
:10D3E0009144DAF8002000FB1C229044E2680133EB
:10D3F0009342DED3E1E600BFBEE90700F8E807008C
:10D40000482B57D10A79482A27D1394645F0C7FE1B
:10D41000C169044600230022B8F800C0B9F8000032
:10D4200000EA0C0021F8020B2069DBF804E0DAF8CE
:10D4300004C001328242F144E044EDD3DBF8002025
:10D4400000FB1E229144DAF8002000FB1C229044CD
:10D45000E26801339342DED3AFE6682A0B462146E9
:10D460007FF4B8AE394645F09AFEC1690446002300
:10D470000022B8F800C0B9F8000000EA0C0021F85A
:10D48000020B2069DBF804E0DAF804C001328242C2
:10D49000F144E044EDD3DBF8002000FB1E22914470
:10D4A000DAF8002000FB1C229044E268013393422A
:10D4B000DED382E6682B41F023810A79682A0B4685
:10D4C00021467FF487AE394645F069FEC1690446BE
:10D4D00000230022B8F800C0B9F8000000EA0C00F0
:10D4E00021F8020B2069DBF804E0DAF804C001320D
:10D4F0008242F144E044EDD3DBF8002000FB1E2221
:10D500009144DAF8002000FB1C229044E2680133C9
:10D510009342DED351E6AA46B3462379D4F81C9051
:10D52000D1F81C80422B40F0B5800A79422A31D1D3
:10D53000394645F034FEC26904460020134698F887
:10D5400000C099F8001041EA0C0103F8011BDAF859
:10D550000410D4F810C0DBF804E003918844991A51
:10D560006145F144EBD3DBF80010DAF800200CFB46
:10D570001E11894403990CFB11229044E26801308A
:10D580009042BFF41AAE1A46D8E75A461C46D34614
:10D590009246C2E7622A28D13946682245F0FFFD4B
:10D5A000C16904460023002298F900C099F80000E0
:10D5B00040EA0C0021F8020B2069DBF804E0DAF8FD
:10D5C00004C001328242F144E044EDD3DBF8002094
:10D5D00000FB1E229144DAF8002000FB1C2290443C
:10D5E000E26801339342DED3E7E5482A27D1394682
:10D5F00045F0D5FDC169044600230022B8F800C0FB
:10D6000099F8000040EA0C0021F8020B2069DBF8D1
:10D6100004E0DAF804C001328242F144E044EDD380
:10D62000DBF8002000FB1E229144DAF8002000FB0A
:10D630001C229044E26801339342DED3BDE5682AA0
:10D6400041F05E80394645F0AAFDC16904460023D9
:10D650000022B8F800C099F8000040EA0C0021F858
:10D66000020B2069DBF804E0DAF804C001328242E0
:10D67000F144E044EDD3DBF8002000FB1E2291448E
:10D68000DAF8002000FB1C229044E2680133934248
:10D69000DED392E5622B40F087800A79622A2CD192
:10D6A000394645F07CFDC26904460020134698F8CF
:10D6B00000C099F8001041EA0C0103F8011BDAF8E8
:10D6C0000410D4F810C0DBF804E003918844991AE0
:10D6D0006145F144EBD3DBF80010DAF800200CFBD5
:10D6E0001E11894403990CFB11229044E268013019
:10D6F0009042BFF462AD1A46D8E7482A27D139468E
:10D7000045F04DFDC169044600230022B8F800C071
:10D7100099F9000040EA0C0021F8020B2069DBF8BF
:10D7200004E0DAF804C001328242F144E044EDD36F
:10D73000DBF8002000FB1E229144DAF8002000FBF9
:10D740001C229044E26801339342DED335E5682A17
:10D750000B4621467FF419AF394645F020FDC169DB
:10D76000044600230022B8F800C099F9000040EAFE
:10D770000C0021F8020B2069DBF804E0DAF804C0A1
:10D7800001328242F144E044EDD3DBF8002000FB9B
:10D790001E229144DAF8002000FB1C229044E2682B
:10D7A00001339342DED308E5482B57D10A79482A42
:10D7B00027D1394645F0F3FCC16904460023002215
:10D7C000B8F800C0B9F8000040EA0C0021F8020BDC
:10D7D0002069DBF804E0DAF804C001328242F14447
:10D7E000E044EDD3DBF8002000FB1E229144DAF880
:10D7F000002000FB1C229044E26801339342DED3F8
:10D80000DBE4682A0B4621467FF4BFAE394645F07B
:10D81000C6FCC169044600230022B8F800C0B9F86C
:10D82000000040EA0C0021F8020B2069DBF804E05C
:10D83000DAF804C001328242F144E044EDD3DBF86F
:10D84000002000FB1E229144DAF8002000FB1C227D
:10D850009044E26801339342DED3AEE4682B40F09B
:10D860004F870A79682A0B4621467FF48EAE3946E7
:10D8700045F095FCC169044600230022B8F800C0B9
:10D88000B9F8000040EA0C0021F8020B2069DBF82F
:10D8900004E0DAF804C001328242F144E044EDD3FE
:10D8A000DBF8002000FB1E229144DAF8002000FB88
:10D8B0001C229044E26801339342DED37DE4AA4601
:10D8C000B3462379D4F81C90D1F81C80422B40F049
:10D8D000B7800A79422A31D1394645F060FCC269E5
:10D8E00004460020134698F800C099F8001081EA19
:10D8F0000C0103F8011BDAF80410D4F810C0DBF8AF
:10D9000004E003918844991A6145F144EBD3DBF8B4
:10D910000010DAF800200CFB1E11894403990CFB5F
:10D9200011229044E26801309042BFF446AC1A469E
:10D93000D8E75A461C46D3469246C2E7622A28D107
:10D940003946682245F02BFCC169044600230022B9
:10D9500098F900C099F8000080EA0C0021F8020B49
:10D960002069DBF804E0DAF804C001328242F144B5
:10D97000E044EDD3DBF8002000FB1E229144DAF8EE
:10D98000002000FB1C229044E26801339342DED366
:10D9900013E4482A28D1394645F001FCC169044600
:10D9A00000230022B8F800C099F8000080EA0C00BB
:10D9B00021F8020B2069DBF804E0DAF804C0013238
:10D9C0008242F144E044EDD3DBF8002000FB1E224C
:10D9D0009144DAF8002000FB1C229044E2680133F5
:10D9E0009342DED3FFF7E9BB682A40F089863946C7
:10D9F00045F0D5FBC169044600230022B8F800C0F9
:10DA000099F8000080EA0C0021F8020B2069DBF88D
:10DA100004E0DAF804C001328242F144E044EDD37C
:10DA2000DBF8002000FB1E229144DAF8002000FB06
:10DA30001C229044E26801339342DED3FFF7BDBB62
:10DA4000622B40F089800A79622A2CD1394645F050
:10DA5000A6FBC26904460020134698F800C099F856
:10DA6000001081EA0C0103F8011BDAF80410D4F865
:10DA700010C0DBF804E003918844991A6145F14431
:10DA8000EBD3DBF80010DAF800200CFB1E11894400
:10DA900003990CFB11229044E26801309042BFF4DC
:10DAA0008CAB1A46D8E7482A28D1394645F077FB8F
:10DAB000C169044600230022B8F800C099F90000AB
:10DAC00080EA0C0021F8020B2069DBF804E0DAF8A8
:10DAD00004C001328242F144E044EDD3DBF800207F
:10DAE00000FB1E229144DAF8002000FB1C22904427
:10DAF000E26801339342DED3FFF75FBB682A0B462F
:10DB000021467FF416AF394645F049FBC16904460A
:10DB100000230022B8F800C099F9000080EA0C0048
:10DB200021F8020B2069DBF804E0DAF804C00132C6
:10DB30008242F144E044EDD3DBF8002000FB1E22DA
:10DB40009144DAF8002000FB1C229044E268013383
:10DB50009342DED3FFF731BB482B59D10A79482ACB
:10DB600028D1394645F01BFBC16904460023002239
:10DB7000B8F800C0B9F8000080EA0C0021F8020BE8
:10DB80002069DBF804E0DAF804C001328242F14493
:10DB9000E044EDD3DBF8002000FB1E229144DAF8CC
:10DBA000002000FB1C229044E26801339342DED344
:10DBB000FFF703BB682A0B4621467FF4BAAE39460D
:10DBC00045F0EDFAC169044600230022B8F800C010
:10DBD000B9F8000080EA0C0021F8020B2069DBF89C
:10DBE00004E0DAF804C001328242F144E044EDD3AB
:10DBF000DBF8002000FB1E229144DAF8002000FB35
:10DC00001C229044E26801339342DED3FFF7D5BA79
:10DC1000682B40F075850A79682A0B4621467FF407
:10DC200088AE394645F0BBFAC1690446002300229C
:10DC3000B8F800C0B9F8000080EA0C0021F8020B27
:10DC40002069DBF804E0DAF804C001328242F144D2
:10DC5000E044EDD3DBF8002000FB1E229144DAF80B
:10DC6000002000FB1C229044E26801339342DED383
:10DC7000FFF7A3BA422A40F0A8800B79422B28D1A3
:10DC8000394645F08CFAC26904460020134698F8DC
:10DC900000C099F8001001FA0CF103F8011BD4F848
:10DCA00010C0D6F804A0D5F804E0991A6145D14413
:10DCB000F044ECD32A6831680CFB1E229044E268E1
:10DCC00001300CFB1A1190428944BFF476AA1A461F
:10DCD000DCE7622B27D16822394645F060FA04461A
:10DCE000C0690023002298F900C099F8001001FAD9
:10DCF0000CF120F8021B2169D6F804E0D5F804C025
:10DD000001328A42F144E044EDD3326801FB1E2225
:10DD100091442A6801FB1C229044E268013393423B
:10DD2000E0D3FFF74ABA482B27D11A46394645F0C7
:10DD300036FA0446C06900230022B8F800C099F8FA
:10DD4000001001FA0CF120F8021B2169D6F804E05A
:10DD5000D5F804C001328A42F144E044EDD3326880
:10DD600001FB1E2291442A6801FB1C229044E268B8
:10DD700001339342E0D3FFF720BA6822394645F0D9
:10DD80000EFA0446C06900230022B8F900C099F8D1
:10DD9000001001FA0CF120F8021B2169D6F804E00A
:10DDA000D5F804C001328A42F144E044EDD3326830
:10DDB00001FB1E2291442A6801FB1C229044E26868
:10DDC00001339342E0D3FFF7F8B9622A40F0A8800C
:10DDD0000B79422B27D16822394645F0E0F90446F9
:10DDE000C0690023002298F800C099F9001001FAD8
:10DDF0000CF120F8021B2169D6F804E0D5F804C024
:10DE000001328A42F144E044EDD3326801FB1E2224
:10DE100091442A6801FB1C229044E268013393423A
:10DE2000E0D3FFF7CAB9622B28D1394645F0B7F9DC
:10DE3000C26904460020134698F900C099F9001001
:10DE400001FA0CF103F8011BD4F810C0D6F804A0B5
:10DE5000D5F804E0991A6145D144F044ECD32A681E
:10DE600031680CFB1E229044E26801300CFB1A1151
:10DE700090428944BFF4A1A91A46DCE7482B27D178
:10DE80001A46394645F08BF90446C0690023002242
:10DE9000B8F800C099F9001001FA0CF120F8021B43
:10DEA0002169D6F804E0D5F804C001328A42F14471
:10DEB000E044EDD3326801FB1E2291442A6801FB45
:10DEC0001C229044E26801339342E0D3FFF775B916
:10DED0006822394645F063F90446C06900230022F0
:10DEE000B8F900C099F9001001FA0CF120F8021BF2
:10DEF0002169D6F804E0D5F804C001328A42F14421
:10DF0000E044EDD3326801FB1E2291442A6801FBF4
:10DF10001C229044E26801339342E0D3FFF74DB9ED
:10DF2000482A40F0A7800B79422B26D1394645F08C
:10DF300036F90446C0690023002298F800C0B9F8F9
:10DF4000001001FA0CF120F8021B2169D6F804E058
:10DF5000D5F804C001328A42F144E044EDD332687E
:10DF600001FB1E2291442A6801FB1C229044E268B6
:10DF700001339342E0D3FFF720B9622B29D11A462F
:10DF8000394645F00CF9C26904460020134698F959
:10DF900000C099F9001001FA0CF103F8011BD4F844
:10DFA00010C0D6F804A0D5F804E0991A6145D14410
:10DFB000F044ECD32A6831680CFB1E229044E268DE
:10DFC00001300CFB1A1190428944BFF4F6A81A469E
:10DFD000DCE7482B26D1394645F0E1F80446C06914
:10DFE00000230022B8F800C0B9F8001001FA0CF1C3
:10DFF00020F8021B2169D6F804E0D5F804C00132EC
:10E000008A42F144E044EDD3326801FB1E22914480
:10E010002A6801FB1C229044E26801339342E0D35A
:10E02000FFF7CBB86822394645F0B9F80446C06915
:10E0300000230022B8F900C0B9F8001001FA0CF171
:10E0400020F8021B2169D6F804E0D5F804C001329B
:10E050008A42F144E044EDD3326801FB1E22914430
:10E060002A6801FB1C229044E26801339342E0D30A
:10E07000FFF7A3B8682A40F043830B79422B394657
:10E0800025D145F08CF80446C0690023002298F899
:10E0900000C0B9F9001001FA0CF120F8021B216947
:10E0A000D6F804E0D5F804C001328A42F144E044D5
:10E0B000EDD3326801FB1E2291442A6801FB1C2229
:10E0C0009044E26801339342E0D3FFF776B8622BC5
:10E0D00025D145F064F80446C0690023002298F970
:10E0E00000C0B9F9001001FA0CF120F8021B2169F7
:10E0F000D6F804E0D5F804C001328A42F144E04485
:10E10000EDD3326801FB1E2291442A6801FB1C22D8
:10E110009044E26801339342E0D3FFF74EB8482BB6
:10E1200025D145F03CF80446C06900230022B8F927
:10E1300000C0B9F8001001FA0CF120F8021B2169A7
:10E14000D6F804E0D5F804C001328A42F144E04434
:10E15000EDD3326801FB1E2291442A6801FB1C2288
:10E160009044E26801339342E0D3FFF726B845F0CC
:10E1700016F80446C06900230022B8F900C0B9F9B6
:10E18000001001FA0CF120F8021B2169D6F804E016
:10E19000D5F804C001328A42F144E044EDD332683C
:10E1A00001FB1E2291442A6801FB1C229044E26874
:10E1B00001339342E0D3FFF700B8422A40F0A88031
:10E1C0000B79422B28D1394644F0E9FFC269044655
:10E1D0000020134698F800C099F8001041FA0CF19D
:10E1E00003F8011BD4F810C0D6F804A0D5F804E059
:10E1F000991A8C45D144F044ECD82A6831680CFB5C
:10E200001E229044E26801300CFB1A1190428944AE
:10E21000BEF4D3AF1A46DCE7622B27D16822394619
:10E2200044F0BDFF0446C0690023002298F900C0F5
:10E2300099F8001041FA0CF120F8021B2169D6F878
:10E2400004E0D5F804C001328A42F144E044EDD341
:10E25000326801FB1E2291442A6801FB1C22904473
:10E26000E26801339342E0D3FEF7A7BF482B27D1E2
:10E270001A46394644F093FF0446C0690023002241
:10E28000B8F800C099F8001041FA0CF120F8021B10
:10E290002169D6F804E0D5F804C001328A42F1447D
:10E2A000E044EDD3326801FB1E2291442A6801FB51
:10E2B0001C229044E26801339342E0D3FEF77DBF15
:10E2C0006822394644F06BFF0446C06900230022EF
:10E2D000B8F900C099F8001041FA0CF120F8021BBF
:10E2E0002169D6F804E0D5F804C001328A42F1442D
:10E2F000E044EDD3326801FB1E2291442A6801FB01
:10E300001C229044E26801339342E0D3FEF755BFEC
:10E31000622A40F0A8800B79422B27D16822394627
:10E3200044F03DFF0446C0690023002298F800C075
:10E3300099F9001041FA0CF120F8021B2169D6F876
:10E3400004E0D5F804C001328A42F144E044EDD340
:10E35000326801FB1E2291442A6801FB1C22904472
:10E36000E26801339342E0D3FEF727BF622B28D146
:10E37000394644F014FFC26904460020134698F958
:10E3800000C099F9001041FA0CF103F8011BD4F810
:10E3900010C0D6F804A0D5F804E0991A8C45D144F1
:10E3A000F044ECD82A6831680CFB1E229044E268E5
:10E3B00001300CFB1A1190428944BEF4FEAE1A469D
:10E3C000DCE7482B27D11A46394644F0E8FE0446DC
:10E3D000C06900230022B8F800C099F9001041FA82
:10E3E0000CF120F8021B2169D6F804E0D5F804C02E
:10E3F00001328A42F144E044EDD3326801FB1E222F
:10E4000091442A6801FB1C229044E2680133934244
:10E41000E0D3FEF7D2BE6822394644F0C0FE04467F
:10E42000C06900230022B8F900C099F9001041FA30
:10E430000CF120F8021B2169D6F804E0D5F804C0DD
:10E4400001328A42F144E044EDD3326801FB1E22DE
:10E4500091442A6801FB1C229044E26801339342F4
:10E46000E0D3FEF7AABE482A40F0A7800B79422BE2
:10E4700026D1394644F093FE0446C06900230022A9
:10E4800098F800C0B9F8001041FA0CF120F8021B0E
:10E490002169D6F804E0D5F804C001328A42F1447B
:10E4A000E044EDD3326801FB1E2291442A6801FB4F
:10E4B0001C229044E26801339342E0D3FEF77DBE14
:10E4C000622B29D11A46394644F069FEC2690446D6
:10E4D0000020134698F900C099F9001041FA0CF198
:10E4E00003F8011BD4F810C0D6F804A0D5F804E056
:10E4F000991A8C45D144F044ECD82A6831680CFB59
:10E500001E229044E26801300CFB1A1190428944AB
:10E51000BEF453AE1A46DCE7482B26D1394644F008
:10E520003EFE0446C06900230022B8F800C0B9F8D6
:10E53000001041FA0CF120F8021B2169D6F804E022
:10E54000D5F804C001328A42F144E044EDD3326888
:10E5500001FB1E2291442A6801FB1C229044E268C0
:10E5600001339342E0D3FEF728BE6822394644F0D7
:10E5700016FE0446C06900230022B8F900C0B9F8AD
:10E58000001041FA0CF120F8021B2169D6F804E0D2
:10E59000D5F804C001328A42F144E044EDD3326838
:10E5A00001FB1E2291442A6801FB1C229044E26870
:10E5B00001339342E0D3FEF700BE682A40F0A0800A
:10E5C0000B79422B394625D144F0E9FD0446C06958
:10E5D0000023002298F800C0B9F9001041FA0CF1AC
:10E5E00020F8021B2169D6F804E0D5F804C00132F6
:10E5F0008A42F144E044EDD3326801FB1E2291448B
:10E600002A6801FB1C229044E26801339342E0D364
:10E61000FEF7D3BD622B25D144F0C1FD0446C0698D
:10E620000023002298F900C0B9F9001041FA0CF15A
:10E6300020F8021B2169D6F804E0D5F804C00132A5
:10E640008A42F144E044EDD3326801FB1E2291443A
:10E650002A6801FB1C229044E26801339342E0D314
:10E66000FEF7ABBD482B25D144F099FD0446C069A7
:10E6700000230022B8F900C0B9F8001041FA0CF1EB
:10E6800020F8021B2169D6F804E0D5F804C0013255
:10E690008A42F144E044EDD3326801FB1E229144EA
:10E6A0002A6801FB1C229044E26801339342E0D3C4
:10E6B000FEF783BD44F073FD0446C06900230022C9
:10E6C000B8F900C0B9F9001041FA0CF120F8021BAA
:10E6D0002169D6F804E0D5F804C001328A42F14439
:10E6E000E044EDD3326801FB1E2291442A6801FB0D
:10E6F0001C229044E26801339342E0D3FEF75DBDF3
:10E700000024FEF75ABD00BF10B50C4C0C4B22780C
:10E7100012B19A7AFF2A0FD10A4A0B481A60F7F70A
:10E720008FF80A48F7F78CF8094B084A064904485D
:10E7300002F03EFB01232370014810BDAC7700209E
:10E74000F06900201C5A0800D05A0800C85A080076
:10E75000A0860100032A05D11E2914BF04490549DA
:10E760003FF035BB1E2914BF03490449F8E700BF39
:10E77000A67F0700AB7F07000D800700028007001F
:10E78000054A0648002303F5C0710133082B42F8FF
:10E790002100F8D1704700BF000001403546526E9D
:10E7A00030B587B00C460592D1E90123174904938F
:10E7B0005528CDE90212236809D054F8042C02A987
:10E7C00018461BF035FEA4F1080007B030BD18460E
:10E7D000009319F00BFC827B009B82B100EB82005E
:10E7E00002A90569019318460422A8470090F7F78B
:10E7F00019F8DDE9000310B120602046E5E718466E
:10E800003EF055FD0146024831F0B6FB4C070800CA
:10E8100001FB070070B586B0084611461A4602ABE8
:10E8200001930F4B009304233DF0ABFD029840F29F
:10E83000734148F085FE40F274410546039848F064
:10E840007FFE084906460C203FF0CDF8049B324677
:10E850002946044602F0ACFA204606B070BD00BF5F
:10E86000142309001C5A0800F0B50C468DB054F86A
:10E87000045B0646A87A174638F0D8FC284638F0DC
:10E8800006FD08AB01931D4B009321460423701E27
:10E890003A4613F0D7FC062205A9099817F064FA46
:10E8A0009DF81C100022402013F0F8FD069B0B99E8
:10E8B000B3FBF0F30446049304AA0A9B039303A852
:10E8C00044F07EFD049E40F27222012130463DF06C
:10E8D0008FFD039A06FB04F362430392049353B142
:10E8E000059928460A44BDF8201002F087FB10B1B4
:10E8F000404231F005FB0E200DB0F0BDF4220900BE
:10E90000F0B50C468DB054F8045B0646A87A17465D
:10E9100038F08CFC284638F0BAFC08AB01931F4B4A
:10E920000093214604233A46701E13F08BFC052207
:10E9300005A9099817F018FA9DF81C10002240202C
:10E9400013F0ACFD069B0B99B3FBF0F30446049364
:10E9500004AA0A9B039303A844F032FD039A049B84
:10E96000624363430392049353B99DF820102846F1
:10E9700002F0FEFA78B96FF01200404231F0C0FAAE
:10E98000012000900598BDF8201002442846F5F7B4
:10E9900055F80028F1D10E200DB0F0BDD4220900A9
:10E9A0002DE9F0410C4694B054F8046B0546B07A5A
:10E9B000174638F03BFC304638F069FC0DAB01934C
:10E9C000374B00933A4607232146681E13F03AFC62
:10E9D00005220AA90E9817F0C7F99DF830100022F9
:10E9E000402013F05BFD0B9B1199B3FBF0F3054640
:10E9F000069306AA109B059305A844F0E1FC0622A5
:10EA000007A90F9817F0B0F99DF8241000224020B4
:10EA100013F044FD089B1399B3FBF0F304460493F1
:10EA200004AA129B039303A844F0CAFC049F40F27B
:10EA3000E232384601213DF0DBFC059A069BDDF809
:10EA40001C806A436B43039D059265437C43069398
:10EA5000BDF834700395049493B99DF83410304692
:10EA600002F086FAC8B13CB1234608EB05023946EC
:10EA7000304602F0C3FA68B90E2014B0BDE8F08148
:10EA8000002100910A9930460A443946F4F7D6FF2E
:10EA90000028E8D0404231F033FA6FF01200F9E775
:10EAA0009C220900F0B50C4687B054F8045B06467A
:10EAB000687A174638F0B4FB284638F0E8FB02AB1A
:10EAC0000193214B00932146701E04233A4613F014
:10EAD000B9FB40F202430122002103983DF07CFC87
:10EAE00040F2F63301220021064604983DF074FC02
:10EAF0004FF4197304460922059808213DF06CFC77
:10EB0000C0B2082802D0052031F0FAF96B680298EB
:10EB10001F689B68984228BF1846FDF7E1FEF6B2D1
:10EB2000E4B2C7F824055EB1002C0CBF022103211A
:10EB30006B680022186844F06EFC0E2007B0F0BD30
:10EB4000A11B18BF0121F3E7042409002DE9F04FB0
:10EB500089B0084611461A4604AB0193774B0093DF
:10EB600004233DF00EFC40F28B21049848F0E8FCB1
:10EB70004FF46F710746059848F0EAFC40F2AF3158
:10EB80000446069848F0E4FC064618B914B96C48E7
:10EB900031F0FEF96B490C203EF025FF9DF81C304A
:10EBA000FF220546427223B1674840F2423131F0FC
:10EBB0009BF94360654B1B782BB9654BD3F8003547
:10EBC00013F00F0305D0634BD3F800351B0711D1A9
:10EBD0000123614A02EB03136B6097F80480D3F8BA
:10EBE00008A085F80980404601F0DAFC24B9FF242A
:10EBF000AC7206E05948CBE72479AC72204601F0AC
:10EC0000CFFC26B33679EE72304601F0C9FCD5F858
:10EC100004B0534F9BF80490242303FB09731B7F1C
:10EC200063B95046FDF75CFE0290B9F1000F11D1B7
:10EC3000B0F1206F02D0B0F1A05F0ED16B7AFF2B44
:10EC400002D0284602F01EFA052031F059F9FF26BD
:10EC5000EE72DCE7B9F1010FF0D1242202FB09F2D8
:10EC6000B8180021DBF800A041604046B95023F0FD
:10EC7000C9F9B8F11F0F8BBF08F01F02424639498E
:10EC80004FF0A04102F5E0720120FF2C41F8220074
:10EC90004AD0204623F0B6F9204623F08FF9FF2E04
:10ECA00045D000213046039623F078F9039A2421B9
:10ECB00001FB09F3F918039381F82160FF2681F81D
:10ECC00020600221CAF86015029BCAF80885CAF8BC
:10ECD0000C45CAF8102500221146CAF824355046C2
:10ECE00044F099FB039BCAF8C065FA5807210AB3A0
:10ECF0004022CAF80423CAF80015DBF8000040F3EC
:10ED00000730F3F73DFDDBF8000040F3073036F045
:10ED100064FB242303FB097700237B772846012328
:10ED20003B7709B0BDE8F08F4FF0FF34B7E74FF005
:10ED3000FF32BCE7CAF80015EBE700BF4424090026
:10ED4000B4F60700005A080093FC0700C9770020BA
:10ED500000F00240003002402424090053FA07006A
:10ED60006C6A00200003005010B50446407A38F069
:10ED700057FA63681B68D3F82435B3F1805F23D05A
:10ED800013D8B3F1006F21D00BD8B3F1007F1FD09F
:10ED90001248B3F1806F18BF0020400040F001001E
:10EDA00010BD0F48B3F1206FF5E7B3F1804F11D0DC
:10EDB00006D8B3F1A05F0FD00A48B3F1005FEAE7CD
:10EDC0000948B3F1004FE6E70848E6E70848E4E7FA
:10EDD0000848E2E70848E0E70848DEE790D003008B
:10EDE0000024F40080841E0000127A0040420F00CC
:10EDF00020A1070048E8010000093D000048E801A3
:10EE0000F0B50C468DB054F8045B0646687A174698
:10EE100038F006FA284638F03AFA08AB01931A4B54
:10EE20000093214604233A46701E13F00BFA062283
:10EE300005A9089816F098FF9DF81C1000224020A4
:10EE400013F02CFB099B0A9904930446069BB3FB21
:10EE5000F0F303AA04A8039344F0B2FA0499039BC5
:10EE6000614303FB04F20491039252B105989DF8AB
:10EE70002C300144284638F0D6FC10B9052031F07A
:10EE80003FF80E200DB0F0BDCC230900F0B50C46C4
:10EE90008BB054F8045B0646687A174638F0C0F920
:10EEA000284638F0F4F907AB0193194B009321463B
:10EEB00003233A46701E13F0C5F9052204A90798EA
:10EEC00016F052FF9DF818100022402013F0E6FAC9
:10EED000089B03930446059B0999B3FBF0F302AA30
:10EEE00003A8029344F06CFA039B029A63436243C3
:10EEF0000393029242B104992846194402F04AF958
:10EF000010B9052030F0FCFF0E200BB0F0BD00BFA3
:10EF1000EC230900F0B50C4693B054F8046B054699
:10EF2000707A174638F07CF9304638F0B0F90CABFF
:10EF300001932B4B009321460623681E3A4613F09B
:10EF400081F9052209A90C9816F00EFF9DF82C10E6
:10EF50000022402013F0A2FA0E9B0F99059304465D
:10EF60000A9BB3FBF0F304AA05A8049344F028FA23
:10EF7000062206A90D9816F0F7FE9DF82010002233
:10EF8000402013F08BFA109B119903930546079BC1
:10EF9000B3FBF0F302AA03A8029344F011FA049B16
:10EFA000039A0298059963436A4345436143AB4220
:10EFB000059104930392029502D00A4830F0E8FFCD
:10EFC00053B10698024409980144304602F0AAF869
:10EFD00010B9052030F094FF0E2013B0F0BD00BF33
:10EFE0009C23090072F107002DE9F04F2DED028BF3
:10EFF00099B0084611461A460CAB0193594B009341
:10F000000C233DF0BEF94FF48D610D9848F0A0FA45
:10F0100040F2E94107460C9848F09AFA40F2644100
:10F020008046149848F094FA40F2AF2106461598AD
:10F0300048F08EFA4FF48C610546169848F088FA2D
:10F040008146B8F1000F03D15FB9474830F0A0FF07
:10F05000474514D0B04512D0A84510D080450ED0F9
:10F060002FB1B7420BD0AF4209D04F4507D01EB1E8
:10F07000AE4204D04E4502D02DB14D4503D140F2F1
:10F08000FD3013F0D1F84FF41973092205210F98C0
:10F090003DF0A2F940F22E434FF6FF728246012165
:10F0A00013983DF099F9109B304A0390934227D072
:10F0B0002F4A981A434243415B00022201211198D2
:10F0C000029396233DF088F90B90129818F004FFF4
:10F0D000B0EE408A48F05CFA26499DF85CB02C20DE
:10F0E0003EF081FC5FFA8AFA0E9B0893BAF1080F92
:10F0F000044607D0204808224FF4197130F050FF21
:10F100000123DAE7B9F1000F02D1BBF1000F02D001
:10F110001A4830F0E1FEDFF870B0C0F80490DBF878
:10F120000020D2F8002512F00F0206D0DBF80820EC
:10F13000D2F8002511070ED10122BDF80C3007933B
:10F140004FEAC2090BEBC202626033B940F22E41B2
:10F15000012013F009F90A4878E7029B022B15D128
:10F16000084873E76424090063E6070048120800B2
:10F170004C120800DC5908000BFC07006EF5070074
:10F1800049FA0700F6F5070028210020B8F1000F22
:10F1900000F0F78098F804300393002F00F0F4801B
:10F1A0003B790593002D00F0F2802B790693002E19
:10F1B00000F0F08033790493029B002B18BF0E23DC
:10F1C0000293137909930999874B242202FB013298
:10F1D00092F82020002A40F0E08045EA06030898D3
:10F1E0000A930DF007F99DF82CA0039B0A90AAF151
:10F1F000020CDCF1000A4AEB0C0A5A1C4FEA0A1A0C
:10F2000005D0184622F02CFF039822F0D7FE059B6C
:10F21000581C03D00021184622F0C0FE5BF80920DC
:10F220000A9BC2F8243545EA0603002B18BF4AF0B2
:10F23000010A029B5BF8091043EA0A02D2B2C1F844
:10F240006C255BF80920039BC2F80C35059BC2F8BE
:10F25000143545EA0603BBB1069B591C03D00021B7
:10F26000184622F09BFE049B5A1C05D0184622F03B
:10F27000F7FE049822F0A2FE5BF80920049BC2F876
:10F280000835069BC2F81035099B58495BF8090000
:10F2900024225A43544B03EB020A9C50CAF8041030
:10F2A0004FF4887144F0A0F85BF809004FF49071B6
:10F2B00044F09AF85BF809004FF4927144F094F826
:10F2C0005BF809004FF4A27144F08EF85BF8090076
:10F2D0004FF4AC7144F088F85BF809204449C2F857
:10F2E00004135BF80900032140F30730F3F748FAF1
:10F2F0005BF8090040F3073036F06FF85BF809302F
:10F300000822C3F800254FF000090123CAE9069935
:10F31000CAF814908AF82030002F43D1B8F1000FBA
:10F3200056D098F8040084F8260001F039F9002E30
:10F3300052D0307984F8290001F032F9002D4FD0F5
:10F34000287984F8280001F02BF9DFED2A7A089B50
:10F35000A36028EE278A0023BCEEC88A84F82530F3
:10F36000606884ED038A04F1240123F0BDF9224B87
:10F370009842024612D1204619B0BDEC028BBDE87E
:10F38000F08F4FF0FF3307E74FF0FF3309E74FF0FF
:10F39000FF330BE74FF0FF330DE7184A18491948C0
:10F3A00047F025FF07983CF05CFD079B2061C4E90E
:10F3B0000539C4E9079928B9606823F01BFA079852
:10F3C00030F060FD387984F8270001F0E9F8A5E70E
:10F3D000FF2384F82630AAE7FF2384F82930ADE71D
:10F3E000FF2384F82830B0E7346B0020C56F070096
:10F3F0001003420000007A440000AD0B0500AD0B85
:10F40000C3EE0700CCFC070010B51DF0EDFD90F831
:10F410002730FF2B044628D0406823F0EBF994F8FE
:10F42000260029F0CFFB94F8270029F0CBFB94F8B5
:10F43000290029F0C7FB94F8280029F0C3FB616874
:10F440000B4A4FF6FF73E384238591424FF000038C
:10F45000C4E90433C4E90733A36103D008329142FD
:10F4600003D10123034A0021D1540E2010BD00BF57
:10F4700028210020BA77002010B51DF0B5FD044604
:10F4800090F8270037F0C6FE94ED030ADFED047A0A
:10F49000B8EE400ABDE8104080EE270A19F09ABD88
:10F4A00000007A4410B51DF09FFD044690F8270037
:10F4B00037F0B0FE6368186840F30730002801DBBE
:10F4C000F3F74EF90023C4E90733A36163681B68AF
:10F4D00043F30733002B08DB5909012203F01F0314
:10F4E00002FA03F3024A42F821300E2010BD00BF99
:10F4F00000E100E038B52DED028B0D461DF074FDE6
:10F50000044690F8270037F085FE284618F0E4FC02
:10F51000B0EE408A48F03CF8DFED057A28EE278A05
:10F520000E20BCEEC88A84ED038ABDEC028B38BD88
:10F5300000007A4413B50A4C40F2811240F22B13BA
:10F54000A14218BF1346019340F2C5130093054929
:10F550004FF4FE7340F275223EF048FC02B010BD3D
:10F5600048120800ABD407002DE9F04715460E46B7
:10F570001F461DF039FD044690F8270037F04AFE7B
:10F580001DB900252846BDE8F08763681B68D3F8DD
:10F590001435013304D12E484FF48D6130F000FD55
:10F5A00046F019FCDFF8B0A080468946A3699D4269
:10F5B00038D86368186840F30730002844DA2A46D0
:10F5C000314604F1100045F062F894F82530054604
:10F5D00093B1012204F1240104F1100045F07EF8FA
:10F5E00004F12401606823F07FF894F8290022F0E8
:10F5F00009FD002384F8253063681B6843F3073353
:10F60000002B08DB5909012203F01F0302FA03F360
:10F61000104A42F82130002DB4D10B233B604FF04B
:10F62000FF35AFE746F0D7FBE368B0EB080061EBCE
:10F630000901984271F10001BBD2FDF70FF9DAF828
:10F640002830002BB2D09CE7F3F78AF8B7E700BF69
:10F6500093F6070000E100E0946B002038B50C46FB
:10F660002046114606221D4612F0B4FD2CB9214653
:10F670000120BDE83840F5F79DBE2968CB0706D4C8
:10F6800011F0030308D10868144A904204D1012CF8
:10F6900014D0134830F068FC124A0A40062A04D0FD
:10F6A0003BB90A68104B9A4203D1012C01D10F4893
:10F6B000F0E7BDE838400120F5F7DCBD08463DF035
:10F6C000EAFD054601462046F5F774FE2A46044643
:10F6D0000021C0683CF0FAFC204638BDF0E4070089
:10F6E00066E507000F0080FF64E307001DE70700E1
:10F6F000012807B50B4606D10B68009340F6162388
:10F70000019302206B460146002202481AF088FD50
:10F7100003B000BD64E307000146014817F04ABC8E
:10F720000CFE0700014A17F08BBC00BF0CFE07005F
:10F73000014A17F085BC00BF64E3070008B508461E
:10F740000AB112F079FD21B11946BDE8084000F078
:10F7500005B8014808BD00BF3CFE070070B506466D
:10F76000086810F003038EB00D4603D10168454AC6
:10F7700091422AD0444C00EA0402062A04D043BB3A
:10F780000268424B9A4224D1023E012E02D94048DF
:10F7900030F0EAFB0AA91AF0FFFC0646286800EAE6
:10F7A0000403062B13D1000944F05BFC04460A9DB8
:10F7B00024B92946304644F02BFC04463149102038
:10F7C0003EF00AF9C0E9025644600EB070BD4468CC
:10F7D000EDE7012E01D02F48DAE710F0010411D037
:10F7E000441002D5002030F0D3FB21460AA847F090
:10F7F000D4FF0C98224600213CF068FC0AA819F0BE
:10F8000045FBE2E701AA40F2132117F031F9019B11
:10F810002BB101AA214620463CF0F4FED5E728682A
:10F82000324603A916F0A0FA20B1DDE9030119F070
:10F8300025FBCAE7286819F0A3FA0446B8B91020D6
:10F84000CDE90A043CF00DFB8DF834400C9028689B
:10F8500006A916F0F5FA0446204616F0B5FC002875
:10F86000CCD03DF018FDFF2806D90B48BBE741106E
:10F870000AA847F084FFEAE7C1B20AA847F0CBFE26
:10F88000EAE700BF0CFE07000F0080FF64E30700FB
:10F890001DE7070066E507004FF10700F0B585B0EA
:10F8A000054617460C4618F0A1FB69460646284651
:10F8B0001AF072FC042F054622D1A307009814D138
:10F8C0002268104B9A4210D101AA21463EF0D8FB83
:10F8D00010B90D4830F000FBDDE901123046521A34
:10F8E000294419F0D7FC05B0F0BD0146002322469B
:10F8F000304616F057FA285C400040F00100F2E76D
:10F900000020F0E74C07080013E907002DE9F14F4C
:10F910008F0705460C46164613D001F00F03022B45
:10F9200019D102F0FD06012E4FEA111104D001B0E9
:10F93000BDE8F04F05F0AEB901B0BDE8F04F04F0FE
:10F94000B7BE4968CBB22D2B00F087800BD8062BB1
:10F950000ED02C2B13D0554A2146284601B0BDE8C5
:10F96000F04F05F0A5B92E2B00F08C809D2BF2D125
:10F97000002EF0D104F10802090A284687E0022A85
:10F9800002D0A16804F0EAFEE768002FE3D017F088
:10F990000309E0D17B68DAB28E2AB8460DD1022E77
:10F9A0004FEA132805D007F1040A08F1FF3BD945B7
:10F9B00015DB08F1010857F8288098F80430312B3E
:10F9C0002BD1022E13D1686A3CF0B0FF686A562230
:10F9D0006FF0020101B0BDE8F04F39F040BF5AF8B6
:10F9E000041F284604F0BAFE09F10109DFE72846A2
:10F9F000D8F8081004F0B2FE012E686A09D1582226
:10FA0000022139F02CFF686A01B0BDE8F04F3CF0EC
:10FA1000B7BF56226FF00201DCE7322B9BD1012EDB
:10FA2000686A0AD13CF0D0FED8F80810686A090963
:10FA300001B0BDE8F04F3CF078BE022E01D13CF0A1
:10FA400079FFD8F80830686A1B0918226FF00101A5
:10FA500001B0BDE8F04F39F082BFA268002A3FF440
:10FA60007AAF002E7FF477AF5168090A022907D1D7
:10FA7000D3682BB1980703D11B79AC2B3FF46BAF44
:10FA800008327AE7002A7FF466AFA16821B901B095
:10FA9000BDE8F04F00F00CB88E0703D10B79922B24
:10FAA0000A46E1D004F10802012166E71DF10700D2
:10FAB0002DE9F04701F1FF3A0546884691464FEAA5
:10FAC0000A2700244FF0FF3617F5807F0CD1731CF6
:10FAD00005D1686A43463022514607F007FE0024EC
:10FAE00044451DD1BDE8F08759F8241071B18A074B
:10FAF0000CD10A79222A09D101360BD1686A47EA6A
:10FB000004033122514607F0F1FD26460134A7F5E2
:10FB10008077D9E72846084ABDE8F04705F0C8B81D
:10FB200059F82410A64208BF896800222846FFF72A
:10FB3000EDFE0134D4E700BF99EA070001F00F039E
:10FB4000022B2DE9F04707460C4604D1BDE8F047EB
:10FB5000090904F04BBC00295BD011F0030558D112
:10FB60000B792C2B3FD1896804F0F8FDE568002D56
:10FB70004FD015F003084CD16E68F2B28E2A2B4696
:10FB800009D1360A05F1040906F1FF3AC24518DC2D
:10FB9000013655F826301A79312A1AD19968384633
:10FBA00004F0DCFD7C6A20463CF09AFE20463CF0E6
:10FBB000BDFE20465622BDE8F0476FF0020139F045
:10FBC0004EBE59F8041F384604F0C8FD08F101087C
:10FBD000DCE7322A1DD19968786A0222BDE8F04735
:10FBE00009093CF08ABD2D2B13D18C688CB1636858
:10FBF0001B0A022B01D1E36833B9261D6368B5EBFC
:10FC0000132F0DD3BDE8F0879A07F6D11B79AC2BE3
:10FC1000F3D121463846064ABDE8F04705F048B81A
:10FC200056F8041F3846FFF789FF0135E6E700BFA5
:10FC3000C2F0070070B5137803F06003202B59D190
:10FC40002D4B90885C7884420ED093F83D488442D6
:10FC500050D103F63C0001255478203C032C49D8B0
:10FC6000DFE804F005050D3018460025F4E701290A
:10FC700003D1072104302FF017FC012070BD0129AA
:10FC800002D12FF001FCF8E70329F6D15188847FD7
:10FC9000C17001F0010282F001018C4218BF81772E
:10FCA0006AB95B68B3F5966FE7D14FF08043B32232
:10FCB000C3F81C257E22C3F8202528F059FF2DF01B
:10FCC000D9FADAE70129DCD00329D6D10B4B1B780E
:10FCD000002BD2D00A4B1B680133CED0002DCCD1E3
:10FCE0005388002BC9D0074B074A9A6603F160027C
:10FCF0009A62C2E70020C1E7542A0020E37900207D
:10FD000008210020946B0020301108002DE9F047F5
:10FD100041F27802002121483CF0D8F91F4B2048DD
:10FD200000211F464FF0FF094FF4E1380A464FF01B
:10FD3000080E4FF4806540F63C0C012603F23C446B
:10FD40001C630CFB01744FF0000A83F80B90C3F89E
:10FD500004801A725A7283F80AE083F825209D867F
:10FD600083F836206287228783F80DA003F13C0ACE
:10FD7000D862C3F818A09D839E776284228400F124
:10FD800040045C614C1C022C03F63C0300F1800033
:10FD90004FF00101D2D1BDE8F08700BF542A002006
:10FDA000542900202DE9F84F4B79022B81468A46D1
:10FDB00015D18B79022B12D14D4F97F8266096B151
:10FDC000BE7B86B197F8623863B197F84A384BB179
:10FDD0004FF0E023D3F8F03DDB0700D500BE002054
:10FDE000BDE8F88F012640F63C037343F91807F885
:10FDF00003909AF802304B709AF800400AEB020820
:10FE000054444445627805D223782344984501D36D
:10FE1000242A18D0052A0CD1204631F04DFF0028A5
:10FE2000D6D040F63C0303FB0673A2789A70237881
:10FE30001C446378042B38D163790A2B35D12346CF
:10FE40004FF0000B2AE01C46DBE743452CD29D18FF
:10FE5000A84529D36B78052BBAD1EB7803F00303BF
:10FE6000022BB5D1284631F027FF0028B0D0AB785F
:10FE7000DB091ED040F63C0303FB067383F80C90AD
:10FE8000AA789A73AA88C2F30A021A8240225A8276
:10FE900000225A841A840BF1010B2B4621795FFA58
:10FEA0008BF291421A78D0D89C18A4EB0A0080B249
:10FEB00096E740F63C0C0CFB0673AA8883F8249066
:10FEC000A97883F826107042A98800EA0C00C2F3D2
:10FED0000A022430C1F30A015A85384400225A87A5
:10FEE00019851A8746F05FFE0028D4D170E700BF5D
:10FEF000542A002000220A4B30B511461446012531
:10FF0000987F1C6000B99D77501C022883F826104A
:10FF100099734FF0010203F63C03F1D130BD00BFED
:10FF2000542A00202DE9F0476F4C984694F826306B
:10FF300099420F467AD0A27B8A421BD0A2788A428D
:10FF400000D1B9B994F862389F4272D094F84A2827
:10FF5000BA4269D094F83E28BA4201D1002F63D149
:10FF60004FF0E023D3F8F03DDB0700D500BE0020C2
:10FF7000BDE8F08700256E4226F4F86626F00306F9
:10FF800036059F424FEA16563CD140F63C0303FB30
:10FF9000054306F12409D96AA14431B106F13000C4
:10FFA0001FFA88F2204446F022FF40F63C0101FB94
:10FFB0000541C87AFF281ED00A8F4B8FB1F834E074
:10FFC00092B29BB29A42B6BFC3EB4E0AA2EB030AAF
:10FFD00092441FFA8AFAD6450AD2724540F63C018D
:10FFE0002BD3A2EB0E0301FB05419BB24B87F246DC
:10FFF000BAF1000F46D14846B9F81430B9F81630B6
:020000023000CC
:1000000046F0D1FD40F63C0303FB0545AB7BBB420C
:1000100008D10C36A01946F042FE18B94146A01985
:1000200046F07FFE0120A3E70125A4E70026354620
:10003000ABE740F63C060125A7E702EB0E0301FB08
:1000400005419BB24B87F2469E451ED940F63C01C6
:1000500001FB05419A42096B01EB030C19D8AEEB89
:100060000302AAEB0E0E73449BB292B29BB1013B0A
:100070000B44002BBFD04FF0000E013A14E0A2EB6E
:100080000E0292B29645FAD9DEE7A3EB0E039BB2BD
:10009000DAE752460021531E6344EAE78B421ED141
:1000A0000CEB02030EF1010EC645A4D093F800A09C
:1000B0008245F3D10D4B1B6898429CD140F63C031E
:1000C00003FB0543002248465A871A8746F06BFD1A
:1000D000074B084A9A6603F160029A628BE7634510
:1000E00089D0013BDEE700BF542A00200821002010
:1000F000946B00203011080010EE103AC3F3C75182
:100100007F39162982B013DC002913DB124A0A4119
:1001100013420DD0DFED117A30EE270A002B8DED62
:10012000000AA8BF9B18009923EA020300EE103AC8
:1001300002B07047DFED097A30EE270A002B8DED13
:10014000010A019A04DB5B0018BF4FF07E53EDE714
:100150004FF00043EAE700BFFFFF7F000000807B15
:10016000054B4FF0FF32072843F8202084BF1B18AF
:1001700083F85020704700BF086A002042F216231F
:10018000984273B50E4619D042F27613984215D0B4
:100190008B070FD00B4D00243046297801236A4687
:1001A00016F0B6FC009848B90134032C05F101059E
:1001B000F2D104E00A68044B9A42EBD1012002B06C
:1001C00070BD00BF2C790800E407080038B5002393
:1001D000C3714FF0FF33C36405463BF0CDFF0446C7
:1001E00040BBB5F87E224AF655239A4224D11549E0
:1001F0000B2205F180003BF014FFF8B195F8802048
:1002000002F11803DBB2012B01D9EB2A18D10E49F8
:10021000032205F1B6003BF004FF48B10B4905226B
:1002200005F1D2003BF0FDFE041E18BF012464005E
:10023000204638BD0424FBE70324F9E70124F7E74F
:100240000224F5E717D5070023D5070027D50700B7
:1002500008B501482FF076FEDAF7070008B5074B1E
:100260000340062B05D0830706D10268044B9A424F
:1002700002D104482FF078FE08BD00BF0F0080FFB8
:1002800064E3070097F2070037B501236A46044686
:100290000D4616F03DFC009B23B903482A46214633
:1002A0002FF06AFE03B030BDA5FB070037B5012370
:1002B0006A4604460D4616F02BFC009B23B9034802
:1002C0002A4621462FF058FE03B030BD99FB0700A7
:1002D000012808B504D1034840F2C7112FF060FE91
:1002E00008BD00BF42FC070008B510B901482FF057
:1002F0004FFE08BD8DF707002DE9F04104460D467D
:1003000017461E4659B1186817F070FE61688142A1
:1003100005D0C388CA88064889212FF02DFEA06821
:1003200033463A462946BDE8F04113F053BB00BFBF
:10033000AEFB07002DE9F04F2DED028B83078BB04C
:1003400004460D4609D10368754A934205D111F060
:10035000030802D10A689A4202D072482FF004FEC4
:1003600042F0DCFE18B1284642F0D8FE08B96E48CB
:10037000F4E7277938461FF04BFB019028791FF0EE
:1003800047FB0690384621F093FBD4E903630490C1
:100390003A46E079009308A9CDE9083642F0FFFE1D
:1003A000C3690393D4F81CB0EB69DDF80CA0029389
:1003B0000746D946B0454BD1662205F10C01E879D4
:1003C00042F0EDFE6622C369049005F10C01E87964
:1003D000059342F0E4FED0F81C804FF00009B145CF
:1003E00061D1009A039B7C6904FB0234059B08EBF6
:1003F000860503EB8609A6EB020B9046009B08F1ED
:10040000FF3A534500F2878004980BB0BDEC028B95
:10041000BDE8F08F48460593019B9847049B5046E2
:1004200098477A69059B9244A26901339144009AE6
:100430009342EFD1D7E90523009902FB11339A4487
:10044000D4E9053202FB1133994408F10108B1E700
:100450000023ECE707935846019B9847079BA26946
:10046000F3EC017AA0EE278A93440AF1010AD14500
:10047000F0D10298069B9847019B584630EE488A77
:100480009847C8EE007A08EB890ACAED007AD4E9E9
:10049000053202FB19339B44029AAB691A4402925B
:1004A00009F101099BE79FED218A43464FF0000ABD
:1004B000DDE7019B2046CDE9022198470399BB69FE
:1004C000F1EC017A029AE0EE278A1C440132B24232
:1004D000EFD346454FEA8B032EBFD84600234FF09B
:1004E00000084B4408F10108A3EB8809BB6935ED0E
:1004F000018A03FB18484046019B984738EE688AFA
:100500000BF1010BC8EE007AC9ED007A7C69A8EB0B
:100510000404D04672E7DFED058A49464246D6E735
:10052000CC5008002CEE070045EC0700000000004E
:10053000D0ED077ADFED0D6A427BB4EEE70AF1EE0B
:1005400010FAD8BFB0EE670AD0ED017A80ED060A46
:10055000B8EE677AC7EE267A67EE807AFCEEE77A25
:1005600017EE903A53435B008364704700007A446F
:100570000E2810B5044610D0084BD3F8A4313BB177
:100580000BF0A8FB20B12046BDE810400BF0E6B907
:100590002046BDE8104025F039BC10BD946B00200A
:1005A0004109054A00F01F000123834052F8210051
:1005B000034342F8213070476C6100202DE9F04F71
:1005C00004288BB004462CD07D4D286818B125F046
:1005D0001DFC00232B6024B37A4B9C4221D001AB3D
:1005E00002932146784B039302A8002601963DF022
:1005F000CDFA0198013025F0D9FD286088B1019B22
:100600000890CDE9063601238DF8243006AB04931B
:1006100021466E4B059304A83DF0B8FA2A68019B69
:10062000D6546B4C6B4D20680BF098F900236A4A46
:100630002360D5F8E8401360002C35D1674E33783D
:1006400023B16748047200F057FC347028F0E0FAD8
:1006500027F076F909F068FE624BD5F8F8400022E1
:100660001A70002C55D020460BF034FB002800F007
:100670008B80A7685C4B3B40062B06D017F0030627
:100680001BD13A68594B9A4204D106A9384619F051
:1006900065FD0646D5F8F830DDF81890DFF86C8176
:1006A0006BB916202FF02CFC94F82530666813B92E
:1006B00020460DF017FF3446BEE70026EAE7D8F8DB
:1006C000004046B163684B4505D121684A46304633
:1006D0003BF0A7FC10B1A3689F4251D1E368C8F872
:1006E0000030D5F8F430A34202D10023C5F8F4302D
:1006F000002320461A4640F2F7413DF0C0FED5F8EF
:10070000F840002CAFD1D5F8F8301C46DB68002B40
:10071000FBD1374FC5F8F4400026069600F0D6FE10
:100720003C680DF11808B146002C2FD1069B3B60A8
:10073000304B1E60304B1C6000F0DEFE2FF0A0FD41
:100740002E4B6B63AB8AC5F8004143F00103AB82CB
:10075000C5F8B4412A4D0AF059FF24222146294800
:100760003BF0B4FC286825F051FB2C60264D28682E
:1007700025F04CFB2C600BB0BDE8F04F28F0CCB955
:10078000E36804F10C088BE7E468BAE7D4F808A042
:10079000C4F8089020460BF09DFA834660B9606863
:1007A0000BF098FA50B9C8F80040304604F1080838
:1007B0002646E0605446B7E70020FAE75846F8E7D7
:1007C0008C6F00200C6C0020AB8D0600E1760700DA
:1007D0005C610020946B002064610020AC770020F5
:1007E000F06900209F7700200F0080FF64E307007E
:1007F00060610020686100205461002088080900C1
:10080000444D0020246D0020F46000208C6C0020FA
:1008100038B5084D084C287821F022FC20683AF0C1
:100820007FFE287821F0EEFB2068BDE838403AF0E2
:1008300077BE00BFF86100203821002008B5064AC5
:10084000034650782BB121F00BFCBDE80840FFF7C0
:10085000DFBF21F0D7FBF8E7F861002013B54FF4B4
:100860009D616A4616F0E0F800216A4608463BF0B2
:10087000C9FE084C3DF02EF808B102B010BDFBF7E0
:10088000EDFFA16A0029F8D16A4608463BF0BAFE9E
:10089000F0E700BF946B00202DE9F3470C461E469D
:1008A00090461CF095FBDDE90A57837C5B423B7068
:1008B000E307814612D414F0030A03D12268394BAE
:1008C0009A4207D020463CF0F9FF002831D0BAF117
:1008D000000F26D12268334B9A4222D1204617F0CE
:1008E00073FB031488F8003003123370287099F8F2
:1008F0001230002B4ED199F80C20042A4AD199F8D5
:100900001120002A46D098F800203178914241D138
:100910002A788A4201BF3A7088F8003033702B7011
:1009200038E0204617F0D8FAFDEEC07A17EE900AAC
:10093000D7E76A4601A9204617F064FA042203218A
:10094000019840F2922311F03DFD009B1868F3F7E7
:10095000E1FA009B88F800005868F3F7DBFA009B87
:1009600030709868F3F7D6FA019B2870032BBED934
:10097000009BDC6820463CF0A1FF70B1204617F0D8
:10098000ABFADFED097A20EE270AFCEEC07A17EE0B
:10099000900A387002B0BDE8F087204617F014FBCB
:1009A000F7E700BFF0E4070000007F4370B52DEDCE
:1009B000028B0646B0EE408A1CF00AFBDFED1F7A80
:1009C00080ED068A28EE278A4289BCEEC88A044652
:1009D00018EE103A9BB29A4209D0426805894381C9
:1009E000B3F5807F02FB05F5426A03D15AB9BDEC2D
:1009F000028B70BD3AB928463BF051FA216A606219
:100A00002A463BF022FB0023AB420AD194F828305F
:100A1000002BECD0BDEC028B3046BDE8704036F0C8
:100A200051BEA27C0AB19A0706D0D4E908126089A7
:100A3000D25C42431212CA540133E5E700008043FE
:100A4000084AD2F8083143B190F8263023F0040365
:100A500080F826300023C2F8083190F82600C0F351
:100A6000800070470050024010B50446084617F059
:100A700033FAD4ED067ADFED1A6A627BB4EEE70A48
:100A8000F1EE10FAD8BFB0EE670AD4ED017A84ED2A
:100A9000050AB8EE677AC7EE267A67EE807AFCEE32
:100AA000E77A17EE903A5343A26D5B009342636579
:100AB0000ED962651346206DD21A184400213BF00E
:100AC00005FB236B53B12046BDE8104043F086BCC4
:100AD000216C8B423CBF61650B46ECE710BD00BF4B
:100AE00000007A442DE9F04F2DED028B85B00E29E0
:100AF0000446039100F08A80084617F077FAC37B1A
:100B00003BB9C38858484FF45C7240F2CA412FF099
:100B100033FA03AB00220121544819F04FFD8046FF
:100B2000039058F8046F07466622012130463BF0D7
:100B30005FFC4FF0000AB24522D10837B100606A6D
:100B4000DFF82C913BF0AEF9B1006062A06A3BF097
:100B5000A9F9B100A062E06A3BF0A4F9C4E90B0670
:100B60004FF0000AB7EE008AB24552D1236B13B1A1
:100B7000204643F033FC05B0BDEC028BBDE8F08F9E
:100B800058F8045F284617F031FAC37B81461BB33F
:100B900000EB8303364A1B6993421DD1AB466622A4
:100BA0005BF8045F0221284611F0F0FB4FF00009CA
:100BB000A94540F2833202D10AF1010ABBE7B9F13B
:100BC000000F5BF8040F14BF11464FF4816146F02B
:100BD000CBFC09F10109EBE728463CF06FFE08B9B0
:100BE000EB0705D54FF48161284646F0BDFCE3E7ED
:100BF000B9F80630019340F2163300931D484FF4C4
:100C00005C7340F2CA4275212FF0B6F900263746D0
:100C100094E757F82AB0584617F0E8F9656AC37B9D
:100C20004FEA8A084544ABB100EB830003694B45AA
:100C300010D1DBF808003AF065FC85ED000AA36AE4
:100C4000DBF80C0098443AF05DFC88ED000A0AF1EC
:100C5000010A89E758463AF055FC85ED000AA36A77
:100C6000434483ED008AF2E7AEFB07002CDB07006C
:100C7000A1A5040053FC0700F8B504460D46FBF798
:100C8000DFFD04F14802284625644FF491610025F8
:100C900015F0EEFE01212046C4E90B5584F84550BD
:100CA00084F8465044F067FEFF2384F85430012155
:100CB00020463BF056FB012120463BF079FA4FF4E9
:100CC00090522946606B3BF001FA4FF4905229464E
:100CD000A06B3BF0FBF926693822294630683BF0CF
:100CE000F5F94FF4A472294670683BF0EFF94FF420
:100CF0008E722946B0683BF0E9F941F2102229468C
:100D0000F0683BF0E3F94FF45272294630693BF04A
:100D1000DDF94FF4D952294670693BF0D7F9B06933
:100D200042F2042229463BF0D1F9256945B3616AB4
:100D3000E36A2846194433F00BFE013020D0D5F881
:100D4000D037032B1CD195F8D427164BD5F8BC67A8
:100D5000D5F8C077062101FB0233B3F90450FBF745
:100D600061FD1023754323730123E38105FA03F327
:100D7000A360AD00002367606673E563A365F8BDFB
:100D8000E36A0133E362012120463BF011FA94F853
:100D90004530002BC9D0FBF745FD0349034846F019
:100DA0001BFA00BFCC2D09000FF80700CCFC070090
:100DB0002DE9F0470E46FF21817211790446307902
:100DC000884203D140F2FD3011F02EFA4348002151
:100DD0006160057A1DB1017E00297BD10125404962
:100DE00000EB051060608B4296F8048092F8049046
:100DF00023D83C4FBB428CBF4FF080674FF0CC777D
:100E000084F809801079A072FFF7CAFB3079364D5B
:100E1000FFF7C6FB636801221A72666896F804A0A1
:100E2000342101FB0AF16A1892F82D3043B12046B3
:100E300000F062F805202FF063F84FF0C867DFE795
:100E4000B8F11F0F936082F8303082F82F3082F8AB
:100E500032308CBF08F01F034346566003F5E07341
:100E600088BF224A2248685098BF4FF0A04240F203
:100E70000C61B9F11F0F42F823108CBF09F01F035A
:100E80004B4603F5E0738CBF184A4FF0A04240F286
:100E90000C6142F823103368C3F80885C3F80C9539
:100EA000C3F82475342303FB0AF3EB5853B13068BD
:100EB000072140F30730F1F763FC306840F3073057
:100EC00034F08BFA342303FB0A55012385F82D30C7
:100ED000BDE8F08707482FF05BF800BF4C210020E9
:100EE0007F1A06008FD00300CC6A00200003005058
:100EF000BB6F07005FFA0700F8B5837AFF2B044643
:100F000033D04668194D377934237B43EA1892F879
:100F10002D20FAB1EB5823B1306840F30730F1F7D8
:100F20000DFC304621F0C4FB342303FB075393F838
:100F300032304BB93368D3F8080521F01FF8336815
:100F4000D3F80C0521F01AF8342303FB07550023CE
:100F500085F82D30A07A27F035FE607A27F032FE32
:100F6000636800221A72FF23A372F8BDCC6A0020C6
:100F700038B543681C681A790623C4F800351E4B3F
:100F80000546342000FB0233022283F82D20002383
:100F9000C4F88815C4F84435C4F8483501232362E1
:100FA000A360D4F850311BB9D4F82431002BF8D009
:100FB0004FF4A871204642F017FA01236361D4F878
:100FC0000431002BFBD04FF48271204642F00CFA22
:100FD000D4F8243173B120464FF4927142F004FAF0
:100FE000D4F8C434C4F8C4340024686821F060FB29
:100FF000204638BD0124F8E7CC6A00202DE9F04FE7
:101000001C46436816461A791B688B46062187B032
:10101000C3F80015194B342101FB023302220746A5
:1010200083F82D204FF0010A4FF000094CB9144D00
:10103000786821F03DFB284607B0BDE8F04F2EF060
:101040009BBBB4F5806FA0464FF0000228BF4FF461
:10105000806801A93846CDE90289CDE904698DF897
:1010600004A08DF805B0F3F7C1F8054B984205468A
:10107000DED1A4EB08044644D8E700BFCC6A0020C8
:101080000000AD0BF8B54568234C2F7924237B4332
:10109000E2180646127F002A32D0E35823B12868AE
:1010A00040F30730F1F74AFB24237B43E218E3586F
:1010B0002D687BB1194BC5F80833537F53B1012319
:1010C0006B61D5F80431002BFBD0242303FB0743CD
:1010D00000225A77242303FB074393F82100FF28BB
:1010E00001D020F04BFF0023C5F800350C4B9D428A
:1010F00004BF01236B60242303FB074400232377F1
:10110000707A27F05FFDB07A27F05CFDF07A27F067
:1011100059FDFF237372F8BD6C6A0020520108006C
:1011200000F002402DE9F04F9B464368DFF85C90E9
:10113000D3F80080DFF858A085B007460D46164664
:10114000BBF1000F01D1012017E07B68DC685C4532
:1011500028BF5C46C84505D1224629464FF00050BD
:101160003AF073FF78686946CDE90054CDE902642E
:1011700021F0B6F9504503D0002005B0BDE8F08F4E
:1011800025442644ABEB040BDAE700BF00F0024035
:101190000000AD0B2DE9F04F4368DFF864A0D3F8F1
:1011A0000090DFF860B085B080460E461546D8F84E
:1011B0000430DB68AB4228BF2B46D1451F4617D110
:1011C0001A4631464FF000503AF03FFF4FF00053BF
:1011D000D8F8040000246946CDE90037CDE902447F
:1011E00021F07EF9584505D0204605B0BDE8F08FC6
:1011F0003346EDE7ED1B3E44D9D10120F5E700BFB2
:1012000000F002400000AD0B2DE9F04F83B099468D
:1012100043681B68D3F80C35013300AF80460D4698
:10122000144604D14F4840F2E9412EF0B9FE002A9D
:1012300000F08F8001F0604BBBF1005F0FD0802A7F
:101240001FD9494BD3F8A431DBB110463AF027FE41
:1012500003462946224618463AF0F7FE0546D8F8D6
:101260000430187921F0BAFA90B905F06043B3F16F
:10127000005F10D03D4AC9F800203D493D4845F087
:10128000B6FFE31D23F00703ADEB030D6B46E0E76C
:10129000FBF7E4FAE3E7D8F8046096F804A05046B8
:1012A00021F09CFA08B1344AE5E7344A242303FBD1
:1012B0000A234FF490715C619D6030687B6042F05E
:1012C00093F830684FF4AC7142F08EF87B68316867
:1012D00058699A68C1F84425C1F848053168012069
:1012E00088605B68F3B93368244AD3F82001D3F8E7
:1012F00058110843F9D099B90121D9603168D1F862
:101300005831002BFBD01E4B242101FB0A22002167
:1013100051611B4AC9F80030934203D00832ACE750
:10132000184BF1E70023C9F80030D8F804301879D9
:1013300021F054FA90B9BBF1005F0AD00A4BD3F800
:10134000A43133B128460AF0C5FC10B128460AF092
:1013500005FB20460C37BD46BDE8F08FFBF77EFA53
:10136000E3E700BF93F60700946B00200A00AD0B83
:10137000C3EE0700CCFC07000B00AD0B346B002064
:101380000000AD0B0800AD0B03791F2B86BF03F0E7
:101390001F03074A4FF0A04203F5E07352F8230001
:1013A000C0F30220063801288CBF002001207047BE
:1013B0000003005008B5436818791F2887BF0D49FE
:1013C00000F01F0202464FF0A04120F029FE012844
:1013D00002D109482EF06CFD02F5E07251F82200AE
:1013E000C0F38100012803D0C31E5842584108BDF4
:1013F0000220FCE70003005029F9070008B5436804
:101400000246187920F00CFE53681A7928B9104664
:1014100020F016FE00F0010008BD1F2A8ABF054B10
:101420004FF0A04302F01F02D3F80405D04000F0B3
:101430000100EFE7000300500379012914BF0322E4
:1014400007221F2B86BF03F01F0306494FF0A04160
:1014500003F5E073120242F0030241F8232000205A
:10146000704700BF0003005013B50E4B1B780446B5
:1014700013B9002002B010BD08236A4600211846A7
:1014800043F041FB0028F4D0204626F007FE002858
:10149000EFD0054BD4F8D4201A60044B94F8C42044
:1014A0001A70E7E7CE790020D86F0020CB770020B4
:1014B000C0B240F0007000F17E40033810289ABF9F
:1014C000014B185C0020704744250900084B1A683E
:1014D0003AB9EFF310820749003A18BF01220A70A7
:1014E00072B6BFF35F8F1A6801321A60704700BF8F
:1014F0006C6F0020AD77002008B5094B1A6812B94F
:10150000052027F049FB1A68013A1A601B682BB9BD
:10151000BFF35F8F034B1B7803B962B608BD00BFF2
:101520006C6F0020AD7700200A4B186880B1C107AE
:1015300009D4820709D4430709D410F4D81F14BF73
:1015400003200620704704207047052070470220C2
:10155000704700BF946F00202DE9F04F9E4B16019D
:1015600081468A4617460FCBADF2AC4D09AD85E8F2
:101570000F0004362A4600231468D4F8001581B9F8
:10158000D4F8600588420CDAD4F86405884208DA99
:10159000D4F86805884204DAD4F86C058842C0F2B1
:1015A000BC800133042B02F10402E5D1002425465E
:1015B000CEE003F108011AF802B089B280201BEADC
:1015C000000F48F2050E18BFE64625F813E0013378
:1015D0009BB28B424FEA5000F1D1013292B2D3005C
:1015E000BA429BB2E5D34FF4004225F813200133F1
:1015F0009BB2760825F81320B6B200231422C4F853
:101600000C35C4F80435C4F80825C4F81435C4F8FA
:101610001035C4F82055C4F82465C4F82835C4F83A
:101620002C35D9F80420127901924FF0FF32CDE920
:101630000222049201AA03F5AC71013352F8040BA3
:1016400044F82100042BF6D10125C4F800554FF4CD
:101650008871204641F0C8FEA560D4F8103133B33C
:101660004FF48871204641F0BFFE5C4B0FCB002643
:1016700005AD85E80F00C4F80065334603F5AC728C
:10168000013355F8041B44F82210042BF6D1002036
:1016900024F0F0FC043041F10001C8E900010DF232
:1016A000AC4DBDE8F08F002248F20C0C97E7FBF739
:1016B000D5F8D2E71AF802B008214FF0800CD4F820
:1016C00004E0AEEB030EBEF1460FF8D96368D5F81F
:1016D00008E51BEA0C0F4EEA060EC5F808E512D025
:1016E000D4F804E0AEEB030EBEF1280FF8D9D5F81C
:1016F0000CE501394EEA060EC5F80CE54FEA5C0C24
:10170000DDD1013255E0D4F804E0AEEB030EBEF1BA
:10171000110FF8D9EBE762B6B9E740F284439E4275
:1017200016D9DFF8D0802E4DD8F80030B3420DD254
:10173000D5F8FC0008B1C8F80010012231460AF0C3
:10174000D9FAC5F8FC0008B1C8F80060D5F8FC501B
:10175000DFF8A480002024F08DFCD8E9002390421B
:101760009941F7D30DB1002C9DD172B6D9F8043050
:101770001C4A1B791C4C1F2B88BF03F01F034FF022
:10178000010606FA03F6D2F8FC3088BF174D43F085
:101790008073C2F8FC3023684FF4307943F00103C2
:1017A00098BF4FF0A045236009FB07F9002260684D
:1017B000134691B28F423FF67DAF6268D21A462A35
:1017C000FBD963681B1A4B45A5D3094B4FF49640D0
:1017D00043F001039847E9E7407D0700507D07008B
:1017E000946B002000ED00E0001000E000030050CA
:1017F00020190900846F00204829002037B500F027
:101800003BF8124C6946C4F8B4003AF0F7FAC4F851
:10181000F400B0B9D4F8F8400CB903B030BD656835
:10182000012D0CD129460A4817F0F2FC01AB0190BA
:101830002A4640F2832120463CF03EFEEDE7E46874
:10184000EAE76B46012240F28321F5E7946B002022
:101850008C82070010B5074BD3F8B44044B1204642
:1018600044F0DAF901462046BDE8104017F0D0BC3C
:10187000662010BD946B0020F8B503782F2B00AFC5
:1018800006466BD0514CD4F8B45045B902203AF01A
:1018900006FB4F49054643F00DFFC4F8B4502846F7
:1018A00044F0BAF90446304644F0B6F92044023018
:1018B0003AF0F5FA0446284644F0AEF929460246C5
:1018C00020463AF0C2FB284644F0A6F9054638B156
:1018D000231813F8012C2F2A1EBF2F2201351A704E
:1018E000304644F099F93146421C60193AF0ADFB9C
:1018F000204644F091F900222146134615469042B5
:101900002ED145B39B00073323F00703ADEB030D46
:10191000204644F081F900236E46651E2044194696
:101920001A4615F801EF04F801E0BEF12F0F01F19E
:10193000010C02D0BEF1000F45D1012B2FD115F8BB
:10194000013C2E2B3AD1531E56F823100023A842F7
:10195000E7D1002363542046BD46F8BD1D4D9EE7E8
:1019600011F8016B02F1020E2F2E08BF01337045F2
:1019700002F1010C0FD92F2E0DD10E782E2E0AD187
:101980004E782E2E07D10332904206D08A782F2A25
:1019900008BF45F001056246B1E70125FBE7022BD0
:1019A0000CD115F8013C2E2B08D115F8023C2E2B3A
:1019B00004D1012A88BF02F1FF32C4E746F822C0F1
:1019C00061460132C2E701336146C0E7946B0020F3
:1019D0008C8207008ED2070070B50E4C0E1805469B
:1019E0004FF48071204641F0FFFC01232360B54293
:1019F00002D10120606070BDD4F80031002BFBD013
:101A00004FF48071204641F0EFFCD4F8083505F81A
:101A1000013BECE700D000402DE9F74F04469DF86C
:101A200030A00F4690469BB169494FF00009012252
:101A300047F6FB70B1FBF2F6B6FBF3F6351F8542B5
:101A400008D909F10109B9F1080F4FEA4202F1D1B1
:101A500002209FE05F4900258B460A68D2F8000506
:101A6000C00740F1A580BAF1000F40F09A80D2F88B
:101A70000805864240F09580D2F80C05814540F07B
:101A80009080504600F5AC7C52F82CC0BCF1FF3F72
:101A900040F0838040B262600125227AE76060F303
:101AA0000602227238790193FEF77AFD019B636189
:101AB000237A6AF3C7132372E368187920F07EFA59
:101AC00063680022C3F80025002D51D16368424AA3
:101AD000934272D002F5A042934270D002F5805238
:101AE00093426ED002F5304293426CD103205BF8F2
:101AF000203000250222C3F80055C3F80455C3F86E
:101B000010254FF4FA42C3F81455C3F80C55C3F826
:101B10000825324A844602EBC000C3F820054FF482
:101B2000004022F83C00042102EBCC02C3F824154B
:101B30004FF0FF31C3F828555080C3F82C559080E2
:101B4000C3F84055D080C3F84455C3F84855C3F88E
:101B50004C55C3F86015C3F86415C3F86815C3F88D
:101B60006C156368C3F80C95C3F80455C3F8086591
:101B7000237A6268397903F07F0303F5AC7320465A
:101B800042F8231063680122C3F80025414635F06E
:101B90003CFF002003B0BDE8F08F013004287FF443
:101BA00071AF0135042D01F104017FF456AF00221D
:101BB000626052B1002005466FE7284697E7012092
:101BC00095E7022093E7FF2091E70320E2E700BFBB
:101BD0000024F400BC1A090000C001405472002027
:101BE00070B5C3680446187920F0C8F962681F4BC5
:101BF0009A4232D003F5A0439A4230D003F5805385
:101C00009A422ED003F530439A422CD10323217AF5
:101C1000174E01F07F01F05C01258D4020EA0500A0
:101C200001F5AC71F05400234FF0FF30636042F8CF
:101C3000210003F5AC7152F82110013105D10133B7
:101C4000042BF6D10023C2F80035E36813B11879EC
:101C500026F0B8FF0023E36070BD0023D7E701231F
:101C6000D5E70223D3E74FF0FF33D0E700C00140B0
:101C7000BC77002008B503280DD8DFE800F00E027D
:101C8000060940F2FA3010F0CFFA4FF44870FAE744
:101C900002482EF057F90248FBE708BDC8F80700D4
:101CA0007CF7070010B50446002024F0E3F9064B4A
:101CB0005A68064B800A40EA8150D31821461844DE
:101CC000BDE810402CF098BD087A002080436D38A4
:101CD00008B502484FF400712EF062F99AF9070036
:101CE00010B5114A1346044653F8F81F11B91620CF
:101CF0002EF006F918688168A14210D1C1681960F8
:101D0000D2F8F430984202D10023C2F8F430002314
:101D1000BDE810401A4640F2F7413CF0CDBBC16827
:101D200000F10C03E2E700BF946B002030B52DED0D
:101D3000068B044683B008302BF092FBAB4BD3EDFF
:101D4000007A04F10C0020EE279A2BF089FB23790E
:101D5000032BB0EE408A40F2A18004F110002BF07A
:101D60007FFBF0EE408A04220DEB020104F1140027
:101D70008DED019A3AF055F9002800F0928084ED3B
:101D8000059A002504220DEB020104F118008DEDE7
:101D9000018A3AF046F910B184ED068A0025042242
:101DA0000DEB020104F11C00CDED018A3AF039F986
:101DB000002878D0C4ED078ADFED8D7A9FED8D5A2B
:101DC0002379FFEE006AE9EE276A052BDFED8A7AB8
:101DD00026EEA66AB8EE000A66EE865A26EE257A48
:101DE00027EE277A66EE067A67EE857A9FED835AAC
:101DF000E6EE057A9FED826A77EE867A9FED816A3C
:101E0000A5EE867A9FED806AA6EE867A77EE876ADF
:101E100077EEC77A38EE087A87EE878AF7EE007A8F
:101E200061D0062B00F09F80042B47D0022B78EE68
:101E3000275A26EE800A37EEC8AA3AD0032B00F0C4
:101E4000CE80012B0CBF76EEA79A77EEE69AB6EE1F
:101E5000008A0ABF29EE888A29EE888AF1EE699AFB
:101E6000B0EE489AC7EEA58A20EE280A34F0D0FEDC
:101E70002AEE280A206234F0CBFE28EE280A60629F
:101E800034F0C6FE29EEA80AA06234F0C1FE29EEA5
:101E9000280AE06234F0BCFE206306E0DFED5B8AD6
:101EA00061E701256EE7002D86D003B0BDEC068BFF
:101EB00030BDDFED569AB1EE489AD3E788EE28AAF6
:101EC000B0EE677AA8EE887A26EE800AB0EE679ABE
:101ED000A8EEC89A7AEE275AF0EE409A37EECAAAD0
:101EE000B0EE478ABEE74A4B18EE902AF6EE005A4B
:101EF000A3EB520306EE103A68EEA55AB7EE087A45
:101F000065EE865A38EEA75AA6EE657AB0EE459A87
:101F100027EE067A38EEE76A27EE287AA6EE669A6A
:101F2000F0EE469AB0EE45AAA6EE26AAE5EE669A2F
:101F300037EE077A78EEA85AF0EE494AA5EE266AFF
:101F4000A7EE489A69EEA59AF0EE4A5AE7EE084ADB
:101F5000E7EE085A29EE289A26EE000AA7EE48AACC
:101F600024EEA88A7EE72A4B18EE902AF6EE005A55
:101F7000A3EB520306EE103A68EEA55AB7EE087AC4
:101F800065EE865A38EEA75AA6EE657AB0EE459A07
:101F900027EE067A38EEE76A27EE287AA6EE269A2A
:101FA00037EE077AB0EE45AAA6EE66AAF0EE469A9C
:101FB000F0EE494AE5EE269AA7EE489AA5EE666A43
:101FC00028EE800AF0EE4A5A69EE809AE7EE084A57
:101FD000E7EE085A29EE289A36EE060ABEE7F0EE3A
:101FE000409AB0EE679AB0EE678A3BE7187000201F
:101FF00083F9A23FEA95323C8964E1BAB3375FBE08
:102000009503353F6AC9693DE42B0EBF000000000F
:10201000DF59375F70B504462DED048B10302BF07F
:102020001FFA404BD3ED007A04F11C0020EE279AF2
:102030002BF016FA94ED088A257B39EE088AF0EE2B
:10204000408A38EE008A002D64D0DFED377AB4EE96
:10205000E79AF1EE10FA59DDDFED347AB4EEE78A53
:10206000F1EE10FAC8BFB0EE678AE66A731B07EE9E
:10207000903AF8EEE77A78EE688A27EE888AC4ED1F
:10208000088AB0EE480A08F027FEFCEEC07AA16A82
:1020900017EE903A31F9132008EE902A627BF8EEA1
:1020A000E88AD2B1F8EE677A5A1C964238EE678A0F
:1020B00003D1002D14BF1A46002231F9123007EE69
:1020C000903AF8EEE77AB7EE007A37EE487A67EEA4
:1020D000887AE7EE287AF0EE678A04F114002BF094
:1020E000BFF904F11800B0EE409A2BF0B9F96FF087
:1020F0000E00B0EE408AB0EE680A0CF07FFDA0EE54
:10210000098AB0EE480ABDEC048B70BDADD5F4EE83
:10211000C87AA5E7B0EE480A08F0DEFD38EE408A3E
:10212000A3E700BF1C7000200000000000FE7F3FFE
:1021300010B504462DED028B0C302BF091F9237E67
:102140000D2BF0EE408A06D1B0EEC08AB0EE480A00
:10215000BDEC028B10BD04F110002BF081F904F1ED
:102160001400B0EE408A2BF07BF9237E0C2B00F29A
:10217000D880DFE803F0070C1116363B533E5F7E34
:102180009BBDCC0038EE888A38EE008ADEE738EE58
:10219000888A38EE408AD9E728EE888A28EE008AB5
:1021A000D4E7F0EEC07AF4EE677AF1EE10FA13D6C7
:1021B0009FED5F7AF4EE477AF1EE10FA0CDC9FEDBA
:1021C0005D7AF4EEC77AF1EE10FA05DAB5EE400A60
:1021D000F1EE10FA00F0A58068EE888A88EE808A19
:1021E000B4E7A8EE880AB0EE408AAFE738EE888AF6
:1021F000D4E7B5EEC00AF1EE10FA06D4F7EE007A95
:10220000B4EEE70AF1EE10FA11DCDFED4B7AF4EEF2
:10221000C07AF1EE10FAC8BFB0EE670AF7EE007AA6
:1022200077EEC07A20EE088AA7EEA88A8EE7B0EE95
:10223000670AF3E7F0EEC87AF4EE677AF1EE10FA87
:1022400012D69FED3B7AF4EE477AF1EE10FA0BDCF2
:102250009FED387AF4EEC77AF1EE10FA04DAB5EEB3
:10226000408AF1EE10FA5CD0C8EE887A37EE808AA8
:102270006CE7F0EEC07AF4EE677AF1EE10FA12D65F
:102280009FED2B7AF4EE477AF1EE10FA0BDC9FED1E
:10229000297AF4EEC77AF1EE10FA04DAB5EE400AC4
:1022A000F1EE10FA3DD078EE888A97E7F4EEC88A0E
:1022B000F1EE10FA0FD5B4EEC08AF1EE10FA3FF548
:1022C00045AFB4EEE80AF1EE10FAD4BFB0EE688A7A
:1022D000B0EE408A3AE7F4EEC08AF1EE10FA23D469
:1022E000B4EEC08AF1EE10FAD8BFB0EE408A2DE706
:1022F000B4EEC80AF1EE10FAD8BFB0EE408AB4EEE0
:10230000E88AF1EE10FAC8BFB0EE688A1EE7B4EEB4
:10231000C08AF1EE10FAD8BFB0EE408AF4EEC88A57
:10232000EFE79FED058A11E7B0EE688A0EE700BF80
:10233000FFFF7F7F00008000000000007FB50C469B
:10234000E107054617D4A20720D12268234B9A4201
:102350001CD14268E36B9A4207D0216AE2630E29DE
:1023600003D004F174002BF0A1F81022002104F135
:102370002C0039F0ABFE20462FF0AAFF0E210246BA
:10238000284604B0BDE8704043F0F7BF69462046D8
:1023900013F056FD0646304613F016FF08B904B098
:1023A00070BD2FF095FFC307044610D46A68C36B55
:1023B0009A4206D0016AC2630E2902D074302BF013
:1023C00075F81022002104F12C0039F07FFE22461E
:1023D0000E21284643F0D1FFDDE700BF98520800E8
:1023E00030B5CA07044685B0084605D48B070DD121
:1023F0000A680F4B9A4209D12FF06AFF0E2201465C
:10240000204605B0BDE8304043F0B7BF694613F041
:1024100017FD0546284613F0D7FE08B905B030BDB4
:102420002FF056FF0E220146204643F0A6FFF1E7AB
:1024300098520800F8B5184B1B7D06460D4603F070
:10244000FF0433BB154B164F187000282246154861
:1024500042F6062108BF0E2714F0CAFB00B1476000
:102460001EB10F4B00221A7301240F4B0D480F4E63
:102470001D70002D4FF0000242F6263108BF0E26D7
:1024800014F0B6FB00B146600DB1084B1C7301207F
:10249000F8BD0020FCE700BFF8600020E3790020D1
:1024A0007C210020A0210020E47900208C21002044
:1024B000F8B5174B1C7D07460D463CBB16F050FC8B
:1024C00011284FEA600304D94FF4337108200FF04C
:1024D00069FF104E3360104B1D70104D04F0FF0467
:1024E00033689C4203DB2EF061FE0120F8BD6100E1
:1024F000042241F00101384617F09AFF58220146A4
:10250000284639F0A2FD01345835E9E70020EDE70F
:10251000F86000207C6F0020AA7700202867002048
:1025200070B51646C2072DED028B04460D4609D440
:10253000830703D10268194B9A4203D020463BF02F
:10254000BDF9E0B1204615F0C7FC2846B0EE408A40
:1025500015F0C2FC3046F0EE408A15F0BDFCB4EE3A
:10256000E88AF1EE10FA06D4B4EEC08AF1EE10FA61
:10257000CCBF35462546BDEC028B284670BD3146A2
:102580000222204600F036F8BDEC028B0146032201
:102590002846BDE8704000F02DB800BFF0E4070009
:1025A0007FB506460D4600F025F80446F00709D42D
:1025B000B10703D132680E4B9A4203D030463BF04C
:1025C0007DF990B1EA0709D4AB0703D12A68084B1B
:1025D0009A4203D028463BF071F930B16946204653
:1025E00013F02EFC13F0F0FD0446204604B070BD3D
:1025F000F0E407002DE9F04F0C4689B00021924627
:102600001DF082F90021834620461DF07DF94FF030
:102610000008059008208DF81F8039F022FC8146C3
:10262000082039F01EFC0746082039F01AFC0599ED
:10263000CDE9007006464B460DF11F02584640F0AA
:1026400001FC059910B9B7482DF0A2FCBAF1000FB2
:102650000CD10223CDE901639DF81F2000974B4662
:1026600058463CF0DFFA09B0BDE8F08FBAF1010F2F
:1026700001D10523EEE79BF80430DBF81C50CC6950
:10268000422B40F0B8810A79422A4FD149469DF841
:102690001F0040F084FDBAF1020FD0F81C9022D147
:1026A0004FF0000C227829788A4228BF0A4689F820
:1026B000002082690169D6F804E091440CF1010C14
:1026C0007A68614515447444ECD83B6801FB1232CA
:1026D0001544326801FB1E221444C26808F1010847
:1026E0004245DDD8BFE74FF0000C227829788A42B6
:1026F00038BF0A4689F8002082690169D6F804E0EB
:1027000091440CF1010C7A68614515447444ECD88D
:102710003B6801FB12321544326801FB1E2214444F
:10272000C26808F101084245DDD89CE7622A52D10F
:1027300049469DF81F00682240F031FDBAF1020FB2
:10274000D0F81C9023D14FF0000C94F90020297888
:102750008A42A8BF0A46A9F8002082690169D6F812
:1027600004E091440CF1010C7A686145154474440D
:10277000EBD83B6801FB12321544326801FB1E2284
:102780001444C26808F101084245DCD86BE74FF0F9
:10279000000C94F9002029788A42B8BF0A46A9F8AB
:1027A000002082690169D6F804E091440CF1010C23
:1027B0007A68614515447444EBD83B6801FB1232DA
:1027C0001544326801FB1E221444C26808F1010856
:1027D0004245DCD847E7482A4FD149469DF81F00BB
:1027E00040F0DDFCBAF1020FD0F81C9022D14FF07E
:1027F000000C228829788A4228BF0A46A9F80020BE
:1028000082690169D6F804E091440CF1010C7A6800
:10281000614515447444ECD83B6801FB1232154401
:10282000326801FB1E221444C26808F101084245C7
:10283000DDD818E74FF0000C228829788A4238BF8B
:102840000A46A9F8002082690169D6F804E091449B
:102850000CF1010C7A68614515447444ECD83B686E
:1028600001FB12321544326801FB1E221444C26877
:1028700008F101084245DDD8F5E6682A54D14946F9
:102880009DF81F0040F08BFCBAF1020FD0F81C90AD
:1028900023D14FF0000CB4F9002029788A42A8BF58
:1028A0000A46A9F8002082690169D6F804E091443B
:1028B0000CF1010C7A68614515447444EBD83B680F
:1028C00001FB12321544326801FB1E221444C26817
:1028D00008F101084245DCD8C5E64FF0000CB4F918
:1028E000002029788A42B8BF0A46A9F800208269E8
:1028F0000169D6F804E091440CF1010C7A68614555
:1029000015447444EBD83B6801FB1232154432681D
:1029100001FB1E221444C26808F101084245DCD8BC
:10292000A1E600BFF8E80700662A40F0F1874946B3
:102930009DF81F0040F033FCBAF1020FD0F81C9054
:102940004FF000022BD14FF0000E2B78D4ED007A1F
:1029500007EE103AF8EEC76AF4EEE76AF1EE10FA05
:1029600001D5F8EE477AC9ED007A8169D0F810C038
:10297000D6F8048089440EF1010E7968F4450D44BF
:102980004444E2D83B680CFB11310D4431680CFB28
:1029900018110C44C16801329142D4D863E64FF05B
:1029A000000E2B78D4ED007A07EE103AF8EEC76AE5
:1029B000F4EEE76AF1EE10FA01DDF8EE477AC9EDC0
:1029C000007A8169D0F810C0D6F8048089440EF1ED
:1029D000010E7968F4450D444444E2D83B680CFB91
:1029E00011310D4431680CFB18110C44C1680132DF
:1029F0009142D4D837E6622B40F0C2810A79422A4C
:102A000052D149469DF81F00682240F0C8FBBAF138
:102A1000020FD0F81C9023D14FF0000C227895F9CA
:102A200000108A42A8BF0A46A9F8002082690169FD
:102A3000D6F804E091440CF1010C7A686145154424
:102A40007444EBD83B6801FB12321544326801FB39
:102A50001E221444C26808F101084245DCD802E68F
:102A60004FF0000C227895F900108A42B8BF0A4650
:102A7000A9F8002082690169D6F804E091440CF1BC
:102A8000010C7A68614515447444EBD83B6801FB3E
:102A900012321544326801FB1E221444C26808F148
:102AA00001084245DCD8DEE5622A53D149469DF84B
:102AB0001F0040F074FBBAF1020FD0F81C9024D133
:102AC0004FF0000C94F9002095F900108A42A8BF3D
:102AD0000A4689F8002082690169D6F804E0914429
:102AE0000CF1010C7A68614515447444EAD83B68DE
:102AF00001FB12321544326801FB1E221444C268E5
:102B000008F101084245DBD8ADE54FF0000C94F91F
